:100000000C94AD180C94E6180C94E6180C94E618B1
:100010000C949F8A0C949F8A0C949F8A0C949F8ABC
:100020000C94E6180C94E6180C94E6180C94E61858
:100030000C94E6180C9485710C94E6180C94E61850
:100040000C94E6180C94B66F0C94EACD0C94E61858
:100050000C940A400C9400400C94E6180C94E6189A
:100060000C94E6180C94E6180C94E6180C94E61818
:100070000C94E6180C94E6180C94E6180C94E61808
:100080000C94B9330C94E6180C94E61805A84CCDE2
:10009000B2D44EB93836A9020C50B9918688083CC2
:1000A000A6AAAA2ABE000000803F4E414E494E49F2
:1000B0005459494E46CDCCCC3D0AD7233C17B7D135
:1000C0003877CC2B329595E6241FB14F0A000020DB
:1000D000410000C84200401C4620BCBE4CCA1B0E5A
:1000E0005AAEC59D7400407A10F35A00A0724E18A3
:1000F000090010A5D4E80000E87648170000E40BDA
:1001000054020000CA9A3B000000E1F5050000809F
:10011000969800000040420F000000A086010000F9
:1001200000102700000000E8030000000064000049
:100130000000000A00000000000100000000002C88
:1001400076D888DC674F0823DFC1DFAE59E1B1B74D
:1001500096E5E3E453C63AE651997696E8E6C2841A
:1001600026EB898C9B62ED407C6FFCEFBC9C9F4032
:10017000F2BAA56FA5F490055A2AF75C936B6CF957
:10018000676DC11BFCE0E40D47FEF520E6B500D02D
:10019000ED902E0300943577050080841E08000042
:1001A000204E0A000000C80C333333330F986E1210
:1001B000831141EF8D2114893BE65516CFFEE6DB16
:1001C00018D1844B381BF77C1D901DA4BBE4242060
:1001D0003284725E228100C9F124ECA1E53D2743FF
:1001E0004F4D4D554E49434154494F4E004452598D
:1001F00052554E004552524F525300494E464F0001
:100200004543484F0053544F505045442E20005012
:1002100072696E7465722073746F707065642064A7
:10022000756520746F206572726F72732E20466937
:100230007820746865206572726F7220616E642028
:10024000757365204D39393920746F207265737468
:100250006172742E202854656D70657261747572B8
:10026000652069732072657365742E205365742050
:10027000697420616674657220726573746172744A
:10028000696E67290A004E6F20436865636B73755A
:100290006D2077697468206C696E65206E756D627B
:1002A00065722C204C617374204C696E653A200095
:1002B0004E6F20436865636B73756D207769746852
:1002C000206C696E65206E756D6265722C204C61C4
:1002D0007374204C696E653A2000636865636B73C4
:1002E000756D206D69736D617463682C204C61734A
:1002F00074204C696E653A20004C696E65204E751D
:100300006D626572206973206E6F74204C61737426
:10031000204C696E65204E756D6265722B312C2004
:100320004C617374204C696E653A20004D31313058
:100330000053657269616C20737461747573206D0C
:1003400069736D617463680A005344207265616467
:10035000206572726F720A002121204B494C4C209B
:1003600063617573656420627920746F6F206D75A9
:10037000636820696E6163746976652074696D6570
:10038000202D2063757272656E7420636F6D6D61D0
:100390006E643A20004D6564696120496E73657230
:1003A00074656400627573793A2070617573656471
:1003B00020666F7220696E7075740A0062757379B9
:1003C0003A2070617573656420666F72207573657D
:1003D000720A00627573793A2070726F6365737385
:1003E000696E670A00506C656173652052657365BC
:1003F00074005052494E5445522048414C54454493
:100400000025533A202553004B494C4C45442E209F
:10041000005072696E7465722068616C7465642E38
:10042000206B696C6C28292063616C6C6564210AFF
:100430000053544F505045442E20005072696E7442
:1004400065722073746F70706564206475652074C4
:100450006F206572726F72732E20466978207468FF
:1004600065206572726F7220616E642075736520FD
:100470004D39393920746F20726573746172742E2E
:10048000202854656D70657261747572652069739A
:100490002072657365742E20536574206974206121
:1004A000667465722072657374617274696E67290F
:1004B0000A006563686F3A004572726F723A004FC6
:1004C0004646004F4E0042696C696E656172204C71
:1004D0006576656C696E6720477269643A0A002127
:1004E000212053544F502063616C6C656420626519
:1004F0006361757365206F6620424C546F75636845
:10050000206572726F72202D20726573746172742F
:100510002077697468204D3939390A002121205328
:10052000544F502063616C6C656420626563617533
:100530007365206F6620424C546F75636820657246
:10054000726F72202D2072657374617274207769E6
:100550007468204D3939390A0050726F62696E67CC
:1005600020506F696E740025532025692F2569007E
:100570002E0A002F0050726F62696E67206D6573DE
:100580006820706F696E74200020284452595255BB
:100590004E2900473239204175746F20426564202E
:1005A0004C6576656C696E67003F20284C2C522C98
:1005B000462C4229206F7574206F6620626F756E1D
:1005C00064732E0A003F2856296572626F73652096
:1005D0006C6576656C20696D706C61757369626CB1
:1005E000652028302D34292E0A00426164205A20CB
:1005F00076616C75650A004E6F2062696C696E6584
:10060000617220677269640A004732384C300044D6
:100610006576696174696F6E0025533A2025730011
:1006200046696E6973686564210A003A207A3A2047
:1006300000206F662000476F696E6720746F3A2054
:10064000580043570A00206469723A0020616E67BF
:100650006C653A00537461727420726164697573D9
:100660003A004D343820506F696E740025533A209B
:1006700025642F256400506F736974696F6E696E0D
:1006800067207468652070726F62652E2E2E0A00D6
:100690003F4C656773206F66206D6F76656D656E84
:1006A0007420696D706C61757369626C65202830A7
:1006B0002D3135292E0A003F2028582C5929206F2A
:1006C0007574206F6620626F756E64732E0A005019
:1006D000726F6265206F7574206F6620626F756E31
:1006E0006473003F53616D706C652073697A652097
:1006F0006E6F7420706C61757369626C652028344C
:100700002D3530292E0A004D3438205A2D50726F65
:100710006265205265706561746162696C697479A3
:1007200020546573740A003F2856296572626F73FE
:1007300065206C6576656C20696D706C6175736998
:10074000626C652028302D34292E0A005374616EA6
:100750006461726420446576696174696F6E3A20E1
:10076000002052616E67653A2000204D61783A2082
:1007700000204D696E3A2000205369676D613A2070
:10078000004D65616E3A200020204D3230312058F6
:10079000004D617820416363656C65726174696FB7
:1007A0006E2028756E6974732F7332290020204DD6
:1007B0003230332058004D6178206665656472617F
:1007C0007465732028756E6974732F732900205225
:1007D0000020204D323034205000416363656C6549
:1007E000726174696F6E2028756E6974732F73322D
:1007F000292028503C7072696E742D616363656CAA
:100800003E20523C726574726163742D616363654E
:100810006C3E20543C74726176656C2D6163636537
:100820006C3E2900204A0020540020530020204D17
:10083000323035204200416476616E636564202861
:10084000423C6D696E5F7365676D656E745F746958
:100850006D655F75733E20533C6D696E5F666565BF
:1008600064726174653E20543C6D696E5F747261A0
:1008700076656C5F66656564726174653E204A3CAE
:100880006A756E635F6465763E29002044002049E6
:100890000020204D333031205000486F74656E6465
:1008A00020504944002E0A00206E6F742064697342
:1008B00061626C65642E205368617265642077699B
:1008C00074680020496E76616C6964206578747282
:1008D000756465722000536C6565702E2E2E005A6B
:1008E0002050726F62652050617374204265640A03
:1008F000005A2050726F6265205061737420426507
:100900006400205A3A200020593A200042656420B1
:10091000583A20004D65736820706F696E74206FBF
:100920007574206F662072616E67650A00436C699A
:10093000636B20746F20526573756D652E2E2E00CB
:10094000616C736F20656E61626C6564290A004E8C
:100950006F204D6F76652E004E6F206D6564696166
:100960000A00456E642066696C65206C6973740AC0
:1009700000426567696E2066696C65206C697374F6
:100980000A00286E6F2066696C6529004E6F74201E
:100990005344207072696E74696E670A0053442074
:1009A0007072696E74696E672062797465200043A5
:1009B000757272656E742066696C653A20002E0A45
:1009C0000044656C6574696F6E206661696C65646E
:1009D0002C2046696C653A200046696C6520646588
:1009E0006C657465643A002569730025696D20257E
:1009F0006973002569682025696D202569730025C4
:100A00006964202569682025696D202569730025A2
:100A1000697920256964202569682025696D20256C
:100A20006973005072696E742074696D653A2000B4
:100A30006F6B006F6666000002FB01F401ED01DFE1
:100A40000144454255473A004D31313220536875D3
:100A500074646F776E004D3131332053004D6567FC
:100A600061205A65726F204F46462E00434F4E4616
:100A700049475F4558504F5254004D4541545041ED
:100A8000434B00434F4F4C45525F54454D504552E8
:100A90004154555245004348414D4245525F5445EB
:100AA0004D504552415455524500424142595354CC
:100AB000455050494E470041524353004D4F544911
:100AC0004F4E5F4D4F44455300544845524D414CA5
:100AD0005F50524F54454354494F4E00455854457A
:100AE0004E4445445F4D3230004C4F4E475F4649BF
:100AF0004C454E414D45004155544F5245504F5283
:100B0000545F53445F5354415455530053445F570B
:100B100052495445005245504541540053444341C5
:100B200052440050524F4D50545F535550504F5205
:100B30005400484F53545F414354494F4E5F434F15
:100B40004D4D414E445300454D455247454E435946
:100B50005F50415253455200434153455F4C494712
:100B600048545F4252494748544E45535300544FEE
:100B700047474C455F4C494748545300534F4654F0
:100B8000574152455F504F574552004255494C44DA
:100B90005F50455243454E54004C4556454C494ED6
:100BA000475F44415441005A5F50524F4245005202
:100BB000554E4F5554004155544F4C4556454C00E9
:100BC0005052494E545F4A4F420050524F4752458F
:100BD0005353004155544F5245504F52545F544562
:100BE0004D50004155544F5245504F52545F504F55
:100BF0005300564F4C554D455452494300454550BE
:100C0000524F4D0042494E4152595F46494C455F53
:100C10005452414E534645520053455249414C5F50
:100C2000584F4E5F584F4646004649524D57415225
:100C3000455F4E414D453A4D61726C696E20322ED2
:100C4000302E392E332D6B616431202844656320AA
:100C5000323720323032312031333A34373A323879
:100C60002920534F555243455F434F44455F5552EA
:100C70004C3A6769746875622E636F6D2F6B61649F
:100C80002F4D61726C696E2050524F544F434F4C40
:100C90005F56455253494F4E3A312E30204D414315
:100CA00048494E455F545950453A4D656761205A51
:100CB00065726F2045585452554445525F434F5515
:100CC0004E543A3120555549443A64626663636430
:100CD00035352D656262612D343631352D616264A2
:100CE000372D3139366161343338663330340A0098
:100CF0002F2F004D31343520533C696E6465783EAA
:100D0000206F7574206F662072616E6765202830D1
:100D10002D31290A003F4A206F7574206F662072BA
:100D2000616E67652028302E303120746F20302EA0
:100D300033290A0020580020204D61783A200020F5
:100D40000020204D696E3A2000203B200020204DDD
:100D500032313120530046523A0020466C6F773AC8
:100D60002000206F7574206F662072616E67650ABF
:100D700000536572766F20003A200020536572762A
:100D80006F200050726F6265204F66667365742035
:100D90005A0050726F6265204F6666736574205A00
:100DA0000064697300656E0043290A0061626C6526
:100DB0006420286D696E2074656D702000436F6C2F
:100DC00064206578747275646573206172652000B3
:100DD0004F46460A00466164652048656967687445
:100DE0002000426564204C6576656C696E67200062
:100DF0004661696C656420746F20656E61626C6524
:100E000020426564204C6576656C696E670A00490E
:100E10006E76616C6964206D6573682E0A004D34CE
:100E2000323120696E636F72726563742070617213
:100E3000616D657465722075736167650A004D6543
:100E4000736820706F696E74206F7574206F6620F0
:100E500072616E67650A00454550524F4D204F4BF9
:100E60000A00290A0020746F20003F5A206F757411
:100E7000206F662072616E6765202800290A0020B5
:100E8000746F20003F59206F7574206F6620726167
:100E90006E676520282D00290A0020746F20003F0E
:100EA00058206F7574206F662072616E6765202808
:100EB0002D004D383400446F6E65207072696E7479
:100EC000696E672066696C650A004D3737004D33DF
:100ED0003100496E76616C6964206578747275645E
:100EE00065720A004361703A00203B0020204D38B3
:100EF00035312058005A2D50726F6265204F66665A
:100F000073657400436F6F6C696E672E2E2E0048F8
:100F1000656174696E672E2E2E00453120255300C1
:100F200020573A0023646566696E65204445464152
:100F3000554C545F004B6420004B6920004B7020DF
:100F400000504944204175746F74756E6520666960
:100F50006E6973686564212050757420746865201B
:100F60006C617374204B702C204B6920616E64207F
:100F70004B6420636F6E7374616E74732066726F5E
:100F80006D2062656C6F7720696E746F20436F6EA1
:100F900066696775726174696F6E2E680A005049E0
:100FA00044204175746F74756E65206661696C6567
:100FB00064212074696D656F75740A00504944207E
:100FC0004175746F74756E65206661696C65642126
:100FD0002054656D706572617475726520746F6FF1
:100FE00020686967680A00504944204379636C654A
:100FF000730025532025692F256900204B643A2072
:1010000000204B693A2000204B703A200020436CAE
:10101000617373696320504944200A002054753A73
:101020002000204B753A2000206D61783A20002086
:101030006D696E3A200020643A2000206269617375
:101040003A20005761697420666F72206865617488
:101050002075702E2E2E00504944204175746F74F7
:10106000756E652073746172740A005049442041A2
:1010700075746F74756E65206661696C6564212096
:1010800054656D706572617475726520746F6F2040
:10109000686967680A00504944204175746F747527
:1010A0006E65206661696C65642120426164206818
:1010B00065617465722069640A0050494420417575
:1010C000746F74756E65004572723A207574663877
:1010D00020666F6E74206E6F7420696E697469612A
:1010E0006C697A65642E004572723A2075746638B0
:1010F00020666F6E74206E6F7420696E697469610A
:101100006C697A65642E004572723A20757466388F
:1011100020666F6E74206E6F7420696E69746961E9
:101120006C697A65642E002568753A2530326875D9
:101130000025303268753A25303268750025303226
:10114000687527253032687500256875642025305C
:101150003268753A25303268750042656400456E24
:10116000636C6F73757265002020202020202000A2
:101170002020202000453A00523A00657272001F7C
:10118000E0201020102010102010202010201030FF
:10119000300840048003001FE03FF03FF03FF01FA5
:1011A000E01FE03FF03FF03FF00FC0078003003F3B
:1011B000FFF038007030FC3020FC10207810203018
:1011C000102C00D02E31D02F7BD02F7BD02E31D0C1
:1011D0002C00D020301020781020FC1030FC30384B
:1011E00000703FFFF03FFFF03800703186302387FA
:1011F000102787902F87D02F03D020301020781011
:101200002078102030102F03D02F87D027879023ED
:1012100087103186303800703FFFF0001DC43F005A
:1012200000000C86198000000D0E198000000F0BC5
:10123000198000000D9F198000000DD399800000D7
:101240001CFBFF0000000000000000000000000088
:1012500000F380001F80007700001980005B1CF6FF
:10126000131DAE5B35AB0635FB5B3DA70CBD9B4B41
:1012700030EB19B19BE39D8E9F9D8E0001E0000035
:10128000000001200000000001E0000000000C0F41
:1012900000FE07022503BB017FFE08FE08FE0508CD
:1012A0000806000040F0C8888898781005080806ED
:1012B0000000C0F88888888888F8050505060001C0
:1012C0002030F830200508080600002070F82020A3
:1012D0002020E00509090600FF2070A8A8B888882A
:1012E0007020070505070001D86C366CD805090980
:1012F0000600FFF8A88888888888A8F8050A0A06E2
:1013000000FE205050505088A8A8887003030306A0
:10131000000340A040FFFFFFFFFFFFFFFFFFFFFFB5
:10132000FFFFFFFFFFFFFFFFFFFFFF0000000605BD
:10133000FF01070706020080808080800080030391
:1013400003060105A0A0A005060606000050F850FF
:1013500050F8500509090600FF2070A8A07028A8C1
:101360007020050707060000C8C81020409898059F
:10137000070706000040A0A040A8906801030306EC
:1013800002058080800309090601FF20404080801B
:10139000804040200309090601FF804040202020B2
:1013A00040408005070706000020A8702070A82094
:1013B0000505050600012020F82020020303060190
:1013C000FFC04080050101060003F8020202060189
:1013D00000C0C0050707060000081010204040802C
:1013E000050707060000708898A8C88870030707DB
:1013F00006010040C040404040E0050707060000ED
:10140000708808102040F8050707060000F808104B
:101410003008887005070706000010305090F8105B
:1014200010050707060000F880F008088870050717
:1014300007060000304080F0888870050707060026
:1014400000F808101020202005070706000070880B
:1014500088708888700507070600007088887808FB
:101460001060020505060100C0C000C0C0020606EB
:101470000601FFC0C000C040800305050601012031
:1014800040804020050303060002F800F80305052C
:101490000601018040204080050707060000708893
:1014A00010202000200507070600007088B8A8B8A3
:1014B0008070050707060000708888F8888888050E
:1014C0000707060000F04848704848F0050707067F
:1014D000000070888080808870050707060000F093
:1014E0004848484848F0050707060000F88080F0A3
:1014F0008080F8050707060000F88080F080808073
:101500000507070600007088808098887005070727
:10151000060000888888F888888803070706010085
:10152000E04040404040E00507070600003810104A
:10153000101090600507070600008890A0C0A090DA
:1015400088050707060000808080808080F80507F6
:101550000706000088D8A88888888805070706003D
:10156000008888C8A8988888050707060000708842
:101570008888888870050707060000F08888F08052
:10158000808005070706000070888888A890680595
:101590000707060000F08888F0A090880507070676
:1015A000000070888070088870050707060000F842
:1015B0002020202020200507070600008888888832
:1015C00088887005070706000088888888505020A2
:1015D00005070706000088888888A8A8500507071F
:1015E00006000088885020508888050707060000FC
:1015F00088885020202020050707060000F80810E2
:10160000204080F80309090601FFE0808080808087
:101610008080E00507070600008040402010100889
:101620000309090601FFE020202020202020E005FA
:1016300003030600052050880501010600FEF8039B
:10164000030306010580402005050506000070081B
:101650007888780507070600008080F0888888F081
:1016600005050506000070808088700507070600E4
:1016700000080878888888780505050600007088C5
:10168000F08070050707060000304840E040404009
:101690000507070600FE7088888878087005070728
:1016A0000600008080F0888888880307070601000C
:1016B0004000C0404040E00409090601FE1000302F
:1016C00010101010906005070706000080808890B9
:1016D000E09088030707060100C04040404040E01A
:1016E000050505060000D0A8A8A8A8050505060060
:1016F00000B0C888888805050506000070888888BD
:10170000700507070600FEF0888888F080800507CE
:10171000070600FE78888888780808050505060011
:1017200000B0C8808080050505060000788070083C
:10173000F00507070600002020F8202020180505E6
:101740000506000088888898680505050600008859
:10175000888850200505050600008888A8A850053F
:10176000050506000088502050880507070600FE82
:1017700088888850204080050505060000F8102064
:1017800040F80309090601FF2040404080404040E6
:10179000200109090602FF8080808080808080808F
:1017A0000309090601FF8040404020404040800579
:1017B000030306000248A890FF5045544700504CD0
:1017C00041005072696E742041626F7274656400EA
:1017D0004D32350050617573696E672E2E2E004DA7
:1017E000323400454550524F4D2056657273696F33
:1017F0006E204572726F7200454550524F4D204920
:101800006E646578204572726F7200454550524F84
:101810004D20435243204572726F72003F0049676A
:101820006E6F726500526573657400496E69746904
:10183000616C697A6520454550524F4D0000FE00AD
:1018400003FF8007C7C00701E00000E00000F000D0
:1018500000700400700E00701F00703F80F00E00DA
:10186000E00F01E007C7C003FF8000FE0000FE009C
:1018700003FF8007C7C00F01E00E00E03F80F01FAC
:1018800000700E00700400700000700000F0000096
:10189000E00701E007C7C003FF8000FE000E000E56
:1018A000000E000E000E000E000E000E007FC03F66
:1018B000801F000E00040004000E001F003F807F08
:1018C000C00E000E000E000E000E000E000E000EE8
:1018D00000FFFFFF7F80FFC0FFC0FFC07F807F80D1
:1018E000FFC0FFC0FFC03F001E000C0050726F62BF
:1018F00065205A204F666673657400200820466193
:101900006374002008204D6178002008204D696E26
:10191000004F6666004F6E004175746F74656D70A0
:1019200000452073746570732F6D6D005A205374D9
:101930006570732F6D6D00592053746570732F6D32
:101940006D00582053746570732F6D6D004164767F
:10195000616E6365642053657474696E67730054C7
:10196000656D70657261747572650053746570732E
:101970002F6D6D00436F6E66696775726174696F74
:101980006E003F004E65787420436F726E65720082
:10199000446F6E65004E65787400486F6D696E67C0
:1019A0002058595A0053746F7265205365747469D6
:1019B0006E6773004C6F61642053657474696E6761
:1019C0007300426564205472616D6D696E670050EA
:1019D000726F6265205A204F6666736574004661B7
:1019E000646520486569676874004F6666004F6EDD
:1019F00000426564204C6576656C696E67004C65D5
:101A000076656C20426564004732394E00473239B2
:101A1000004175746F20486F6D65004D6F74696F7C
:101A20006E0053572D4D6F64650053746F770044FB
:101A300065706C6F790053656C662D546573740026
:101A4000526573657400436F6E6669677572617481
:101A5000696F6E00526573746F72652044656661CC
:101A6000756C7473004C6F61642053657474696E97
:101A700067730053746F72652053657474696E6781
:101A80007300424C546F7563680050726F6265203A
:101A90005A204F666673657400416476616E6365B3
:101AA000642053657474696E6773004D61696E00DC
:101AB0003F004261636B0053746F70004D3232001F
:101AC000417474616368204D65646961004D323111
:101AD000005072696E742066726F6D204D65646986
:101AE000610052656C65617365204D6564696100D4
:101AF000436F6E66696775726174696F6E005465D5
:101B00006D7065726174757265004D6F74696F6E8A
:101B100000526573756D65205072696E740054755E
:101B20006E650053746F70205072696E740050615E
:101B3000757365205072696E7400496E666F20532C
:101B4000637265656E000A4D3234004D32332025D4
:101B500073003F005374617274205072696E740098
:101B600043616E63656C005072696E740043616E10
:101B70006E6F7420656E746572207375626469722D
:101B80003A200002202E2E000152656672657368AD
:101B9000004D61696E002100486F74656E642074A9
:101BA0006F6F20636F6C64004261636B0050726FF3
:101BB00063656564004D6F74696F6E00446973619D
:101BC000626C65205374657070657273004D3834B3
:101BD000004D34382050726F626520546573740074
:101BE0004732384F0A4D3438205031300042656456
:101BF000204C6576656C696E67004175746F20488E
:101C00006F6D6500473238004D61696E00BE17B9CF
:101C100017436F6F6C646F776E0050726568656113
:101C20007420240046616E205370656564004E6F19
:101C30007A7A6C65004D61696E0050726F62652042
:101C40005A204F666673657400466C6F7700466174
:101C50006E205370656564004E6F7A7A6C65005330
:101C600070656564004D61696E00486F6D696E67EF
:101C7000204661696C6564006F70656E005452495E
:101C8000474745524544003A20007A5F70726F62C0
:101C900065007A5F6D696E00795F6D696E00785FCF
:101CA0006D696E005265706F7274696E6720656E43
:101CB0006473746F70207374617475730A00207498
:101CC0006F6F206C6F6E6720657874727573696FC3
:101CD0006E2070726576656E7465640A0020636FAD
:101CE0006C6420657874727573696F6E20707265AC
:101CF00076656E7465640A00486F6D6520257325EE
:101D0000732573204669727374005761726E696E31
:101D1000673A20486F6D696E672042756D70204488
:101D2000697669736F72203C20310A000202040058
:101D300000E0C0000000C000000000000068430098
:101D400000634300007A430000A0400000A0400070
:101D5000000040FFFDFCFAF8F6F4F2F0EEECEAE9E0
:101D6000E7E5E3E1E0DEDCDAD9D7D5D4D2D0CFCDD8
:101D7000CBCAC8C7C5C3C2C0BFBDBCBAB9B7B6B469
:101D8000B3B2B0AFADACAAA9A8A6A5A4A2A1A09ECB
:101D90009D9C9A99989795949392908F8E8D8B8A0B
:101DA0008988878684838281807F7E7D7B7A79782B
:101DB00077767574737271706F6E6D6C6B6A69682B
:101DC00067666564636261605F5E5D5C5B5A59581B
:101DD000585756555453525150504F4E4D4C4B4AF4
:101DE0004A4948474646454443424241403F3E3EB9
:101DF0003D3C3B3B3A39383837363535343332326F
:101E00003130302F2E2E2D2C2B2B2A292928272715
:101E100026252524232322212120201F1E1E1D1CB0
:101E20001C1B1B1A1919181817161615151413133D
:101E300012121111100F0F0E0E0D0D0C0C0B0A0AC1
:101E4000090908080707060605050404030302023A
:101E500001000000000001000000010000800055AA
:101E60005555000000400033333300AAAA2A004928
:101E700092240000002000C7711C0099991900D11C
:101E8000451700555515003BB113002449120011A8
:101E9000111100000010000F0F0F00E3380E004377
:101EA000790D00CCCC0C00C3300C00E8A20B006410
:101EB000210B00AAAA0A00703D0A009DD809004221
:101EC0007B090092240900DCD308008888080010F0
:101ED00042080000000800F0C1070087870700756E
:101EE000500700711C07003EEB0600A1BC0600690C
:101EF00090060066660600703E0600611806001730
:101F0000F4050074D105005BB00500B290050062D5
:101F10007205005555050078390500B81E05000505
:101F20000505004EEC040087D40400A1BD04009018
:101F3000A7040049920400C17D0400EE690400C7B3
:101F4000560400444404005C3204000821040041AB
:101F5000100400000004003FF00300F8E003002636
:101F6000D20300C3C30300CCB503003AA803000AA0
:101F70009B0300388E0300C08103009F750300D0CF
:101F8000690300505E03001D5303003448030091B1
:101F90003D03003333030016290300381F03009765
:101FA000150300300C0300030303000BFA02004981
:101FB000F10200BAE802005CE002002DD802002D18
:101FC000D0020059C80200B0C0020031B90200DAE4
:101FD000B10200AAAA0200A0A30200BC9C0200FA5F
:101FE0009502005C8F0200DF8802008282020045B9
:101FF0007C02002776020027700200436A02007C00
:10200000640200D05E02003F590200C85302000083
:102010000061430000614300007A430000E0C0001B
:102020000000C00000000053657474696E6773207F
:1020300053746F72656400290A00206279746573B5
:102040003B20637263200053657474696E6773206C
:1020500053746F726564202800454550524F4D20DF
:102060006461746173697A65206572726F722E0A99
:1020700000290A002062797465733B206372632033
:10208000002073746F7265642073657474696E6781
:102090007320726574726965766564202800202853
:1020A00063616C63756C6174656429210A00202189
:1020B0003D2000454550524F4D20435243206D690D
:1020C000736D61746368202D202873746F7265646A
:1020D0002920002053697A653A2000496E646578AA
:1020E0003A2000204D61726C696E3D563836290ADF
:1020F00000454550524F4D2076657273696F6E20D2
:102100006D69736D617463682028454550524F4D69
:102110003D0048617264636F646564204465666174
:10212000756C742053657474696E6773204C6F61AD
:102130006465640A000000FA430000FA430000A04E
:10214000400000C8410000A0420000A0420000C8BA
:10215000430080C043F4010000F40100006400006B
:10216000008813000020286D6D2900203B204C655D
:1021700076656C696E67200020204D343230205324
:10218000004175746F20426564204C6576656C690A
:102190006E670020460020480020204D3134352055
:1021A00053004D6174657269616C20686561747576
:1021B0007020706172616D657465727300204A00F1
:1021C0002020473239205720490020204D31343912
:1021D0002043203B20556E69747320696E2043654F
:1021E0006C736975730A0054656D706572617475FE
:1021F000726520556E697473002020473231203B90
:10220000004C696E65617220556E6974730024F428
:10221000D43050C38E20C2A24017828B7011127A24
:10222000910D816CD90AA861E108C7586607615110
:1022300043061E4B5D05C145A7041A411104093D23
:102240009803713931034036DB0265339102D43093
:102250005402802E1D02632CEE01752AC501B028A0
:10226000A001102781018F2564012B244B01E0225E
:102270003401AC211F018D200D01801FFC00841E44
:10228000ED00971DDF00B81CD200E61BC600201B26
:10229000BC00641AB200B219A8000A19A0006A189A
:1022A0009900D117910040178B00B51684003116A4
:1022B0007E00B31579003A157300C7146F005814E7
:1022C0006A00EE1366008813630025135E00C712D0
:1022D0005B006C12570015125400C11151007011AF
:1022E0004F0021114B00D61049008D1047004610B9
:1022F000440002104200C00F4000800F3E00420F19
:102300003C00060F3B00CB0E3800930E37005C0EEE
:102310003500270E3400F30D3200C10D3100900D51
:102320003000600D2E00320D2D00050D2C00D90C53
:102330002B00AE0C2900850C29005C0C2700350C05
:1023400027000E0C2600E80B2400C40B2400A00B71
:1023500023007D0B23005A0B2100390B2100180BA1
:102360002000F80A1F00D90A1E00BB0A1E009D0AA1
:102370001D00800A1D00630A1C00470A1B002C0A6E
:102380001B00110A1A00F7091A00DD091900C40917
:102390001900AB091900920917007B09180063099D
:1023A00017004C09160036091600200916000A0904
:1023B0001500F5081500E0081400CC081400B80852
:1023C0001400A4081400900813007D0812006B0884
:1023D00013005808120046081200340811002308A0
:1023E00011001208110001081100F0071000E007A9
:1023F0001000D0071000C0071000B0070F00A107A1
:10240000100091070E0083070F0074070F00650787
:102410000E0057070E0049070E003B070D002E0760
:102420000E0020070D0013070D0006070D00F9062A
:102430000C00ED060D00E0060C00D4060C00C806EA
:102440000C00BC060C00B0060C00A4060B0099069C
:102450000C008D060B0082060B0077060B006C0645
:102460000B0061060A0057060B004C060A004206E4
:102470000A0038060A002E060A0024060A001A0678
:102480000A001006090007060A00FD050900F40508
:102490000900EB050900E2050900D9050900D0058E
:1024A0000900C7050900BE050900B5050800AD050E
:1024B0000800A50509009C050800940508008C0586
:1024C0000800840508007C050800740508006C05F8
:1024D0000700650508005D050700560508004E0564
:1024E00007004705070040050800380507003105CB
:1024F00007002A050700230507001C05060016052E
:1025000007000F0507000805060002050700FB0489
:102510000600F5040700EE040600E8040600E204E5
:102520000700DB040600D5040600CF040600C9043A
:102530000600C3040600BD040600B7040600B1048B
:102540000500AC040600A6040600A00405009B04D8
:10255000060095040500900406008A040500850421
:102560000500800406007A04050075040500700467
:1025700005006B04050066040500610405005C04A9
:10258000050057040500520405004D0405004804E9
:102590000500430405003E0404003A040500350428
:1025A0000500300404002C04050027040400230463
:1025B00005001E0404001A0404001604050011049A
:1025C00004000D04040009040500040404000004D0
:1025D0000400FC030400F8030400F4030400F00307
:1025E0000400EC030400E8030400E4030400E00337
:1025F0000400DC030400D8030400D4030400D00367
:102600000400CC030400C8030300C503030024F442
:1026100004D9201BC40C5C0E9804C4095F02650732
:102620007101F405F900FB04B30048048700C103FD
:1026300069005803550003034500BE023A008402B6
:10264000310053022A002902250004022000E4017F
:102650001C00C8011900AF01170098011400840183
:102660001300710110006101100051010E004301BF
:102670000D0036010B002B010B0020010B00150192
:1026800009000C01090003010800FB000800F30029
:102690000800EB000700E4000600DE000600D8009A
:1026A0000600D2000600CC000500C7000500C200ED
:1026B0000500BD000400B9000400B5000400B1002D
:1026C0000400AD000400A9000400A5000300A2005E
:1026D00003009F0004009B00030098000300950086
:1026E000020093000300900003008D0002008B00A5
:1026F00003008800020086000200840003008100BD
:1027000002007F0002007D0002007B0002007900D1
:1027100002007700010076000200740002007200DF
:102720000100710002006F0002006D0001006C00EA
:1027300002006A00010069000200670001006600F3
:1027400001006500010064000200620001006100F8
:102750000100600001005F0002005D0001005C00FC
:1027600001005B0001005A000100590001005800FF
:1027700001005700010056000100550001005400FF
:1027800001005300000053000100520001005100FD
:102790000100500001004F0001004E0000004E00FB
:1027A00001004D0001004C0001004B0000004B00F7
:1027B00001004A00010049000100480000004800F3
:1027C00001004700010046000000460001004500EE
:1027D00000004500010044000100430000004300E8
:1027E00001004200000042000100410000004100E1
:1027F0000100400001003F0000003F0001003E00DA
:1028000000003E0001003D0000003D0001003C00D2
:1028100000003C0000003C0001003B0000003B00C9
:1028200001003A0000003A000100390000003900C0
:1028300001003800000038000000380001003700B7
:1028400000003700010036000000360000003600AE
:1028500001003500000035000000350001003400A3
:102860000000340000003400010033000000330099
:10287000000033000100320000003200000032008E
:102880000100310000003100000031000100300083
:10289000000030000000300001002F0000002F0079
:1028A00000002F0000002F0001002E0000002E006D
:1028B00000002E0001002D0000002D0000002D0062
:1028C00000002D0001002C0000002C0000002C0056
:1028D00000002C0001002B0000002B0000002B004A
:1028E00000002B0001002A0000002A0000002A003E
:1028F00000002A0001002900000029000000290032
:102900000000290000002900010028000000280024
:102910000000280000002800000028000100270017
:10292000000027000000270000002700000027000B
:1029300001002600000026000000260000002600FE
:1029400000002600010025000000250000002500F1
:1029500000002500000025000000250001002400E3
:1029600000002400000024000000240000002400D7
:1029700001002300000023000000230000002300CA
:1029800000002300000023000000230001002200BB
:1029900000002200000022000000220000002200AF
:1029A00000002200010021000000210000002100A1
:1029B0000000210000002100000021000000210093
:1029C0000100200000002000000020000000200086
:1029D0000000200000002000000020000000200077
:1029E00001001F0000001F0000001F0000001F006A
:1029F00000001F0000001F0000001F0001001E005B
:102A000000001E0000001E0000001E000000393003
:102A100000003325000087190000B00F0000DB081C
:102A20000000BD040000740200003F0100002043CC
:102A30006F756E7420583A0045310045002C2073A4
:102A4000797374656D2073746F70706564212048AC
:102A500065617465725F49443A2000486561746934
:102A60006E67204661696C65640048656174696ED3
:102A700067206661696C6564004572723A204D4159
:102A80005854454D50004D415854454D5020747296
:102A900069676765726564004572723A204D494EF8
:102AA00054454D50004D494E54454D502074726967
:102AB00067676572656400202F0020403A007C3C07
:102AC0003E5E2B3D3F2F5B5D3B2C2A225C00436129
:102AD0006E6E6F74206F70656E20737562646972BC
:102AE000200053442063617264206F6B0A006F7092
:102AF000656E526F6F74206661696C65640A00765A
:102B00006F6C756D652E696E6974206661696C65A0
:102B1000640A004E6F20534420636172640A002EE1
:102B20000A006F70656E206661696C65642C2046D2
:102B3000696C653A200046696C652073656C656355
:102B40007465640A002053697A653A200046696C0E
:102B500065206F70656E65643A2000454E442053D1
:102B60005542524F5554494E450A002220706F730A
:102B7000002220706172656E743A220053554252F1
:102B80004F5554494E452043414C4C207461726767
:102B900065743A220053756263616C6C204F7665F0
:102BA00072666C6F77004578636565646564206D57
:102BB000617820535542524F5554494E4520646523
:102BC0007074683A00667265736800646F696E6756
:102BD000002066696C653A20004E6F7720005772BE
:102BE0006974696E6720746F2066696C653A2000AD
:102BF0006D61726C696E66772E6F726700322E306F
:102C00002E392E332D6B616431001FFFFFFFFFFF54
:102C1000FF600000000001FF400000000000FF8096
:102C200000000000007F83CF00000C303F87FF8052
:102C3000000C301F867980000C000F8C30C7838C0D
:102C400030E78C30CFC7CC31F38C30DCECEC33B9CF
:102C50008C30D86C6C33198C30D06C0C33198C30B0
:102C6000D86C0C33198C30DC6C0E3B198C30CF7C5B
:102C7000079F198C30C77C038F19400000000000AB
:102C800002600000000000061FFFFFFFFFFFF8705A
:102C9000012C0190012701B0012201C0011D01F0AA
:102CA0000118011002130130020E016002090190A7
:102CB000020401C002FF000003FA004003F5008097
:102CC00003F000D003EB002004E6007004E100E014
:102CD00004DC004005D700C005D2004006CD00D07E
:102CE00006C8008007C3003008BE00F008B900C065
:102CF00009B400B00AAF00B00BAA00D00CA50000C8
:102D00000EA000500F9B00C01096005012910000C2
:102D1000148C00C0158700B0178200B0197D00D058
:102D20001B7800001E730040206E0090226900F0A6
:102D300024640040275F0090295A00E02B550010C2
:102D40002E500020304B0010324600E033410090FE
:102D5000353C001037370070383200A0392D00B0F4
:102D60003A2800A03B2300603C1E00103D19009053
:102D70003D1400103E0F00703E0A00C03E050000EA
:102D80003F0000403FFBFF803FF6FFC03FF1FF20C8
:102D900020506C616E6E657242756666657242792E
:102DA0007465733A20002046726565204D656D6F2D
:102DB00072793A200020436F6D70696C65643A2027
:102DC00044656320323720323032310A00204C61B2
:102DD000737420557064617465643A203230323106
:102DE0002D30392D3033207C20417574686F723A54
:102DF00020286B61642C20416E79637562696320C1
:102E00004D656761205A65726F2041424C20313216
:102E100056290A004D61726C696E20322E302E39AF
:102E20002E332D6B6164310A0020536F6674776115
:102E300072652052657365740A0020576174636877
:102E4000646F672052657365740A002042726F7761
:102E50006E206F75742052657365740A0020457882
:102E60007465726E616C2052657365740A00506FF0
:102E700077657255700A0073746172740A00473284
:102E8000385859004D31303031006572726F722000
:102E900077726974696E6720746F2066696C650A61
:102EA00000446F6E6520736176696E672066696C99
:102EB000652E0A004D323900456E6473746F70736D
:102EC00000255320256320256320256320256300EA
:102ED00020503A00205A3A0020593A0020583A002F
:102EE000656E6473746F7073206869743A200000B3
:102EF0000000010200090A000000000403080700A6
:102F000000000000000000000000000000000000C1
:102F10004D6F76652025736D6D004D6F76652030A1
:102F20002E316D6D004D6F766520316D6D004D6FEA
:102F300076652031306D6D004D6F76652041786982
:102F400073004D6F76652045787472756465720004
:102F50004D6F7665205A004D6F76652059004D6F94
:102F600076652058005072696E742066726F6D200D
:102F70004D6564696100FFFFFF205A3A2000205927
:102F80003A200042656420583A20004D6567612070
:102F90005A65726F2052656164792E005072696EB5
:102FA00074696E672E2E2E005072696E7420506107
:102FB0007573656400220A00556E6B6E6F776E2024
:102FC000636F6D6D616E643A2022006F6B00204567
:102FD00000205A0020590020204D3932205800533B
:102FE000746570732070657220756E6974003B2083
:102FF00000DB0FC93F45BCDA3F8FB30240FCF0272E
:103000004056946140FE4B9B4084A5D840E0231875
:1030100041346A5641E859974164DBD5416E271720
:1030200042B4B75542CE1A9742C8AED542B5885A77
:1030300043D40684BFA65FA7BF7443E0BF10B11A94
:10304000C01C2C58C0E8F697C0B849D6C04E4E17E1
:10305000C124D355C1802497C1A0B5D5C1121A1778
:10306000C244AE55C2781797C26CACD5C267885AB5
:10307000C320746F6F206C6F6E67206578747275F3
:1030800073696F6E2070726576656E7465640A0090
:1030900020636F6C6420657874727573696F6E203D
:1030A00070726576656E7465640A006F6B0A005213
:1030B0006573656E643A200020453A00205A3A0054
:1030C00020593A00583A0000002200250028002B21
:1030D0000000002100240027002A00020202020250
:1030E00002020204040404040404040303030303AB
:1030F00003030301010101010101010102040810A0
:1031000020408001020408102040800102040810C1
:1031100020408080402010080402014572726F72C6
:103120002077726974696E6720746F20454550522C
:103130004F4D210A00544845524D414C2052554EA6
:103140004157415900546865726D616C2052756E2B
:103150006177617900006FDB53E211241FBECFEF6E
:10316000D0E4DEBFCDBF84B78093491514BE0FB63F
:10317000F894A89580916000886180936000109217
:1031800060000FBE12E0A0E0B1E0E2E1F3EE01E08A
:103190000BBF02C007900D92A439B107D9F725E102
:1031A000A4E9B2E001C01D92A934B207E1F718E129
:1031B000CCEAD8E104C02197FE010E945CEECB3A34
:1031C000D107C9F70E942BDC0C947DF10C94000010
:1031D000FC01A081B1811C92A281B3818C918F5F8F
:1031E0008C930280F381E02D90818CE0989F800D7C
:1031F0001124E2E4F3E113AE84AF0895FC0184915D
:103200000895FC0180810895009751F0FC0180E051
:103210009191992331F0907C9038D1F38F5FF8CF62
:1032200080E00895119800C087FD43C0419800C018
:10323000119A00C000C0119800C086FD46C0419898
:1032400000C0119A00C000C0119800C085FD3BC0AD
:10325000419800C0119A00C000C0119800C084FDC0
:1032600030C0419800C0119A00C000C0119800C041
:1032700083FD25C0419800C0119A00C000C011987C
:1032800000C082FD1AC0419800C0119A00C000C061
:10329000119800C081FD0FC0419800C0119A00C074
:1032A00000C0119800C0419800C0119A00C000C031
:1032B0000895419ABCCF419AF0CF419AE5CF419A07
:1032C000DACF419ACFCF419AC4CF419AB9CF90E09B
:1032D00080E00895CF93DF93DB01F9019C91913059
:1032E000C1F0943080F094509C938830D1F4808168
:1032F0009181009771F0019791838083480F591F46
:10330000EA01188206C08C3539F49C5F9C93943096
:1033100041F4DF91CF9108958B3339F781E08C939D
:10332000F8CF20813181B9016F5F7F4F7183608356
:10333000420F531FEA018883808191818F35910567
:103340006CF7E7CF0F931F9381E0009194141091D5
:1033500095142091961430919714409190145091A7
:103360009114609192147091931404171507260715
:10337000370708F480E01F910F91089590E080E0F6
:1033800008952091F703833021F425FD0CC024FD1E
:103390000CC030E0A90102C0559547958A95E2F727
:1033A000CA018170089581E0089580E008958091B8
:1033B000130484FD0BC08091150487FD07C0909114
:1033C0001604937081E019F480E0089581E0089577
:1033D0002FEB280F2A3108F047C0E22FF0E0809150
:1033E000130490911404A0911504B091160404C024
:1033F000B695A795979587952A95D2F780FD02C037
:1034000081700895E750FC4FE081EE2341F18091F7
:10341000610790916207E80FF92FF11D808190ED0F
:10342000980F9A3030F08E3251F4818180538A3077
:1034300098F4F093E803E093E70381E008958D3278
:1034400011F08B3249F4818190ED980F9A3088F316
:103450008E3211F48281EACFF0E0E0E0EACF109200
:10346000E8031092E703E9CF80E00895CF93DF935C
:1034700085E4AEDF882309F188E040911304509180
:1034800014046091150470911604972F9170C92F40
:1034900090E0D92FCC0FDD1F71FB222720F930E0FF
:1034A000220F331F220F331FC22B67FB442740F923
:1034B000C42B8C2BDF91CF91089580E0DECF88DF85
:1034C000882341F081E02091E7033091E803232B2A
:1034D00009F480E00895B0E0A0E0E1E7FAE10C949F
:1034E00080EE6B01E9014A3009F4D5C0453109F09D
:1034F00081C0DB011296ED91FC91F280968187816B
:10350000139A00C00000E6E2F0E03197F0F7092FCF
:10351000182FEF2CE29420EFE22230E1B32EBF0C03
:10352000E80188EF7FDE00C0000086E290E00197AE
:10353000F0F7BFE1BF1508F49BC08F2D807780683E
:1035400071DE8E2D6FDE00C0000086E290E00197F4
:10355000F0F780E867DE80E065DE00C0000086E20C
:1035600090E00197F0F78AEF5DDE00C0000086E290
:1035700090E00197F0F7005F1F4F8881807F52DE57
:1035800089918295807F4EDEC017D107B1F700C0C8
:10359000000086E290E00197F0F7F394E0E1EE0E90
:1035A000FB10BECF1398D6011296ED91FC9180814D
:1035B0009281980F92832181921708F09FC1948184
:1035C0009F5F94839381890F821710F08FEF820F92
:1035D0008383458150E0440F551F70E060E0868191
:1035E00097810E9429F181E0CDB7DEB7E9E00C9424
:1035F0009CEEDEC1FB0102811381423309F485C1D7
:1036000008F48DC1463409F475C1473409F482C108
:103610004B3349F789812B81D80112967C911297FF
:1036200013963C91213009F4BFC1233009F0A0C1A9
:1036300048EF480F582F91E0341708F490E031E03C
:10364000541708F030E0492F432B61E0571708F476
:1036500060E0462311F4932331F2FA8030E0F9015F
:10366000E656FE4FD0802A563E4FF901E08099C1C0
:1036700080EE8F0D8068807FD5DD8F2D8295807FD5
:10368000D1DD00C0000086E290E00197F0F780E80D
:10369000C9DD80E861CF0B9A1398399A4198099A4D
:1036A000119A139A00C0000086E290E00197F0F7AB
:1036B00088E790E0CEE9DFE0FE013197F1F701976E
:1036C000D9F788EFAFDD00C0000086E290E00197F7
:1036D000F0F780E2A7DD80E0A5DD00C0000086E213
:1036E00090E00197F0F780E09DDD80E89BDD00C071
:1036F000000086E290E00197F0F780E093DD80E142
:1037000091DD00C0000086E290E00197F0F7CE0165
:103710000197F1F7CE010197F1F7CE010197F1F78B
:10372000CE010197F1F7CE010197F1F7CE01019794
:10373000F1F7CE010197F1F7CE010197F1F7CE0134
:103740000197F1F7CE010197F1F7CE010197F1F75B
:10375000CE010197F1F7CE010197F1F7CE01019764
:10376000F1F72197F1F780E25DDD80E45BDD00C0D9
:10377000000086E290E00197F0F780E253DD80E6FA
:1037800051DD00C0000086E290E00197F0F7D0E044
:10379000C0E08C2F8077806845DD8D2F43DD00C031
:1037A000000086E290E00197F0F780E83BDD80E0E2
:1037B00039DD00C0000086E290E00197F0F78AEF63
:1037C00031DD00C0000086E290E00197F0F780E272
:1037D000119800C0419800C0119A00C000C0119813
:1037E00000C0419800C0119A00C000C0119800C0EC
:1037F000419800C0119A00C000C0119800C04198C3
:1038000000C0119A00C000C0119800C0419800C0CB
:10381000119A00C000C0119800C0419800C0119AD0
:1038200000C000C0119800C0419800C0119A00C0AB
:1038300000C0119800C0419800C0119A00C000C09B
:10384000119800C0419800C0119A00C000C01198A2
:1038500000C0419800C0119A00C000C0119800C07B
:10386000419800C0119A00C000C0119800C0419852
:1038700000C0119A00C000C0119800C0419800C05B
:10388000119A00C000C0119800C0419800C0119A60
:1038900000C000C0119800C0419800C0119A00C03B
:1038A00000C0119800C0419800C0119A00C000C02B
:1038B00000C00000E6E2F0E03197F0F7815009F037
:1038C00087CF88EFAFDC00C0000086E290E0019770
:1038D000F0F7CF5FD05FC03209F05BCF80E0A2DCB1
:1038E00080ECA0DC00C0000086E290E00197F0F7D9
:1038F000139879CEF8018581888375CE80E0CDB7A5
:10390000DEB7E9E00C949CEE53C0B901C8010E94F7
:1039100034CE69CED80111968C91888364CE44311F
:1039200091F0473109F05FCE1882D80112968C9140
:103930001297898315968C91159781508A831396D7
:103940008C918B8350CED80115964C91159750E0F1
:10395000440F551F70E060E016968D919C910E9477
:1039600029F1F801128280818150838314823BCE39
:10397000381708F438CE871708F435CEFA80E12CD2
:10398000D12C243070F46ACEBE01C8010E9434CE1E
:10399000898198819D0D98838E0D8983FF0C09F490
:1039A00022CEF7FEF6CFF0CF58E0580F482F43CE87
:1039B000EF92FF920F931F93CF93DF93EC018B0154
:1039C0007A018A859B858617970731F088819981CE
:1039D0000E9421D01B870A87B701888199810E94A4
:1039E00024C82E813F81820F932F911D9F838E8348
:1039F00090E080E0CDB7DEB7E6E00C949FEEB0E05B
:103A0000A0E0E5E0FDE10C947FEEEC017B018A0192
:103A10008A859B858617970731F0888199810E9456
:103A200021D0FB86EA8688859985019609F5CC80A8
:103A3000DA808E81D80EA880B980D5015596ED9197
:103A4000FC91C5010995C80E780110E0F70121919C
:103A50007F0121111FC08E819F81810F911D9F8346
:103A60008E8390E080E0CDB7DEB7EAE00C949BEE69
:103A7000EE80FF80B801888199810E9424C88E0D54
:103A80009F2D911D288539852817390780F681E0FB
:103A900090E0E9CF4C2D6D2DC5010E9479D0D80E54
:103AA000180FD4CFB0E0A0E0E8E5FDE10C9482EE81
:103AB000EC01D62E1CAD0BAD7C0184E0E80EF11CB0
:103AC000E98DFA8DC7010995412F480F2D2D602FE3
:103AD000C7010E9479D09BAD890F8BAF81E090E048
:103AE000CDB7DEB7E7E00C949EEEA6E0B0E0EBE7E2
:103AF000FDE10C9478EE7E836D83342EFC014080D2
:103B0000518062807380C301B20120E13EE040E059
:103B100050E00E94BFED49015A0189018CE3C82E93
:103B2000D12CE12CF12CC301B201A70196010E9416
:103B3000BFED69837A838B839C83CA01B901A70196
:103B400096010E94BFED6B017C01332061F1C3013E
:103B5000B20120E831E541E050E00E94BFED2901CB
:103B60003A015901DF92CF92C40168E170E00E94EE
:103B700035EE9F938F935F924F9289E491E19F93EB
:103B80008F93FE81FF938D818F930E942AE70FB65A
:103B9000F894DEBF0FBECDBF88E0FAE04F165104A7
:103BA000D8F089E019C081149104D1F48A818F93EF
:103BB00099819F93DF92CF928DE391E19F938F93B1
:103BC000EE81EF93FD81FF930E942AE70FB6F894F0
:103BD000DEBF0FBECDBF85E02696E1E10C9494EEEA
:103BE0000436110568F4DF926F939F928F9281E300
:103BF00091E19F938F939E819F93ED81EF93E4CF0B
:103C0000DF926F939F928F9287E291E19F938F93C0
:103C10009E819F93ED81EF930E942AE70FB6F8945F
:103C2000DEBF0FBECDBF86E0D7CF8091E703909176
:103C3000E803009731F04AE050E070E060E00C9457
:103C4000B2E560E070E0CB0108958091E7039091C8
:103C5000E803009731F04AE050E070E060E00C9437
:103C600085E460E070E0CB010895EFDF97FD0AC0C6
:103C7000ECDF6F3F71058105910509F02CF4E5DF5C
:103C8000862F089580E008958FEF0895CF93C62F73
:103C900016DC882311F0E9DFC82F8C2FCF9108950F
:103CA0008091E7039091E803892B39F0DEDF91E002
:103CB000811101C090E0892F089591E0FCCFCF934E
:103CC000DF93C82FD62FFBDB882321F0E9DFDF91BC
:103CD000CF9108958C2F7CDB8111F9CF8D2FF7CFF9
:103CE000B4DFCB010895CF93DF93EB01E8DB8823AA
:103CF00011F0F6DFEC01CE01DF91CF9108950F9323
:103D00001F93CF938091E7039091E8030097D9F038
:103D1000FC018F01C1912C2F2F7D81F0C53411F052
:103D2000C536B9F7F801108270E060E00E942FE319
:103D3000F801C083CF911F910F91089570E060E06A
:103D40000E942FE3F7CF60E070E0CB01F3CFCF927A
:103D5000DF92EF92FF926A017B01B1DB882319F0B9
:103D6000CEDF6B017C01C701B601FF90EF90DF90C1
:103D7000CF900895CF92DF92EF92FF92CF93C82F0A
:103D80000E94E0CC6B017C0124EA30E74DE75FE361
:103D90006091310170913201809133019091340131
:103DA0000E9491E787FD18C08AEF90E0A0E0B0E0A4
:103DB0008C0D9D1DAE1DBF1D809362049093630406
:103DC000A0936404B0936504C0932701CF91FF9042
:103DD000EF90DF90CF90089580E090E0DC01E8CF95
:103DE000CF9380912304811154C010927D131092BF
:103DF0007E1310927F1310924B1310924A1310925D
:103E00004D1310924C1310924F1381E080934E1378
:103E100082E2809350131092551310925413E9E6E6
:103E2000F3E127E733E18FEF81932E173F07E1F7A7
:103E3000C1E0C09366132CE53EEA30935C132093F7
:103E40005B13C0935D1310925E1310925F1390E4A6
:103E500090936013109261132BE53EEA3093781330
:103E6000209377132FE131E03093491320934813C7
:103E70009EE190936D1391E190936E139CE190936A
:103E80006B1380936A13809369130E9473CEC0935F
:103E9000230481E08093220488E691E190937912D3
:103EA0008093781210927B1210927A1253985B9A38
:103EB00052985A9A3898409A0E94A1A3109272047C
:103EC000CF910895FC0180E0309749F094919923B7
:103ED00031F0907C903809F08F5F3196F7CF0895DC
:103EE000B0E0A0E0E6E7FFE10C947FEEEC015B01BF
:103EF0008A01FB01099587FD10C0C82ED12CF12C39
:103F0000E12C2196F801C082D182E282F382CE01B7
:103F1000CDB7DEB7EAE00C949BEE982F907E903CF4
:103F2000A9F48F7190E0B0E0A0E06C017D0156E053
:103F3000CC0CDD1CEE1CFF1C5A95D1F7CE0101966E
:103F4000F50109958F73C82A2296DCCF982F907FB0
:103F5000903E11F58F7090E0B0E0A0E06C017D0123
:103F600036E0CC0CDD1CEE1CFF1C3A95D1F7CE01DF
:103F70000196F50109958F73C82A46E0CC0CDD1C2B
:103F8000EE1CFF1C4A95D1F7CE010296F50109956A
:103F90008F73C82A2396B6CF982F987F903F79F5D4
:103FA000877090E0B0E0A0E06C017D0186E0CC0C71
:103FB000DD1CEE1CFF1C8A95D1F7CE010196F501A0
:103FC00009958F73C82A96E0CC0CDD1CEE1CFF1CF3
:103FD0009A95D1F7CE010296F50109958F73C82AFB
:103FE00026E0CC0CDD1CEE1CFF1C2A95D1F7CE017F
:103FF0000396F50109958F73C82A249683CF982FCD
:10400000907C903841F4807C803869F42196CE0110
:10401000F5010995F8CF8E7F8D3F28F02196CE01CE
:10402000F5010995F8CFC12CD12C76016BCF9CE01E
:10403000899F802D112491E0980F909321042CE00A
:10404000280F20934B0730E02E5F3F4F40917A13AB
:104050004217130619F014F080E0089520917C13A4
:104060009217D0F7662341F08E5F0E9458CF80915F
:104070004B078E5F0E9458CF80914B0790917A1327
:10408000891750F320917C1390912104291720F374
:1040900010927D1380937E1381E008952091200477
:1040A000022E000C330B8217130641F0809320047C
:1040B0006DE872E186E493E10C9421D00895ACE0C0
:1040C000B0E0E5E6F0E20C9481EE6F3F710581050A
:1040D000910509F070F482E493E1E4DCE0914A1385
:1040E000F0914B133196849190E02C96E8E00C947B
:1040F0009DEEF0907D13E0907E132091220421111B
:104100000FC047E051E16E2D8F2D0E94D2D090E07C
:1041100080E0F80EF0927D13E0927E139927E5CFB0
:10412000C0904A13D0904B1326E433E13A8329839D
:104130002F2D30E03C832B832E2D30E03E832D83CA
:1041400018861F822FEF3FEF3A8729871C861B8630
:104150000FEF1CE19E012F5F3F4FAB01BC01C60179
:104160000E9459AFB60186E493E10E9421D08F816D
:104170009885CFCF4F925F926F927F928F929F924E
:10418000BF92CF92DF92EF92FF920F931F93CF9344
:10419000DF93CDB7DEB728970FB6F894DEBF0FBE1A
:1041A000CDBF7C016A014901FB0190818CE0989FA1
:1041B000800D1124982FF7012081822F880F820F04
:1041C000880F80937D1390937E134115510561F103
:1041D000FA82E9827C836B8301111FC0AE014B5FC1
:1041E0005F4FB401C6017CDE6C016D817E818F81E1
:1041F00098856115710581059105B1F060DFF701C2
:1042000080818F5F8083853148F3CE0101960E94C3
:10421000E818E4CFB12C860129C08A01B12C26C050
:10422000452846284728B1F728960FB6F894DEBFF0
:104230000FBECDBFDF91CF911F910F91FF90EF90F7
:10424000DF90CF90BF909F908F907F906F905F9006
:104250004F900895B39407C0B1102DC001151105FA
:10426000C9F20F5F1F4F01151105A9F2AE014B5F97
:104270005F4FB401C60134DE6C014D805E806F80FB
:1042800078844114510461047104A9F0F0E24F16DE
:1042900051046104710401F3D301C2018D97A10996
:1042A000B1090297A105B10530F04BE24416510463
:1042B0006104710479F6F7018081482F4B0D552771
:1042C000551F4631510534F0853020F0CE0101965E
:1042D0000E94E81881E0411451046104710409F45A
:1042E00080E0B80EF70180818B0D8083BB2009F43C
:1042F00097CFBA94AE014B5F5F4FB401C801F0DDB8
:104300008C016D817E818F819885D9DEEFCFCF932F
:10431000DF93FC0125AD211104C021E025AF0E94EF
:1043200073CEC0914813D0914913E0917713F09167
:10433000781382E00995E0917713F091781381E08A
:10434000099530E020E044E1BE0186E493E10E945B
:104350006ECE29E733E147E1BE0186E493E10E9496
:104360006ECEE0917713F091781380E00995DF919C
:10437000CF9108954F925F926F927F928F929F920A
:10438000AF92BF92CF92DF92EF92FF92CF93DF93E3
:1043900000D000D0CDB7DEB70E94E0CC6B017C012D
:1043A000809127018F3FC1F10E94E0CC8090620490
:1043B00090906304A0906404B09065046819790932
:1043C0008A099B0997FD28C080912E1390912F1385
:1043D0008F5F8F70891701F1E0912701E53008F0B8
:1043E000DCC024E0E29FF0011124E256FE4F808100
:1043F0009181A281B38189839A83AB83BC8320E0BE
:1044000030E0A901BE016F5F7F4F82E791E00E941B
:10441000ADC28FEF809327010E94A1A38091730406
:1044200082FFC4C08091710481111DC091E09093FE
:10443000710480917804892780932707109278046B
:1044400083E080936701109273040E94E0CC6C506B
:104450007E4F8F4F9F4F60937404709375048093C9
:1044600076049093770480916D0490916E04A091EE
:104470006F04B0917004A7019601281B390B4A0BF9
:104480005B0BDA01C901B7FF05C08091790488236D
:1044900009F4C5C1D701C6018C599F4FAF4FBF4F1B
:1044A00080936D0490936E04A0936F04B093700496
:1044B00060917204062E000C770B77FF03C0719594
:1044C000619571099091720480916C04981371C088
:1044D000633008F06EC01092720480917204809371
:1044E0006C04643008F075C0809127078111F3C017
:1044F000809140139091411389559C4241F48091E1
:104500002801882309F4F9C08150809328010E9472
:10451000747680907B0790907C07A0907D07B09088
:104520007E0781110E948176D501C4013AE0B695DB
:10453000A795979587953A95D1F7009741E0A407FD
:10454000B10520F08FEF9FEFA0E0B0E09695879542
:10455000209167012111E3C03091790431118BC1A1
:10456000809140139091411389559C4209F46AC18E
:1045700080917A04811166C18091680490916904E8
:10458000A0916A04B0916B04C81AD90AEA0AFB0A1E
:10459000F7FC66C10E94CD8D63C180916801909146
:1045A0006901A0916A01B0916B0125CF109271044D
:1045B0005ACF633009F091CF8091720487FD07C014
:1045C00081E0880F880F8093720464E086CF8FEFBC
:1045D000F8CF80914A0721E030E040E050E08823A6
:1045E00009F456C08090460790904707A09048076E
:1045F000B090490781149104A104B104E9F170E07D
:1046000090E080E00E9495E720E030E040E85EE343
:104610000E94F6E72B013C01C701B6016819790930
:104620008A099B090E9495E79B01AC01C301B20175
:104630000E9429EF20E030E04AE754E40E94F6E7C8
:104640004B015C0120E030E040EA52E40E944EF071
:1046500024E630E040E050E087FF12C020E030E088
:1046600040EF51E4C501B4010E944EF02AE030E071
:1046700040E050E087FF04C021E030E040E050E03F
:10468000C0924607D0924707E0924807F092490748
:10469000A09172040A2E000CBB0B0E9407EE24E0CE
:1046A00030E040E050E00E94E1ED809142079091BF
:1046B0004307A0914407B0914507820F931FA41FA1
:1046C000B51F8093420790934307A0934407B0938C
:1046D000450710927204D701C6018856954CAF4F1A
:1046E000BF4F8093680490936904A0936A04B093C9
:1046F0006B0481E080936701FBCE8CE080932801FE
:104700008091660490916704009729F00197909337
:1047100067048093660481E080936701F8CE009778
:1047200041F040916604509167044817590708F01A
:1047300017CF80917904811111C0223038F02430D4
:1047400008F43FC0243011F41092670182E493E131
:10475000DEDD81E0809341078093790483E09EDC75
:1047600081E080936613E0914013F0914113099525
:104770001092410780917904811127C01092270778
:10478000809140139091411389559C4209F0F0CEDD
:104790000E94E0CCDC01CB018C199D09AE09BF0958
:1047A0008090660490906704B12CA12C881699061D
:1047B000AA06BB0608F0D4CE9093670480936604E3
:1047C000CFCE81E080936701C1CF86E493E10E9460
:1047D000F1CF91E0811101C090E09093790488239A
:1047E00069F2809140139091411389559C42B9F42C
:1047F0000E94E0CCDC01CB018C199D09AE09BF09F8
:10480000C0906604D0906704F12CE12CC816D9063C
:10481000EA06FB0620F490936704809366040F90E9
:104820000F900F900F90DF91CF91FF90EF90DF905E
:10483000CF90BF90AF909F908F907F906F905F9040
:104840004F90089548E9C40E4AE3D41EE11CF11CC0
:10485000C0926804D0926904E0926A04F0926B04FA
:10486000809179048111DBCF809167018130B9F6A5
:1048700010926701D4CF009709F470CF52CFACE00B
:10488000B0E0E5E4F4E20C9481EEF0907D13E0906A
:104890007E1320912204211112C047EE50E16E2DAB
:1048A0008F2D0E94D2D090E080E0F80EF0927D1320
:1048B000E0927E1399272C96E8E00C949DEEC09030
:1048C0004A13D0904B1326E433E13A8329832F2DEA
:1048D00030E03C832B832E2D30E03E832D831886E1
:1048E0001F827A8769871C861B860FEF1CE19E0159
:1048F0002F5F3F4F4EEF58E1BC01C6010E94EEAF63
:10490000B60186E493E10E9421D08F819885CDCFB6
:10491000A4E0B0E0EEE8F4E20C947DEE7C01062F1A
:104920005A01122F862F660F990B9C012E563E4F6F
:10493000690186E0882E912C11160CF03DC0AE0165
:104940004F5F5F4F6EEF78E1C701CADA7C01698182
:104950007A818B819C81611571058105910561F1D9
:104960006D3371058105910509F450C06E377105ED
:104970008105910509F44AC06A32710581059105E6
:1049800001F507FF11C08EE591E10E3F11F08AE5B8
:1049900091E136E01302B001112471DF66E070E0AE
:1049A0000E9449EE161B60C065E470E080E090E074
:1049B00086DB115069F510E0812F2496ECE00C9411
:1049C00099EE643271058105910571F4A114B10469
:1049D000D1F0E6E01E02B0011124C50150DFB401A0
:1049E0000E9449EE161BA8CF603471058105910520
:1049F00051F41150F6016081062E000C770B880BE4
:104A0000990B5DDB99CF5BDB115096CF07FDBBCFD8
:104A100061E089819A81AB81BC81CD97A105B10507
:104A200009F460E0600F6A30A4F01150862F6AE04C
:104A30000E9428EE092F682F880F770B605D7F4F4B
:104A4000072E000C880B990B3ADB112309F4B3CF26
:104A5000602F062E000C770B605D7F4F072E000C39
:104A6000880B990B2CDB1150112309F4A4CF86E09D
:104A70001802B0011124C70102DF66E070E00E9455
:104A800049EE161B99CFE2E4F3E183AF64AF6FEF19
:104A90007FEFCA01F4CEACE0B0E0E1E5F5E20C94C2
:104AA00081EEF0907D13E0907E132091220421117D
:104AB00012C047EC50E16E2D8F2D0E94D2D090E0B5
:104AC00080E0F80EF0927D13E0927E1399272C96E9
:104AD000E8E00C949DEEC0904A13D0904B1326E46E
:104AE00033E13A8329832F2D30E03C832B832E2D15
:104AF00030E03E832D8318861F827A8769871C8663
:104B00001B860FEF1CE19E012F5F3F4F41E059E1F3
:104B1000BC01C6010E94EEAFB60186E493E10E949B
:104B200021D08F819885CDCF6FEF7FEFB4CFB0E0EC
:104B3000A0E0EDE9F5E20C947FEE5C016B01C2D9D7
:104B4000E82EC6010E940419F12C03E110E0081BB5
:104B50001109C5E20E151F050CF4CFE18C2F90E072
:104B60009C012E5F3F4F40917A134217130609F0C4
:104B70008CF5099720917C13281719065CF1409158
:104B80004D0750914E0760914C0710927D13C093D2
:104B90007E1325E1C501BCDED1E0C114D104A9F02A
:104BA0006AE370E080E090E08ADA0E151F05A4F455
:104BB000C45F80917A13C81740F020917C134C2F6A
:104BC0004950550B241715064CF4CDB7DEB7EAE073
:104BD0000C949BEED0E0E1CFDD23B9F3802F880F5A
:104BE000080F000F00937D13C0937E1360E270E006
:104BF00080E090E064DAC60197DFE7CFACE0B0E098
:104C0000E4E0F6E20C947DEE982F862F6A0179019C
:104C1000B02E692F0CDA882309F487C01091220482
:104C2000C701002371F14ED9A82E80904A139090AD
:104C30004B13111142C02FEF3FEF122F23E12A191E
:104C400040914D0750914E0760914C07C60160DEC0
:104C5000AA2009F46AC0B6E08B9F600111246AE3C0
:104C600070E080E090E02BDA57E0C516D10408F43C
:104C700042C060E270E080E090E021DAC81AD90A10
:104C8000F3CF0E940419A82E80904A1390904B13E2
:104C9000112389F2FE0133968AE0DF011D928A9585
:104CA000E9F786E493E19A83898308ED1CE19E018C
:104CB0002F5F3F4F41E059E112C0FE0133968AE079
:104CC000DF011D928A95E9F786E493E19A8389834F
:104CD00008ED1CE19E012F5F3F4F4EEF58E1B701F9
:104CE000C4010E94EEAFB40186E493E10E9421D09A
:104CF0002F813885A2CF40914B07212F30E0A6E0CD
:104D0000AA9EC00111242E5F3F4F281739070CF4CB
:104D10009C0180E8821B80937D1340937E13BB200F
:104D200041F06FEF7FEFC701AADD2C96ECE00C9409
:104D300099EEC701F9DEF9CF0C9474B04F925F92EF
:104D40006F927F928F929F92BF92CF92DF92EF925B
:104D5000FF920F931F93CF93DF931092180410923A
:104D600017042FE320931B0410921A0410921904C5
:104D70001092130410921404109215041092160449
:104D80009C01F90190812F5F3F4F9032D1F39E3407
:104D9000C9F4818190ED980F9A3020F08D3211F096
:104DA0008B3281F432969F012F5F3F4F8081805379
:104DB0008A3008F46DC09F012F5F3F4F80818032A1
:104DC00009F468C0F0936207E09361078F010F5FF9
:104DD0001F4FC0816AE270E0C8010E9443F1009752
:104DE00031F0FC01319780818032E1F31182CD34C2
:104DF00021F0C43511F0C734D9F5F80180810F5F77
:104E00001F4F8032D1F380538A3090F5C0931B043A
:104E100090E080E06AE0AF014F5F5F4F689F9001D4
:104E2000699F300D1124C901C0972081820F911D07
:104E300027FD9A95FA01208120532A3060F3909340
:104E40001A0480931904DF0131962C912032D9F392
:104E5000CD3461F58E31910539F0F0F4873191054B
:104E600019F08C31910511F5B0931804A093170433
:104E7000DF91CF911F910F91FF90EF90DF90CF9036
:104E8000BF909F908F907F906F905F904F9008950C
:104E9000F90189CFF9018FCF8537910538F0873730
:104EA000910510F3803A13E09107F1F280906107C9
:104EB0009090620740E050E0BA0130E020E0C12C61
:104EC000D12C7601C394FD013196DC91DD2309F4E8
:104ED00084C0D132F1F4CD34E1F480329105C9F4CB
:104EE00040931304509314046093150470931604B4
:104EF000F0931804E093170463E270E0CF010E947E
:104F000043F1009709F4B4CFFC011082B1CFDF0167
:104F1000DACFD154DA3108F05BC0DF011D911032D5
:104F200091F0A0EDA10FAA30E8F01E3271F4A1813A
:104F3000A053AA30B8F02115310519F49F01215072
:104F40003109B12C13C0FD01E8CF1D3211F01B3225
:104F500091F7A181B0EDBA0FBA3020F0AE3259F717
:104F6000A281E6CFBE2EB818309759F3AD2FB0E02E
:104F70002601370104C0440C551C661C771CDA95C9
:104F8000D2F74429552966297729A750BC4FBC92EE
:104F9000A081A154AA3108F4BACFDF01D191DD2359
:104FA00009F491CF00EDB02EBD0E19E01B15A8F746
:104FB00013EDB12EBD0E11E01B1578F7DB3269F34E
:104FC000FD013196DC91D03209F07DCFDF01F8CFC1
:104FD00021153105E9F69D01DBCF309318042093AC
:104FE00017044093130450931404609315047093B2
:104FF00016043ECFFC0165917591859194910895B9
:1050000080E00C94F7888F929F92AF92BF92CF92DC
:10501000DF92EF92FF92CF93DF93EC0180909B049D
:1050200090909C04A0909D04B0909E0420E030E0FD
:10503000A901C501B4010E9491E7882309F452C077
:10504000C880D980EA80FB80A7019601C501B40120
:105050000E9491E718160CF04AC02091E3033091AA
:10506000E4034091E5035091E603C701B6010E94B5
:1050700091E7882321F1C092E303D092E403E09208
:10508000E503F092E6032091DF033091E0034091C5
:10509000E1035091E203C701B6010E94F6E79B01CC
:1050A000AC0160E070E080E89FE30E94AEEE6093A8
:1050B000140170931501809316019093170160916C
:1050C0001401709115018091160190911701DF91E3
:1050D000CF91FF90EF90DF90CF90BF90AF909F90D7
:1050E0008F90089560E070E080E89FE3F0CF60E08B
:1050F00070E0CB01ECCF682F70E090E080E00C9482
:1051000017B0B0E0A0E0E7E8F8E20C9479EEEC012B
:105110002091930430919404409195045091960409
:10512000688179818A819B810E94AEEE4B015C018E
:1051300020919704309198044091990450919A04D9
:105140006C817D818E819F810E94AEEE6B017C011E
:10515000A501940160910C0170910D0180910E01E7
:1051600090910F010E9491E7882309F454C0809226
:105170000C0190920D01A0920E01B0920F012091AE
:10518000D7033091D8034091D9035091DA03C50178
:10519000B4010E94F6E72B013C010E94C2EF4B01D3
:1051A0005C0120E030E040EA50E40E9491E71816EC
:1051B00034F4812C912CC0EAAC2EC0E4BC2E20E04B
:1051C00030E0A901C501B4010E944EF087FF03C081
:1051D000812C912C5401A5019401C301B2010E94BC
:1051E000AEEE6093CF037093D0038093D10390937E
:1051F000D203C501B4010E9491EF6093CD03062E46
:10520000000C770B6F5F7F4F6630710514F066E01E
:1052100070E06093CB03D0910A011091CD03A701F8
:10522000960160911001709111018091120190918D
:1052300013010E9491E7811123C0D11375C0209101
:10524000B3033091B4034091B5035091B60360911C
:10525000CF037091D0038091D1039091D2030E942B
:10526000F6E72091B7033091B8034091B90350910C
:10527000BA030E94AFEECDB7DEB7E0E10C9495EE35
:10528000C0921001D0921101E0921201F09213012C
:105290002091DB033091DC034091DD035091DE036C
:1052A000C701B6010E94F6E74B015C010E94C2EF04
:1052B0006B017C0120E030E040EA50E40E9491E77D
:1052C000181634F4C12CD12CB0EAEB2EB0E4FB2E2E
:1052D00020E030E0A901C701B6010E944EF087FF2F
:1052E00003C0C12CD12C7601A7019601C501B401E0
:1052F0000E94AEEE6093D3037093D4038093D503E2
:105300009093D603C701B6010E9491EF6093CE033C
:10531000062E000C770B6F5F7F4F6630710514F01F
:1053200066E070E06093CC03C091CE03D11305C05A
:1053300080910B018C1709F470C08091CD0390917E
:10534000CE0390930B0180930A010C2E000CDD0B11
:1053500027E01203C0011124FC01EC0FFD1FEE0F2A
:10536000FF1FEE0FFF1FE055FB4F2081318142816F
:1053700053812093C7033093C8034093C9035093CC
:10538000CA030091CC03002E000C110BFC01E00FAE
:10539000F11FEE0FFF1FEE0FFF1FE055FB4F608167
:1053A0007181828193810E94AEEE6093C3037093FA
:1053B000C4038093C5039093C6032091CB0337E0C9
:1053C0002303F0011124CE0FDF1FCC0FDD1FCC0F04
:1053D000DD1FC055DB4F288139814A815B812093D5
:1053E000BF033093C0034093C1035093C203E00F47
:1053F000F11FEE0FFF1FEE0FFF1FE055FB4F608107
:105400007181828193810E94AEEE6093BB037093A1
:10541000BC038093BD039093BE038090D303909010
:10542000D403A090D503B090D6032091C30330914C
:10543000C4034091C5035091C603C501B4010E9445
:10544000F6E72091C7033091C8034091C9035091FA
:10545000CA030E94AFEE6B017C01C092B703D092E9
:10546000B803E092B903F092BA032091BB033091E4
:10547000BC034091BD035091BE03C501B4010E941D
:10548000F6E72091BF033091C0034091C1035091D2
:10549000C2030E94AFEEA70196010E94AEEE609398
:1054A000B3037093B4038093B5039093B603C7CE50
:1054B000ACE0B0E0EEE5FAE20C9486EE182F88231B
:1054C00079F020E030E0A9016091A0047091A1047E
:1054D0008091A2049091A3040E9491E78823F1F0A7
:1054E00080919F048117D1F00E94A0738CE0E6E8C0
:1054F000F1E0DE01119601900D928A95E1F7CE015F
:105500000196FFDD80919F04882361F082E791E09E
:105510000E94F67310929F040E94B3862C96E3E0DB
:105520000C94A2EE81E080939F0482E791E00E94B8
:10553000C273F2CFCF92DF92EF92FF9280E0B8DF9A
:1055400010929704109298041092990410929A0461
:105550001092930410929404109295041092960461
:105560001092A4041092A5041092A6041092A7040D
:105570001092A0041092A1041092A2041092A3040D
:1055800040EB54E027E0C12CD12C60ECE62E6FE715
:10559000F62E90E080E0FC01EE0FFF1FEE0FFF1FE4
:1055A000E40FF51FC082D182E282F3820196873038
:1055B000910589F72150445E5F4F2111EACFFF909A
:1055C000EF90DF90CF9008954F925F926F927F920D
:1055D0008F929F92AF92BF92CF92DF92EF92FF9203
:1055E0001F93CF93DF93EC01162F20919B043091F2
:1055F0009C0440919D0450919E04688179818A8128
:105600009B810E9491E7882309F497C0B0909F0482
:1056100080E04EDFC880D980EA80FB8020E030E067
:10562000A901C701B6010E944EF087FF03C0C12C3B
:10563000D12C7601C0929B04D0929C04E0929D04F0
:10564000F0929E042DEB37E346E855EBC701B60117
:105650000E9491E787FD0BC02DEB37E346E855E349
:10566000C701B6010E944EF018160CF076C0A701D3
:10567000960160E070E080E89FE30E9429EF60936C
:10568000DF037093E0038093E1039093E20380EFE4
:105690009FEFA9E7B4EC8093E3039093E403A09316
:1056A000E503B093E603BB2009F447C040907201C4
:1056B0005090730160907401709075018090760134
:1056C00090907701A0907801B0907901C0907A0114
:1056D000D0907B01E0907C01F0907D0181E0E8DEDC
:1056E000112359F1A301920160917201709173012C
:1056F00080917401909175010E9491E781111BC006
:10570000A5019401609176017091770180917801F3
:10571000909179010E9491E781110DC020917A0149
:1057200030917B0140917C0150917D01C701B60110
:105730000E9491E781110E940187DF91CF911F9113
:10574000FF90EF90DF90CF90BF90AF909F908F90A1
:105750007F906F905F904F90089560E070E0CB0174
:105760008ECF8F929F92AF92BF92CF92DF92EF92A5
:10577000FF92C090A004D090A104E090A204F09009
:10578000A30420E030E0A901C701B6010E9491E71F
:105790008823E1F1A701960160E070E080E89FE3D3
:1057A0000E9429EF6B017C018090A4049090A504D5
:1057B000A090A604B090A70420E030E0A901C501A4
:1057C000B4010E9491E7882329F1A501940160E0CA
:1057D00070E080E89FE30E9429EFC092D703D09247
:1057E000D803E092D903F092DA036093DB0370935D
:1057F000DC038093DD039093DE03FF90EF90DF9056
:10580000CF90BF90AF909F908F900895C12CD12CD6
:105810007601CACF60E070E0CB01DFCFCF92DF929C
:10582000EF92FF926B017C0183E3C816D104E1047F
:10583000F10470F082E3C81AD108E108F10862E3CC
:1058400070E080E090E00E9457CC0E947770ECCF2F
:10585000C701B6010E9457CC0E947770FF90EF906D
:10586000DF90CF900895BC0190E080E00C9417B0D9
:1058700080915F07813069F09091981492FB88279E
:1058800080F992FF07C097FB882780F991E089276C
:10589000089581E008959091981494FB882780F9E9
:1058A00094FF06C081E090919E12911101C080E0AA
:1058B0000895ACE0B0E0EFE5FCE20C9479EE1092D4
:1058C0004A078091270710922707882361F020E07C
:1058D00040E070E060E083E491EA0E94918C2C96B5
:1058E000E0E10C9495EE2091390130913A0140911C
:1058F000420750914307CA01820F931F2436310596
:1059000009F0E9C34730510544F006978A30910504
:105910000CF0F0C38AE090E0F7C306964A3F5F4F71
:10592000ACF380914107882309F4D0C160918A12B9
:1059300070918B12072E000C880B990B0E9497E731
:1059400011E0209186123091871240918812509177
:1059500089120E944EF018160CF010E010936104AA
:1059600080907A0190907B01A0907C01B0907D01A5
:1059700020E030E0A901C501B4010E9491E7C12CEB
:10598000D12CE0EAEE2EE0ECFE2E87FD06C0C12C05
:10599000D12C70EAE72E70E4F72E20E030E04AE7E1
:1059A00054E4C501B4010E94F6E7A70196010E94E4
:1059B000AFEE2DEC3CEC4CEC5DE30E94F6E70E9470
:1059C00091EF6B017C0180E2F7FE09C0F094E09456
:1059D000D094C094C11CD11CE11CF11C8DE24090FC
:1059E0007201509073016090740170907501209164
:1059F00076013091770140917801509179012987A2
:105A00003A874B875C8780937B0460E230E1C31662
:105A100037E2D306E104F1048CF0C701B60120E1BE
:105A200037E240E050E00E94E1EDCA01B9012AE00E
:105A300030E040E050E00E94E1ED605D60937C0466
:105A400060E248EEC41643E0D406E104F1048CF0B1
:105A5000C701B60128EE33E040E050E00E94E1EDDE
:105A6000CA01B9012AE030E040E050E00E94E1EDD7
:105A7000605D60937D04C701B60124E630E040E03C
:105A800050E00E94E1ED6AE0862E912CA12CB12C11
:105A9000CA01B901A50194010E94E1ED605D609326
:105AA0007E04C701B601A50194010E94E1ED6B01DE
:105AB000CA01B901A50194010E94E1EDCC2009F4CD
:105AC00033C32EE220937F04605D6093800450E333
:105AD000C50EC09281046BE774E089E594E00E94F2
:105AE0004EF120E030E0A901C301B2010E9491E72C
:105AF00020E030E040E05FEB87FD04C020E030E0D4
:105B000040E05FE3C301B2010E94AFEE0E9491EF5B
:105B1000CB010E94718BBC0184E594E00E944EF1A0
:105B200020E030E0A90169857A858B859C850E94FB
:105B300091E720E030E040E05FEB87FD04C020E02B
:105B400030E040E05FE369857A858B859C850E9423
:105B5000AFEE0E9491EFCB010E94718BBC018FE4EC
:105B600094E00E944EF18091981400E117E283FDC9
:105B700028C091DE882309F4E9C2809190149091A5
:105B80009114A0919214B09193140097A105B105BE
:105B900009F4DCC2BC01CD01615F784D8F4F9F4F8E
:105BA00020E137E240E050E00E94BFED60919414A4
:105BB0007091951480919614909197140E94BFED66
:105BC00089010E94C78A4B015C018D829E82AF824F
:105BD000B886D62E809126018017C1F10093260148
:105BE000C80164E670E00E9435EE7B0188E48E9D7A
:105BF000B0018F9D700D112490E080E00E9495E728
:105C00002AE037ED43E25CE30E94F6E70E9496EF5C
:105C100060934E040115110509F09BC210924904CE
:105C200010923F0480E880933E0489E494E0FC01F4
:105C300001900020E9F7CF0189549440982F990FE3
:105C4000890F880F90E8981B90933D04809125015F
:105C5000D816E1F18092250141E08D819E81AF81CE
:105C6000B88580389145A140B10508F440E06DE267
:105C700074E0CE0105960E94751D982F990F990F1B
:105C8000891B880F805880932C04282D2370822E26
:105C9000E9F401151105A9F0A0E1B7E2A01BB10BD1
:105CA0002D813E814F8158850E94FDED980150E085
:105CB00040E00E94BFED211531054105510509F075
:105CC0006EC210923F0480E880933E040E94E0CCB4
:105CD0000091250410912604209127043091280476
:105CE0006B017C01C01AD10AE20AF30A970186010E
:105CF00037FD11C0209124042095209324046A5478
:105D00007C4F8F4F9F4F60932504709326048093A0
:105D1000270490932804D090240411E0D11001C0EE
:105D200010E081E00E944E2080917A13873180F448
:105D300080917C13843060F03BE1E32E32E1F32E5E
:105D400003E126E044E069E086E493E10E94F7D0B5
:105D500080917A138431B8F480917C13823098F06A
:105D6000DD2009F435C280917F07882309F430C211
:105D700085EE91E17C0102E123E042E068E686E401
:105D800093E10E94F7D080917A138C3108F06EC0B5
:105D900040908612509087126090881270908912FD
:105DA000A0908A12B0908B12843198F480917C1369
:105DB000883078F08091610480FF0DC287E991E11D
:105DC0007C010CE022E048E064E486E493E10E9478
:105DD000F7D080917A13883040F4B7FEFFC14BE7CB
:105DE00051E167E082E40E94432580917A138C316F
:105DF000B0F480917C13843190F020E030E040E0FA
:105E00005FE3C301B2010E94AFEE0E9491EF77FF02
:105E10000EC24BE751E16CE182E40E944325809180
:105E20007A138C3118F580917C138431F8F08091CD
:105E30007F078823D9F024E6829FC001112481586E
:105E40009F4F6FEF70E00E9449EECB010E94F08BF4
:105E500027E620937D132CE120937E130E94942546
:105E600065E270E080E090E00E945F2014DD88230E
:105E700079F180917A13843358F580917C138A32BA
:105E800038F107E028E04AE26AE286E493E10E9402
:105E90009ECF05E022E04CE262E386E493E10E94BB
:105EA0009ECF24E04AE061E38AE20E946ECF6091D7
:105EB00048137091491382E3809362138BE28093BD
:105EC000631322E633E142E386E493E10E946ECE5F
:105ED00080917A13853350F480917C13813330F0B4
:105EE00024E04AE461E386E30E946ECF80917A1356
:105EF000843368F480917C13823348F002E020916F
:105F00004E0442E367E386E493E10E949ECF8091D2
:105F10007A13803358F580917C13883238F1809160
:105F20002B04811751F080912A0410932B048F5F6A
:105F3000833008F0A5C180932A0480912A0481113E
:105F4000A2C180914904882389F080913D04809307
:105F50007D1380E380937E1389E494E00E9494256E
:105F600065E270E080E090E00E945F2080917A130B
:105F7000883208F05DC080917C138D3108F458C0E0
:105F80002BE040E86DE180E00E946ECF80917A13B3
:105F9000873208F04DC080917C138F3108F448C0DF
:105FA00083E080937D1306E200937E1368E570E042
:105FB00080E090E00E945F208BE080937D1300934F
:105FC0007E13DD2009F491C184E594E00E949425BC
:105FD00088E280937D1306E200937E1369E570E00A
:105FE00080E090E00E945F2080E380937D13009327
:105FF0007E13DD2009F49EC18FE494E00E94942575
:106000008DE480937D1306E200937E136AE570E0D1
:1060100080E090E00E945F2085E580937D130093EF
:106020007E13DD2009F4ABC189E594E00E9494253C
:1060300080917A13833348F580917C138B3228F159
:1060400083E00E944E2083E080937D1303E300935E
:106050007E1366E070E080E090E00E945F2081E0C7
:106060000E944E208091390190913A010E94F08B5C
:106070002CE020937D1300937E130E94942565E20B
:1060800070E080E090E00E945F2080917A1381347C
:1060900008F025CC80917C13863308F420CC109234
:1060A0007D138EE380937E1387E190E10E940419B3
:1060B000082F863108F088C187E190E10E9494257D
:1060C000053109F40CCC60E270E080E090E00E94C1
:1060D0005F200F5FF5CF243631054CF485369105EE
:1060E00004F58A30910534F48AE090E009C08436E2
:1060F0009105BCF0883EE3E09E0714F087EE93E044
:106100002817390709F40DCC90933A01809339018F
:1061100010924207109243071092440710924507CD
:1061200000CC84E690E0F0CF662351F02EE220937D
:106130007F04605D6093800480E280938104CBCC17
:1061400080E28093800480937F04F6CF10E000E02B
:1061500038CD2E2D80E2243628F08E2D64E60E9464
:106160001CEE805D80937F0490E22A3040F03AE09C
:10617000822F632F0E941CEE0E941CEE905D909374
:106180008004822F6AE00E941CEE905D909381044F
:106190006FE774E089E494E00E944EF146CD2983D4
:1061A0003A834B835C8381E020383145414051057F
:1061B00008F480E0482F6FE374E0CE0101960E945E
:1061C000751D982F990F990F891B880F80587CCDCA
:1061D0008FEA91E1CFCD8FE791E1F2CDC5010E9429
:1061E000F08BFC01808193E0803229F4818192E080
:1061F000803209F491E0892F880F880FE92EE81A80
:106200008E2D855B80937D1387E080937E1323E042
:1062100030E0291B3109CF01820F931F0E94942582
:1062200069E070E080E090E00E945F20DECDCB016D
:106230000E94F08BFC01808193E0803229F48181FF
:1062400092E0803209F491E0892F880F880FF92EAF
:10625000F81A8F2D855B80937D138CE180937E13DC
:1062600023E030E0291B3109CF01820F931F0E94E8
:10627000942569E070E080E090E00E945F20CFCD3F
:1062800010922A045ACE8230B1F480913F048823C0
:1062900091F048E751E160E386E30E944325809155
:1062A0003E0480937D1380E380937E138FE394E01C
:1062B0000E9494255BCE80912D04882309F456CE4C
:1062C00086E380937D1300E300937E136FEF7FEFEF
:1062D00085E791E10E943F2480912C0480937D13F7
:1062E00000937E138DE294E0E3CF87E00E9460820A
:1062F00080FF15C024E5E22E24E0F22EF701619123
:106300007F01662309F464CE6F320CF06FE3062E32
:10631000000C770B880B990B0E945F20EFCF8091C8
:106320004F0780FD51CE6FEF7FEF80E791E10E9434
:106330003F244ECE87E00E94608281FF15C09FE41B
:10634000E92E94E0F92EF70161917F01662309F4AB
:1063500057CE6F320CF06FE3062E000C770B880BD4
:10636000990B0E945F20EFCF80914F0781FD44CEB3
:106370006FEF7FEF80E791E10E943F2441CE87E0FD
:106380000E94608282FF15C089E5E82E84E0F82E25
:10639000F70161917F01662309F44ACE6F320CF058
:1063A0006FE3062E000C770B880B990B0E945F2081
:1063B000EFCF80914F0782FD37CE6FEF7FEF88E6FA
:1063C00091E10E943F2434CE809129041817B1F046
:1063D000009116101093290487E190E10E9404199E
:1063E000081708F050C00F5FE02FF0E0E95EFF4EA5
:1063F0008081807C8038B9F300931610E0901610ED
:10640000F12C9701295E3F4E7901C9010E940419C0
:10641000182F60E870E0C7010E944B25153108F085
:106420005ECA60E270E080E090E00E945F2014317C
:1064300009F455CA60E270E080E090E00E945F20BD
:10644000133109F44CCA60E270E080E090E00E94F1
:106450005F20123109F443CA212F30E02E5F3F4FF5
:106460004AEF4203B001439F700D112460587F4FE3
:1064700087E190E10E944B2560E270E080E090E0CF
:106480000E945F202CCA10921610B8CF80915F072F
:10649000823059F000DA882349F08091981482FB09
:1064A000882780F991E08927089581E0089581E0A7
:1064B0000895DC01EC918E2F90E0FC01EE0FFF1FA0
:1064C000E80FF91FEB50FD4E80818F778083089590
:1064D000892B79F41092900082E0809391001092C1
:1064E000950010929400C19A80917100826080930F
:1064F00071000895B0E0A0E0E0E8F2E30C947CEED7
:10650000EC017B0188818C3008F0A4C090E0FC0194
:10651000EE0FFF1FE80FF91FEB50FD4E80818F77C4
:106520000E949FB219821A8288812CE0622F0E94F9
:106530001CEE829FB001112430E020E0AB01420F3D
:10654000531FFA01EE0FFF1FE40FF51FEB50FD4E36
:10655000908197FD07C02F5F3F4F2C30310571F7B9
:1065600090E0B6DF7880072D10E06801CC0CDD1CD0
:10657000F601E00FF11FEB50FD4E808180688083B3
:1065800077FC68C080E2E81682E0F8060CF03FC0B5
:106590008A8128E532E0281B310987FD3395220FD7
:1065A000331F220F331F032E000C440B550B898120
:1065B00078E8872E912C881A910887FD9394880C8F
:1065C000991C880C991C092C000CAA08BB0860E0D7
:1065D00070E0CB01F7FC0AC0B701653B710514F010
:1065E00064EB70E0072E000C880B990B2819390911
:1065F0004A095B090E94B0ED24EB30E040E050E036
:106600000E94E1ED820E931EA41EB51E74018BE064
:106610008715D8F0298188E890E0821B910927FD31
:106620009395880F991F880F991FE816F906BCF4F7
:1066300002972FB7F894E601C00FD11FCB50DD4E63
:10664000880F991F9A8389832FBF62E370E080E0EF
:1066500090E0E4D8CDB7DEB7EDE00C9498EE2A8157
:1066600088E592E0821B910927FD9395880F991F79
:10667000880F991FE816F906DCF6C701D9CFCF932A
:10668000DF93EB01682F70E08AE193E133DF6881EB
:1066900079818A819B81643F21E0720781059105A0
:1066A00020F464EF71E080E090E0B8D880B182FB24
:1066B000882780F9DF91CF910895A4E0B0E0E3E668
:1066C000F3E30C9487EE8EEE92E0A0E0B0E08983D5
:1066D0009A83AB83BC83BE016F5F7F4F8AE5CFDFB8
:1066E0002496E2E00C94A3EEA4E0B0E0EAE7F3E342
:1066F0000C9487EE8EEE92E0A0E0B0E089839A835E
:10670000AB83BC83BE016F5F7F4F8AE0B8DF249606
:10671000E2E00C94A3EEA4E0B0E0E1E9F3E30C9432
:1067200087EE84EF91E0A0E0B0E089839A83AB83A9
:10673000BC83BE016F5F7F4F8CE3A1DF2496E2E054
:106740000C94A3EEA4E0B0E0E8EAF3E30C9487EE47
:1067500084EF91E0A0E0B0E089839A83AB83BC83AF
:10676000BE016F5F7F4F80EA8ADF2496E2E00C94DF
:10677000A3EE1F920F920FB60F9211240BB60F9239
:106780002F933F934F935F936F937F938F939F9339
:10679000AF93BF93EF93FF938091A40387FF27C02C
:1067A00010929500109294008091A4038F5F8093C3
:1067B000A4038091A403082E000C990B20911913B7
:1067C0002817190629F024F08091A4038C30DCF1FD
:1067D0008091940090919500049680349C4908F42F
:1067E0007DC08091940090919500049679C080912D
:1067F000A403082E000C990B2091191328171906D1
:1068000099F294F2E091A4038E2FEE0F990BFC0104
:10681000EE0FFF1FE80FF91FEB50FD4E808187FF41
:10682000C3CFE091A4038E2FEE0F990BFC01EE0F66
:10683000FF1FE80FF91FEB50FD4E808160E08F775E
:106840000E94FBCBB1CF2091940030919500E09154
:10685000A4038E2FEE0F990BFC01EE0FFF1FE80F24
:10686000F91FEB50FD4E81819281820F931F90930F
:10687000990080939800E091A4038E2FEE0F990B5E
:10688000FC01EE0FFF1FE80FF91FEB50FD4E80815A
:1068900087FF11C0E091A4038E2FEE0F990BFC012E
:1068A000EE0FFF1FE80FF91FEB50FD4E808161E0F6
:1068B0008F770E94FBCBFF91EF91BF91AF919F919A
:1068C0008F917F916F915F914F913F912F910F9099
:1068D0000BBE0F900FBE0F901F90189580E49CE99F
:1068E00090939900809398008FEF8093A403E3CF57
:1068F0009091C00095FFFCCF8093C6000895CF9380
:10690000DF93EC018991882311F0F2DFFBCFDF9157
:10691000CF910895CF93DF93EC018991882311F0F3
:10692000E7DFFBCF8DE0E4DF8AE0E2DFDF91CF91AC
:106930000895CF93DF93EC01FE0184912196882383
:1069400011F0D6DFF9CFDF91CF910895CF93DF9388
:10695000EB01EFDFCE01D3DFDF91CF9108950F93ED
:106960001F93CF938C01C62F84EE9EE0E2DFC80117
:10697000E0DF8AE3BDDF80E38C0FBADF8AE0B8DFB7
:10698000CF911F910F910895CF92DF92EF92FF92D6
:106990006A017B01CEDF42E0C701B6010E94BEB2B0
:1069A000FF90EF90DF90CF900895CF93DF9365EF46
:1069B0007EE00E9402C3C0912913D0912A1348811E
:1069C00059816A817B818CEE9EE0DEDF4C815D81A6
:1069D0006E817F8184ED9FE2D7DF40912513509136
:1069E0002613609127137091281381ED9FE2CCDF6D
:1069F00089EE9EE09EDF85E691E29BDF8AE078DF0C
:106A0000DF91CF910895C0DF8AE072CFAEE4B0E0AD
:106A1000ECE0F5E30C9477EE70E060E085E40E9432
:106A2000731E9AA789A781117CC26EEB70E083E583
:106A30000E94731E3C0165E070E083E40E94731EB7
:106A40008C0160E085E50E945F1E8DAF60E08AEBFF
:106A500090E10E942B9E0E94E0CC69877A878B8709
:106A60009C8780916401909165010E976816790664
:106A700054F08BE690E15DDF0E9499C3C25BDF4F6B
:106A8000E2E10C9493EE29853A854B855C85205E86
:106A9000314B4F4F5F4F2BAB3CAB4DAB5EAB87E504
:106AA00090E147DF0E94EE6F8FE780938C1281E0C8
:106AB0008093660160E083E490E10E942B9E8985CB
:106AC0009A85AB85BC85898B9A8BAB8BBC8B8BA74E
:106AD0009CA7ADA7BEA7198E1A8E1B8E1C8E19A25D
:106AE0001AA21BA21CA219821A821B821C822FE7E7
:106AF00030E040E050E02D873E874F87588B80E0A4
:106B000090E4ACE1B6E48D839E83AF83B8871D8AA1
:106B10001E8A1F8A188EFFE7CF2ED12CE12CF12C74
:106B20002F961FAE2F971FA618AA19AA1AAA1DA240
:106B30001EA21FA218A691E09FAB312C212C812C04
:106B4000912C54019301072C000C440B550B2296F9
:106B50002CAF3DAF4EAF5FAF2297402F002E000C01
:106B6000550B5CAF4BAFC3014E969C01092E000C38
:106B7000440B550B26962CAF3DAF4EAF5FAF26971B
:106B8000CC979C01990F440B550B2A962CAF3DAF27
:106B90004EAF5FAF2A9736E0631A7108C301072C26
:106BA000000CAA0BBB0B2E968CAF9DAFAEAFBFAF48
:106BB0002E9780916601882309F48DC00E94E0CC55
:106BC0002B013C0110917F05112309F473C00E9431
:106BD0003E7010927F058090861290908712A09050
:106BE0008812B0908912A50194016D897E898F89E0
:106BF000988D0E944EF087FF04C08D8A9E8AAF8ACE
:106C0000B88EA50194016D817E818F8198850E9447
:106C100091E7181624F48D829E82AF82B886229660
:106C20006CAD7DAD8EAD9FAD22970E9497E76D8FC5
:106C30007E8F8F8F98A39FA92D8D3E8D4F8D58A14C
:106C4000992309F472C1C501B4010E944EF01816CF
:106C50008CF5D301C20129893A894B895C89821B51
:106C6000930BA40BB50BAC01BD014858534161090E
:106C7000710977FD1FC04D855E856F8578894C1938
:106C80005D096E097F0975956795579547954093FE
:106C90008C128DA39EA3AFA3B8A78D8D9E8DAF8DB3
:106CA000B8A18D8B9E8BAF8BB88F49865A866B8629
:106CB0007C861FAA26966CAD7DAD8EAD9FAD2697C6
:106CC0000E9497E7A50194010E9491E787FF21C0E8
:106CD0008CEB9FE02EDE109266010E94EE6FCCCE10
:106CE0004BEEC42ED12CE12CF12C76C124E130E006
:106CF00040E050E02D873E874F87588B34E1C32E0C
:106D0000D12CE12CF12C76C1CD86DE86EF86F88A77
:106D100071C1D301C2012BA53CA54DA55EA5821B67
:106D2000930BA40BB50BB7FD47C089A50E94636FF9
:106D30008AE0DEDDD301C2018053984FAF4FBF4FD1
:106D40008BA79CA7ADA7BEA72F969FAD2F9791119C
:106D50006FC02FA538A949A95AA9C501B4010E943D
:106D60004EF018160CF050C020E030E040E050E447
:106D7000C501B4010E94AFEE6FA778AB89AB9AABA7
:106D8000A3019201205E314B4F4F5F4F2BAB3CABC9
:106D90004DAB5EAB2E966CAD7DAD8EAD9FAD2E979F
:106DA0000E9497E7A50194010E9491E7881F882718
:106DB000881F2F968FAF2F9789859A85AB85BC85C5
:106DC0008D8F9E8FAF8FB8A329893A894B895C89B3
:106DD000281739074A075B0720F42D8F3E8F4F8F06
:106DE00058A38D8D9E8DAF8DB8A1481A590A6A0A95
:106DF0007B0A91E849169FE4590692E169067104FD
:106E000060F18EE99FE066CFD301C2012BA93CA9B6
:106E10004DA95EA9821B930BA40BB50B4BE55AE25F
:106E20006AE67AE2B7FDC8CF80E00E94FD6FC4CF6A
:106E30002A966CAD7DAD8EAD9FAD2A970E9497E7E7
:106E40009B01AC01C501B4010E9491E787FFB4CF5B
:106E500045E351E365E471E3E7CFABADBCADA2150B
:106E6000B3050CF05BC0B3E02B1631040CF456C034
:106E700081E49FE05EDD84E29FE05BDD49815A8131
:106E80006B817C818DE39FE0BEDD84E29FE051DD7C
:106E900049A15AA16BA17CA189E39FE0B4DD84E202
:106EA0009FE047DD498D5A8D6B8D7C8D85E39FE09A
:106EB000AADD2DAD222309F4DFCD89819A81AB8132
:106EC000BC8180938D1290938E12A0938F12B093F9
:106ED00090122CEA35EC47E25EE369A17AA18BA11E
:106EE0009CA10E94F6E76093911270939212809396
:106EF00093129093941220E030E543EC50E4698DB6
:106F00007A8D8B8D9C8D0E94F6E76093951270931D
:106F100096128093971290939812AECD0E94BA2148
:106F200048CE86E990E105DDA9CDC501B4010E94F6
:106F300091E787FFBFCED301C20129853A854B85F2
:106F40005C85821B930BA40BB50BAC01BD014858AB
:106F500053416109710977FDADCE2114310409F463
:106F6000FCC02DA13EA14FA158A5280F391F4A1FD3
:106F70005B1F298B3A8B4B8B5C8B2DA13EA14FA1C4
:106F800058A5281B390B4A0B5B0BC701B6010E94A1
:106F9000B0ED29893A894B895C890E94E1EDCD8465
:106FA000DE84EF84F888C20ED31EE41EF51E34E1A1
:106FB000C316D104E104F1040CF498CE4CEEC416CF
:106FC000D104E104F1040CF08BCE50E8C516D104D5
:106FD000E104F1040CF498CECD86DE86EF86F88AC3
:106FE0008EEF90E0A0E0B0E08C199D09AE09BF09DA
:106FF0006C017D018BE390E19CDC6D857E858F8546
:1070000098890E949C2686E390E193DCC701B60133
:107010000E949C264D815E816F8178858FE290E190
:10702000B3DC4D895E896F89788D88E290E1ACDCB4
:1070300033E0231631040CF490C0C701B6010E945E
:1070400097E720E030E040E850E40E94F6E76983EB
:107050007A838B839C832D813E814F8158856D89F6
:107060007E898F89988D0E94AEEE2BED3FE049EC32
:107070005FE30E94F6E79B01AC0169817A818B8115
:107080009C810E9429EF6FAB78AF89AF9AAF698975
:107090007A898B899C890E9497E72FE632E143E841
:1070A0005AE30E94F6E76D837E838F8398872AE9EF
:1070B00039E949E15FE36FA978AD89AD9AAD0E94E6
:1070C000F6E769837A838B839C839B01AC010E94E2
:1070D000AFEE2D813E814F8158850E9429EF69A333
:1070E0007AA38BA39CA320E030E040E05EE36D81B7
:1070F0007E818F8198850E94F6E729813A814B81B4
:107100005C810E94F6E7698F7A8F8B8F9C8F4FA9E5
:1071100058AD69AD7AAD82E290E136DC4D815E8199
:107120006F8178858CE190E16EDC8DE090E101DC8F
:1071300049815A816B817C8187E090E125DC49A1FE
:107140005AA16BA17CA181E090E11EDC498D5A8D92
:107150006B8D7C8D8BEF9FE056DC8D859E85AF859A
:10716000B8898C0D9D1DAE1DBF1DB595A795979532
:10717000879580938C124CAD4F930F933F922F9233
:1071800087EE9FE09F938F9322EF3FE03F932F93F3
:107190001F920E940E9E5FEF251A350A0FB6F894D3
:1071A000DEBF0FBECDBF2D8D3E8D4F8D58A12D83DF
:1071B0003E834F835887498A5A8A6B8A7C8A1FABE1
:1071C00079CD66E378E00E9402C36091510D709121
:1071D000520D8091530D9091540D0E9495E7AB0193
:1071E000BC018DE298E0D0DB4091810D5091820D81
:1071F0006091830D7091840D8AE298E0C5DB409127
:10720000850D5091860D6091870D7091880D87E2F4
:1072100098E0BADB4091630750916407609165077D
:107220007091660784E298E0EECBCF93DF936AED2E
:1072300077E00E9402C3C1E4DDE04CA95DA96EA91C
:107240007FA981ED97E0A0DB48AD59AD6AAD7BAD7C
:107250008EEC97E099DB4CAD5DAD6EAD7FAD87E216
:1072600098E0D1DBDF91CF910895CF93DF9366EB68
:1072700077E00E9402C3C1E4DDE04CA15DA16EA1F4
:107280007FA18DEA97E080DB48A559A56AA57BA57B
:1072900084ED9FE279DB4CA55DA56EA57FA581ED10
:1072A0009FE272DB48A959A96AA97BA98EEC9FE2EB
:1072B000AADBDF91CF910895CF93DF9361E977E067
:1072C0000E9402C3C1E4DDE0688179818A819B81EB
:1072D0000E9495E7AB01BC0188E897E055DB6C8123
:1072E0007D818E819F810E9495E7AB01BC0184ED79
:1072F0009FE24ADB688579858A859B850E9495E7B0
:10730000AB01BC0181ED9FE23FDB6C857D858E8505
:107310009F850E9495E7AB01BC018EEC9FE273DB79
:10732000DF91CF910895AF92BF92CF92DF92EF920B
:107330000F931F93CF93DF935B01EA0169018823C9
:1073400009F452C081E897E0F4DAF50160817181B7
:107350008281938146E00E94BEB2E1100AC088E7B4
:1073600097E0E7DA688179818A819B8146E00E9413
:10737000BEB281E797E0DDDAF6016081718182813A
:10738000938143E00E94BEB28AE697E0D2DAF80128
:10739000608171818281938143E00E94BEB281E667
:1073A00097E0C7DAF6012081318142815381F801EB
:1073B00060817181828193810E94AEEE43E00E94E0
:1073C000BEB2EE2099F08AE093DA8CE497E0B1DA6D
:1073D000688179818A819B8146E00E94BEB28AE001
:1073E00087DA8AE085DA02C0E110EFCFDF91CF9132
:1073F0001F910F91EF90DF90CF90BF90AF900895C5
:10740000A6E5B0E0E6E0FAE30C9477EE2DB63EB6E2
:1074100087E00E947B8281110AC061E086E50E94BC
:10742000461E8DA3853090F087E297E082DA0FB692
:10743000F8943EBE0FBE2DBE0FB6F8943EBE0FBEF2
:107440002DBECA5ADF4FE2E10C9493EE2DA1222308
:1074500019F087E097E06DDA6AE080E50E94461E49
:10746000182F8CEF810F8F3218F083EE96E0DECF6D
:1074700060E085E40E945F1E882309F447C031E084
:1074800038AFE0902913F0902A13D7012D913D9148
:107490004D915C91609172017091730180917401C2
:1074A000909175010E94AFEEAB01BC0188E50E948E
:1074B000A71E69877A878B879C87F701248135818E
:1074C00046815781609176017091770180917801B2
:1074D000909179010E94AFEEAB01BC0189E50E9459
:1074E000A71E6D877E878F87988BBE01635F7F4F56
:1074F000CE0109960E94DBC381110BC063E68FECBD
:1075000096E00E942B9E87EB96E090CF83E088AFB9
:10751000B8CF8CE40E94E819082F882309F44EC1E3
:107520000E94351E8EA3803118F080E996E07ECF50
:10753000FEA1F13009F444C160E083E50E945F1EC2
:1075400022968FAF2297882321F0011102C037E0E5
:107550003EA38DA1833018F086E796E0EAD990919A
:107560009F0429969FAF299780E00E94582A0E9485
:10757000E6851D8A1E8A1F8A188E198E1A8E1B8E0A
:107580001C8E83EF9FE4A3ECB7E48D8F9E8FAF8FAB
:10759000B8A383EF9FE4A3ECB7EC89A39AA3ABA3B2
:1075A000BCA3A12FB0E0BBABAAABEDB7FEB724E004
:1075B000129FE019F10911240FB6F894FEBF0FBE17
:1075C000EDBF8DB79EB7019624969FAF8EAF2497DF
:1075D0002DA148ADBE01635F7F4FCE0109960E9489
:1075E00011C50E94E0CC611571058105910511F06E
:1075F0000E9426E319AA1CAA1DAA1EAA1FAAAEA1B0
:10760000A150BB0B6396BFAFAEAF6397812F90E0E5
:10761000B0E0A0E067968CAF9DAFAEAFBFAF67970D
:10762000B9A9AB2FB0E0BCA7ABA7EAA9FBA9AE17DD
:10763000BF070CF07BC21196B8A7AFA3FF93EF93DF
:10764000BF93AF9382E696E09F938F938CE696E08C
:107650009F938F931F920E940E9E2DB73EB7275F78
:107660003F4F0FB6F8943EBF0FBE2DBF3EA1332350
:1076700009F48CC10E94D7E22AE030E040E050E0FB
:107680000E94E1ED0E9497E720E030E040EA50E4FC
:107690000E944EF00FEF1FEF181614F001E010E0FB
:1076A0000E94D7E228E631E040E050E00E94E1EDA0
:1076B0000E9497E72B013C010E94D7E227E130E0CE
:1076C00040E050E00E94E1ED6B5F7F4F8F4F9F4F96
:1076D0000E9497E769AF7AAF8BAF9CAF8DA18430E2
:1076E000B9F449AD5AAD6BAD7CAD84E596E04CD9AB
:1076F000B301A2018CE496E047D986E496E019D95B
:107700000130110511F483E4F3D882E496E011D935
:10771000B801110F880B990B0E9497E721966CAF67
:107720007DAF8EAF9FAF219720E030E040E153E482
:107730000E94F6E72D966CAF7DAF8EAF9FAF2D9771
:107740001FA6EFA56396AEADBFAD6397EA171B0604
:107750000CF01CC12296FFAD2297F11134C00E949B
:10776000D7E224E130E040E050E00E94E1ED675EC6
:107770007F4F8F4F9F4F0E9497E721962CAD3DADD5
:107780004EAD5FAD21970E94F6E79B01AC01C301AE
:10779000B2010E94AFEE2B013C0120E030E044EB4F
:1077A00053E40E9491E71816ACF420E030E044EB7B
:1077B00053E4C301B2010E94AEEEEDCF1EA2BCCED7
:1077C00022E02EA3B9CE2D962CAD3DAD4EAD5FADD2
:1077D0002D97DDCF20E030E0A901C301B2010E9466
:1077E0004EF087FF0BC020E030E044EB53E4C301D0
:1077F000B2010E94AFEE2B013C01ECCF00912913A6
:1078000010912A13D80114962D913D914D915C91C0
:1078100017976D857E858F8598890E94AEEE61965B
:107820006CAF7DAF8EAF9FAF619726E33AEF4EE826
:107830005CE3C301B2010E94F6E76B017C010E9488
:1078400026EF28966CAF7DAF8EAF9FAF2897F801DB
:10785000208131814281538169857A858B859C8520
:107860000E94AEEE4B015C0129AD3AAD4BAD5CAD73
:1078700028966CAD7DAD8EAD9FAD28970E94F6E742
:107880009B01AC01C501B4010E94AFEE4B015C014C
:1078900089829A82AB82BC82C701B6010E9483F0C2
:1078A00029AD3AAD4BAD5CAD0E94F6E761962CADCB
:1078B0003DAD4EAD5FAD61970E94AFEE6B017C01B7
:1078C000CD82DE82EF82F88620E030E040EE50ECA0
:1078D000C501B4010E9491E787FF3AC080E090E0C3
:1078E000A0EEB0EC89839A83AB83BC8320E030E0C8
:1078F00040E050ECC701B6010E9491E787FF37C016
:1079000080E090E0A0E0B0EC8D839E83AF83B887E9
:10791000FDA1F43071F449815A816B817C8186E349
:1079200096E032D84D815E816F81788584ED9FE24B
:107930006AD8198A1A8A1B8A1C8ABE016F5E7F4F19
:10794000CE0101960E9480C62FA52F5F2FA7F9CEEA
:1079500020E030E041E653E4C501B4010E944EF05E
:10796000181624F680E090E0A1E6B3E4BBCF20E057
:1079700030E041E653E4C701B6010E944EF018160C
:107980003CF680E090E0A1E6B3E4BECF20E048AD55
:10799000BE01635F7F4FCE0109960E9411C54B0166
:1079A0005C01EBA5FCA5EE0FFF1FEE0FFF1F249659
:1079B0008EAD9FAD2497E80FF91F80829182A2823D
:1079C000B382A50194016D8D7E8D8F8D98A10E944B
:1079D0004EF0181624F48D8E9E8EAF8EB8A2A5019F
:1079E000940169A17AA18BA19CA10E9491E787FFD4
:1079F00004C089A29AA2ABA2BCA2A50194016CA961
:107A00007DA98EA99FA90E94AFEE6CAB7DAB8EAB1A
:107A10009FAB8FA198A5092E000CAA0BBB0B8FA3BF
:107A200098A7A9A7BAA7BC01CD010E9497E76BA7A9
:107A30007CA78DA79EA79B01AC016CA97DA98EA9EF
:107A40009FA90E9429EF2B013C014D8A5E8A6F8A13
:107A5000788E2496AEADBFAD2497B8ABAFA710E03B
:107A6000C12CD12C7601EFA5F8A96191719181917A
:107A70009191F8ABEFA7A30192010E94AEEE9B019A
:107A8000AC010E94F6E79B01AC01C701B6010E9460
:107A9000AFEE6B017C011F5FF9A9F11720F72BA551
:107AA0003CA54DA55EA50E9429EF0E948DF0698F2F
:107AB0007A8F8B8F9C8F2DA12230A0F16FA178A59A
:107AC00089A59AA50E9474B081E396E00E9499343A
:107AD00067966CAD7DAD8EAD9FAD67970E9474B01B
:107AE0008BE296E00E94993443E0C501B4010E9404
:107AF000BEB280E20E94783481E03DA133300CF4C4
:107B000080E0E12C8E010F5D1F4F9E01235E3F4FF1
:107B1000AE01475E5F4FBE016B5E7F4F04DC8AE0C3
:107B20000E94783489A98F5F89AB7ACD0E940028A2
:107B300080E296E00E94993481E09DA119160CF034
:107B400080E0EE24E3948E010F5D1F4F9E01235EC3
:107B50003F4FAE01475E5F4FBE016B5E7F4FE3DB81
:107B6000698D7A8D8B8D9C8D0052110926E042E043
:107B70000E946EE29F938F938FE096E09F938F9386
:107B800089E196E09F938F931F920E940E9E0E9420
:107B9000CD8529968FAD29970E94582A0E9401878A
:107BA00046CC8F929F92AF92BF92EF92FF920F932B
:107BB0001F93CF93DF9386EC94E00E949934C0E04A
:107BC000D7E0D15021F080E20E947834FACF8C2F98
:107BD0000E947B28CF5FC73099F78AE00E947834F3
:107BE00000EB14E0C0E080E20E9478348C2F0E9409
:107BF0007B287801D7E080E20E947834F70180800A
:107C00009180A280B38020E030E0A901C501B401D9
:107C10000E944EF087FD03C08BE20E94783443E05F
:107C2000C501B4010E94BEB2D150FCE1EF0EF11CBF
:107C3000D111E1CF8AE00E947834CF5F0C5F1F4FF3
:107C4000C73089F68AE00E947834DF91CF911F9186
:107C50000F91FF90EF90BF90AF909F908F900895FD
:107C6000811107C08FEB94E00E9499348AE00C9454
:107C7000783483EC94E0F8CF88EB94E00C9499345A
:107C800082EB94E00C949934CF9384E50E945F1AC0
:107C9000C0E08823F1F00E94351EC82F1816CCF4DE
:107CA000EFDF8DE40E9478348091190490911A04DA
:107CB0000E94332C83EC98E00E9499346C2FCC0FF7
:107CC000770B880B990B0E9474B08AE00E9478347D
:107CD000CFEF8C2FCF910895CF93C82F6AE978E02A
:107CE0000E94EBC2C11101C0CBDF40918D125091B7
:107CF0008E1260918F127091901281E998E00E942B
:107D0000C43420E030E543EC50E46091911270916E
:107D1000921280919312909194120E94F6E7AB0117
:107D2000BC018EE898E00E94C4342CEA35EC47E2AE
:107D30005EE36091951270919612809197129091E6
:107D400098120E94F6E7AB01BC018BE898E00E9414
:107D5000C4348AE00E947834CF910895CF93DF93A2
:107D6000EB010E949934BE01DD0F880B990B0E9434
:107D700074B0DF91CF9108950E94EE6F0E945C8BEA
:107D800080912207813099F077DF8BE394E00E94A5
:107D9000993460E081E394E00E942B9E6EE571E0EF
:107DA00080E090E00E940E2C81E0809322070895ED
:107DB000CF92DF92EF92FF921F93CF93DF9300D089
:107DC00000D0CDB7DEB78EEEC82E82E0D82EE12CE3
:107DD000F12CC982DA82EB82FC82BE016F5F7F4F99
:107DE0008AE50E943F3381110EC010E0812F0F9071
:107DF0000F900F900F90DF91CF911F91FF90EF9018
:107E0000DF90CF9008950E94A233C982DA82EB827C
:107E1000FC82BE016F5F7F4F8AE50E943F33182FBF
:107E2000882319F329DF8CE195E00E949934A4DFBF
:107E3000DDCFCF92DF92EF92FF921F93CF93DF932C
:107E400000D000D0CDB7DEB78EEEC82E82E0D82E9F
:107E5000E12CF12CC982DA82EB82FC82BE016F5FD9
:107E60007F4F8AE00E943F3381110EC010E0812FC6
:107E70000F900F900F900F90DF91CF911F91FF9077
:107E8000EF90DF90CF9008950E94A2330E945D335F
:107E90000E9474330E945D33C982DA82EB82FC82D5
:107EA000BE016F5F7F4F8AE00E943F33182F882307
:107EB000E9F2E2DE8FED94E00E9499345DDFD7CFE6
:107EC000EC018B01F42E0E94EE6F209709F47CC028
:107ED000D7DECE010E9499348AE00E9478340115E1
:107EE000110511F40FE01FE20E94F01E1F930F9383
:107EF000DF93CF9381E094E09F938F9381E08F9302
:107F00000E940E9E0E94CD8DC0914713C695C695C6
:107F100082E493E10E948721DC2FDD0F1D2F1C0FCF
:107F20008DB79EB707960FB6F8949EBF0FBE8DBF54
:107F300083E00E944E2010927D13C0937E1387E150
:107F400090E10E94942510927D13D0937E136FEFE1
:107F50007FEF82EF93E00E943F2410927D131093F5
:107F60007E136FEF7FEF85EE93E00E943F2486E45F
:107F700093E10E94F1CF8111DBCF7EDE81E194E0BD
:107F80000E94993489EE93E0019739F000C0000017
:107F9000EEE5F9E03197F0F7F7CFF89489EE93E04A
:107FA000019739F000C00000E6EEF3E03197F0F7FA
:107FB000F7CF0E94EE6FFF2021F00E943A72A89541
:107FC000FECF0E94F571FBCF0115110511F40FE0F2
:107FD0001FE2C8E0D4E088CF80918B0D90918C0D8A
:107FE0002FEF3FEF981751F0E92FF0E0E557F24FF0
:107FF000228130E09F5F9F7790938C0DC901089597
:108000001F920F920FB60F9211240F900FBE0F9078
:108010001F9018951F920F920FB60F9211240BB656
:108020000F922F938F939F93EF93FF939091C6009E
:1080300020918C0DE0918B0D81E08E0F8F772817AA
:1080400029F0F0E0E557F24F9283E82FE0938B0D93
:10805000FF91EF919F918F912F910F900BBE0F90F9
:108060000FBE0F901F9018958EBD0DB407FEFDCF6B
:1080700008958FEF8EBD0DB407FEFDCF8EB5089528
:10808000909164009B7F90936400982F906A9695DE
:108090009CBD80FD03C091E0863009F490E09DBD59
:1080A0000895A8E0B0E0E7E5F0E40C9477EEB82E90
:1080B0008091740E843008F0F6C131E6D32E8091A1
:1080C000740E843008F021C180918B0D90918C0D3D
:1080D000891B8F7709F419C17FDF97FF0AC0CCDDB8
:1080E00081E393E00E94993480918B0D80938C0DF5
:1080F000E6CF8A3019F08D3009F0FEC01092730E71
:108100008091110E9091120EFC01E35FF14F1682E7
:10811000892B19F40E947770D2CF1092120E109210
:10812000110E03E11EE0F8018191803209F446C08E
:108130008E3409F09DC06CE273E0C8010E9410E724
:108140007C01892B41F06EE470E0C80104960E9426
:1081500043F1009709F4C8014AE050E070E060E0A4
:1081600001960E9485E42B013C0180910D0E9091B7
:108170000E0EA0910F0EB091100E0196A11DB11D13
:10818000481659066A067B0629F060E089EF92E0FE
:10819000EF2851F16AE270E0C8010E9472F19C017F
:1081A000009729F1982F901BF12C992349F09150B9
:1081B000F801E90FF11D8081F826F7CF8F01B3CFC9
:1081C0004AE050E070E060E0C90101960E9485E459
:1081D0002F2D30E050E040E06217730784079507C9
:1081E00051F060E08AED92E00E947EC268CF60E0CC
:1081F00080EB92E0F9CF40920D0E50920E0E6092FD
:108200000F0E7092100E809122078130E1F467E426
:1082100070E0C8010E9443F10097A9F04AE050E0E5
:1082200070E060E001960E9485E46230710581058E
:10823000910548F48FE092E00E94993460E085E077
:1082400092E00E942B9EF80180818D3481F583811C
:10825000823309F445C0883301F1803341F58181CF
:10826000843329F58281813311F50E94DD861FC098
:108270008091981480FFC7CF64EB7EE2C8010E9412
:1082800010E7009731F0FC01838180538A3008F0B9
:10829000BACF60E086E892E0A7CF8281803339F4DC
:1082A0008181813321F410926601109278048091CB
:1082B000130E8B3309F403CF8091740E843008F0D1
:1082C000FECE8091760E8D9DC001112463E17EE08B
:1082D0008958914F0E944EF180E00E943EC2EFCE3D
:1082E0008281813321F78181813309F741E070E098
:1082F00060E088E49AE0E4DD21E13EE043E15EE015
:1083000063E77EE00E946A19DACE8091981483FDBB
:10831000CAC082FFC8C087FDC6C01A82198281E622
:10832000F82E94E0E92E29E6D22E8091740E843046
:1083300008F0B9C00E94A2198111B5C041E050E017
:10834000BE016D5F7F4F8BE992E10E945ED60B818B
:1083500010E0019711F00FEF1FEF8091A3129091A1
:10836000A412A091A512B091A61280939414909398
:108370009514A0939614B09397140E94A2190F3FDE
:10838000100741F4811106C077DC89E493E00E9474
:108390009934CBCF4091760E242F30E00A3061F033
:1083A0000D3051F0882309F470C089819A810097BB
:1083B00019F001969A8389831092A50389819A8185
:1083C000F29EF001F39EF00D1124EC58F14FDF0105
:1083D000A80FB91F13961C92892BA9F50E947770DC
:1083E0000E94A219882309F4A0CF8BE992E10E9490
:1083F000A66B80918F148823F1F1815080938F14A4
:108400008D9DC001112462E08059994F0E945FD96F
:10841000E0918F1424E0E29FF0011124E459F94F18
:1084200040815181628173814093941450939514DB
:1084300060939614709397148BE992E10E9463D530
:108440000E943ED172CF1A82198283818D3479F4D1
:108450008481823361F48581853349F48681805338
:108460008A3028F0809198148B7F8093981481E053
:108470000E943EC2B5CF0E9430D18091981488608E
:1084800080939814E092220750CF4F9DA0011124B1
:108490004958514F9E012F5F3F4F65EA73E0802F8F
:1084A0000E946A1942CF0E94E0CC6B017C01BB2084
:1084B00041F0C0921C04D0921D04E0921E04F09280
:1084C0001F048091F3039091F403A091F503B09100
:1084D000F6030097A105B10529F140911C045091C4
:1084E0001D0460911E0470911F04840F951FA61F28
:1084F000B71FA7019601281B390B4A0B5B0BDA014A
:10850000C901B7FD0FC0B8DB6091610770916207C8
:1085100088E593E00E940FD940E070E060E090E0D1
:1085200080E0E9CE8091190190911A01A0911B0180
:10853000B0911C01892B8A2B8B2B79F090912E13F3
:1085400080912F13981709F4C4C0C0921C04D092D4
:108550001D04E0921E04F0921F048091AA039091E2
:10856000AB03A091AC03B091AD0346015701881A4B
:10857000990AAA0ABB0AD501C401B7FDC0C19091EE
:108580002E1380912F1320910801981709F4D5C05C
:10859000E0912F133BE5E39FF0011124EA51F84FDE
:1085A0008081281799F0809308010E94E0CCB09058
:1085B00008010B2D10E084E00E949FB20115110507
:1085C00009F0BEC060E084E00E94FBCB80917E0594
:1085D000882309F487C100912F0110913001C8014F
:1085E000029720918A1230918B12281739070CF4C8
:1085F00079C180902F138C82812C912C5401809111
:108600002E132C81821709F4FDC0822F90E03BE5E8
:10861000389FF001399FF00D1124E057F84F45893C
:1086200056896789708D452B462B472B81F4418DE8
:10863000528D638D748D452B462B472B41F4458D10
:10864000568D678D70A1452B462B472BE9F14BE5E5
:10865000489F9001499F300D1124C9018057984FC0
:108660001C01FC0161817281838194810E948DF0E3
:108670006D837E838F839887F10161A172A183A1AD
:1086800094A10E9495E72B013C01F10165A176A11F
:1086900087A190A50E9495E79B01AC01C301B2019F
:1086A0000E9429EF2D813E814F8158850E94F6E777
:1086B0002B013C01AC019B01C501B4010E944EF0AD
:1086C00087FF02C0530142018C818F5F8F708C83C2
:1086D00096CFBB2019F01092AE033FCF0E94E0CCA2
:1086E00000911C0410911D0420911E0430911F0460
:1086F0008090190190901A01A0901B01B0901C016C
:10870000080D191D2A1D3B1D601B710B820B930B5D
:1087100097FDE1CF8091AE0381111FCF81E080935F
:10872000AE0380E00E940A7281E00E940A7282E039
:108730000E940A720E94F57110CF80917F0731CF9D
:108740000F3F110511F461E03ECFE3EFFEE2E4914B
:10875000E150EA3008F051C0F0E0EF54FC4B0C94CB
:108760005CEEBB43C043C543CF43FD43FD43D94308
:10877000E143E943F34384B5806884BDB7BC26CFA9
:1087800084B5806284BDB8BC21CF809180008068B0
:1087900080938000109389000093880017CF809108
:1087A000800080628093800010938B0000938A0089
:1087B0000DCF8091B00080688093B000B092B3007C
:1087C00005CF8091B00080628093B000B092B40079
:1087D000FDCE809190008068809390001093990066
:1087E00000939800F3CE8091900080628093900077
:1087F00010939B0000939A00E9CE003811050CF00D
:10880000A2CFE0CEB801110F880B990B0E9497E719
:108810002B013C012091290130912A0140912B012B
:1088200050912C01C501B4010E94F6E7A301920109
:108830000E94AFEE4B015C0100912D0110912E01C1
:10884000AC019B01C301B2010E944EF018168CF0DE
:10885000B801012E000C880B990B0E9497E72B01A1
:108860003C01A50194010E9491E7181614F424011B
:1088700035018090A6039090A703A090A803B09024
:10888000A903A3019201C501B4010E944EF018167C
:10889000D4F420E037ED43EA5CE3C301B2010E9467
:1088A000F6E72B013C0128E431EE4AE75FE3C5011E
:1088B000B4010E94F6E79B01AC01C301B2010E9422
:1088C000AFEE2B013C014092A6035092A7036092A9
:1088D000A8037092A903C301B2010E9491EFCB01DA
:1088E0000E9421CDF4E6CF0ED11CE11CF11CC092F8
:1088F000AA03D092AB03E092AC03F092AD030E94C6
:10890000777080912207882309F4D0C01091090163
:10891000113061F18091981480648093981481E003
:108920008093090164EF71E080E090E00E940E2CDA
:108930000E9453D38091981484FFCDC0123028F444
:1089400060E085E993E00E942B9E83E080936701BD
:108950000E94E0CC6C597F4F8F4F9F4F60936D0406
:1089600070936E0480936F04909370040E94E0CC27
:108970006B017C01109118011123F1F08091F80333
:108980008823D1F04091AF035091B0036091B103BF
:108990007091B20346015701841A950AA60AB70AD4
:1089A000B501A40177FD1AC0833009F490C00CF022
:1089B00081C081300CF085C0212F30E0A8EEB3E0FB
:1089C0000E940DEEC60ED71EE81EF91EC092AF0320
:1089D000D092B003E092B103F092B2030E94BA21A8
:1089E0008091F203882379F10E94E0CC6B017C0135
:1089F0008091EE039091EF03A091F003B091F10309
:108A0000A7019601281B390B4A0B5B0BDA01C90140
:108A1000B7FD19C02091F20330E0A8EEB3E00E9448
:108A20000DEEC60ED71EE81EF91EC092EE03D092C0
:108A3000EF03E092F003F092F10380E00E94636F95
:108A40008AE00E9478348091ED03882379F10E94B6
:108A5000E0CC6B017C018091E9039091EA03A09145
:108A6000EB03B091EC0346015701881A990AAA0A50
:108A7000BB0AD501C401B7FD19C02091ED0330E058
:108A8000A8EEB3E00E940DEEC60ED71EE81EF91E3A
:108A9000C092E903D092EA03E092EB03F092EC0378
:108AA0000E942BB380E393E10E943C712896E2E19F
:108AB0000C9493EE843009F07FCFE2D884EA93E0FF
:108AC00003C0DED883ED93E00E94993475CFD8D8E7
:108AD0008CEB93E0F9CF112309F448CF36CFA2E114
:108AE000B0E0E5E7F5E40C9478EE9091400D93FD4D
:108AF0007EC0082FC9D8182F87FD79C089E40E944D
:108B00005F1A882309F48BC00E94351E282F30E09D
:108B10001216130614F421E030E0220F331F220F47
:108B2000331FF901E855FB4F80819181198A0E941A
:108B300021CD80918A1290918B128635910574F027
:108B4000002381F00E94148B0DC082E50E945F1A01
:108B5000882309F46CC00E94701EE9CF0E945C8BD0
:108B60000E9499C360918A1270918B12072E000C9B
:108B7000880B990B0E9497E72091861230918712FB
:108B800040918812509189120E944EF0181644F0BC
:108B9000298984E09FE0222329F049894A8B48C033
:108BA0008FE09FE09F938F938AE19FE09F938F9345
:108BB0001F920E940E9E0F900F900F900F900F909B
:108BC00031E03A8B35C060E070E0CB014FC0C701A7
:108BD000B6010E9491E787FF0EC08091660188234D
:108BE00021F0109266010E9499C330927E05629630
:108BF000E1E10C9494EE4601570100E098C08FE348
:108C00000E947834CFC020E030E040E450E40E947D
:108C10004EF018160CF004C12601370101C183E59E
:108C20000E945F1A898B811196CF01118ECF1A8A0B
:108C300083E50E945F1A882331F00E94701E909392
:108C4000300180932F0182E40E945F1A882331F063
:108C50000E94701E90932E0180932D0186E40E9445
:108C6000E819882309F4AFCF0E947F1E6093290181
:108C700070932A0180932B0190932C013324339419
:108C800020E030E0A9010E9491E7811101C0312C60
:108C900030927E05002309F4AACF5A89552309F49E
:108CA000A6CF10927E0581E0809366011D821E8210
:108CB0001F82188619861A861B861C8680E09CE314
:108CC000ACE1B6E48D879E87AF87B88B812C912C61
:108CD00090E8A92E9FEBB92E00E0412C512C3201D7
:108CE00060918A1270918B12072E000C880B990BE1
:108CF0000E9497E76B017C01A50194010E9491E716
:108D00008823A9F020918612309187124091881211
:108D100050918912998991115ACFC701B6010E94C9
:108D200091E7082F001F0027001F460157010E94EE
:108D3000E0CC6B017C01DC01CB0129853A854B85B8
:108D40005C85821B930BA40BB50BB7FD2EC0D7011E
:108D5000C60188519C4FAF4FBF4F89879A87AB8719
:108D6000BC87812F0E94636F80E29FE00E9499344C
:108D7000411451046104710409F441CFC301B201EB
:108D8000605F784D8F4F9F4F6C197D098E099F0949
:108D900028EE33E040E050E00E94BFEDCA01B90187
:108DA0000E949C268AE00E94783480E07AD90E9452
:108DB000E0CC60931C0470931D0480931E04909378
:108DC0001F04209186123091871240918812509191
:108DD000891229833A834B835C83C501B4010E94C5
:108DE000AEEE9F77411451046104710409F00BCF7A
:108DF00020E030E040E85FE30E9491E787FF10C089
:108E00003A89412C512C3201332331F085E0482E30
:108E10008DE0582E612C712C4C0C5D1C6E1C7F1C3F
:108E20000023C1F18D819E81AF81B885892B8A2B6A
:108E30008B2B61F0D701C6012D813E814F81588572
:108E4000821B930BA40BB50BB7FD24C029813A817B
:108E50004B815C816D857E858F8598890E94AEEE01
:108E600020E030E040EC5FE30E9491E787FDB5CE63
:108E7000D701C601805A9541AF4FBF4F8D839E8366
:108E8000AF83B88729813A814B815C812D873E87EA
:108E90004F87588B80916601882309F49ECE411438
:108EA00051046104710461F030E1C31A37E2D30A5E
:108EB000E108F108C418D508E608F708F7FE8DCEDA
:108EC0001A8A0ECFA5E4B0E0E8E6F7E40C9477EE5A
:108ED00026968FAF26972091F80328AB81E08093E8
:108EE000F80380911B048D3409F4EEC4843511F429
:108EF0000C947B5C873491F48091190490911A044E
:108F00008D31910509F45DC308F0E1C1843091050C
:108F100009F401C330F4029708F45AC20E9401D93F
:108F2000D2C28531910509F4CEC24C97B9F787E0DA
:108F30000E946082811111C08091130490911404E9
:108F4000A0911504B0911604EEE0B695A7959795FB
:108F50008795EA95D1F780FDB6C20E94A073109262
:108F60003C0160919F048CE40E945F1E982E80E07B
:108F70000E94582A0E94E0CC60931C0470931D0448
:108F800080931E0490931F040E94E68581E08093E5
:108F9000DB060E94F287C0901304D0901404E09086
:108FA0001504F090160479E1F694E794D794C794E9
:108FB0007A95D1F7C0FE0DC081E00E946082182F23
:108FC00082E00E94608211110C94B85C11E0811162
:108FD00001C010E08091130490911404A091150435
:108FE000B091160467E1B695A795979587956A9510
:108FF000D1F780FF02C00C949E5C1111C6C2809113
:10900000130490911404A0911504B09116043B2F01
:109010003170A32E3113BBC28C2D8170A12E811310
:10902000B6C211E0AA24A394BB24B39482E50E94A3
:109030005F1A882309F4AFC20E947F1E68A379A338
:109040008AA39BA320E030E0A9010E9491E7882336
:1090500079F0111105C0A11003C0BB2009F424C18F
:10906000CE0180960E944BC30E94A2330E945D33C2
:10907000112309F489C0AA2009F483C01092720157
:109080001092730110927401109275011092760182
:109090001092770110927801109279010E94B386A4
:1090A0008BE39DE10E94FA276B017C018FE39DE138
:1090B0000E94FA272B013C01AC019B01C701B601BC
:1090C0000E944EF018160CF06BC2A7019601C30166
:1090D000B2010E9429EF9B01AC010E94F6E720E05B
:1090E00030E040E85FE30E94AFEE0E948DF021E0A7
:1090F00030E048E452E40E94F6E769837A838B8388
:109100009C8380917A0190917B01A0917C01B09128
:109110007D018CA39DA3AEA3BFA320E030E040EC73
:109120005FE3C301B2010E94F6E72B013C0177FA2D
:10913000709477F8709420E030E040EC5FE3C70172
:10914000B6010E94F6E79058DE0111966D01ECA081
:10915000FDA00EA11FA1A30192010E9405860E94FD
:10916000918A109272011092730110927401109200
:109170007501109276011092770110927801109289
:10918000790180E00E945F89AA2019F081E00E94A5
:109190005F89BB2009F488C083E00E947B82811133
:1091A00083C00E94B38680917A0190917B01A09147
:1091B0007C01B0917D0180938F0490939004A093E3
:1091C0009104B09392040091291310912A13F8018D
:1091D000C080D180E280F380A701960160E070E05A
:1091E00080EE92E40E94AEEE609383047093840458
:1091F0008093850490938604D80114964D905D90D9
:109200006D907C901797A301920160E070E080EE72
:1092100092E40E94AEEE609387047093880480937A
:10922000890490938A042DE030E044EE52E4C301B7
:10923000B2010E944EF018160CF4B7C12EE030E0D7
:1092400042EE52ECC301B2010E9491E787FDADC12D
:109250002DE030E04EEE52E4C701B6010E9491E7E6
:1092600018160CF4A2C12EE030E042EE52ECC70119
:10927000B6010E944EF087FD98C11C8E1D8E1E8E79
:109280001F8E88E0E3E8F4E0DE01119601900D9274
:109290008A95E1F7BE01645E7F4FCE0101960E9480
:1092A00080C682E00E945F890E94B3868091DA06C0
:1092B0008093DB06992019F081E00E94582A0E94D1
:1092C000CD8583E0809367010E940187FCC08A35C9
:1092D000910509F4EAC250F58E31910509F474C183
:1092E0008A9709F01BCE80912207833008F4EBC0E7
:1092F00089E40E945F1A082FF12C882319F00E943C
:10930000701EF82E8AE40E945F1AE82E882309F462
:10931000CAC10E94701E182F0111C8C1173008F46D
:10932000CBC184E199E00E949934CDC08B35910581
:1093300009F4BEC28C35910509F0F0CD42E9242E26
:1093400041E0342E52E7E52E51E0F52EC12CD12C10
:1093500010E0F10181911F010E945F1A082F8823FC
:1093600049F10E947F1E2B013C01D7012D913D91B7
:109370004D915C910E94AEEE4B015C012DEB37E309
:1093800046E855EB0E9491E787FD0AC02DEB37E3D5
:1093900046E855E3C501B4010E944EF0181654F496
:1093A000133011F0C02E0D2DF701408251826282E0
:1093B0007382D02E1F5FF4E0EF0EF11C143049F6DB
:1093C000CC2009F479C20E94B3860E9401877BC039
:1093D00080912207833008F476C0F3E8CF2EF4E0C2
:1093E000DF2EA2E7EA2EA1E0FA2E10E088E5810F39
:1093F0000E945F1A882309F472C00E947F1E4B01ED
:109400005C01812F0E94C119882359F0D7012D9149
:109410003D914D915C91C501B4010E94AFEE4B01AD
:109420005C01F60180829182A282B3821F5FF4E028
:10943000CF0ED11C24E0E20EF11C1330B9F685E406
:109440000E945F1A882309F455C00E947F1E6B0199
:109450007C0183E00E94C119882371F020917E0174
:1094600030917F014091800150918101C701B60187
:109470000E94AFEE6B017C01C0928F04D0929004E9
:10948000E0929104F092920440E050E0BA0186E448
:109490000E94A71E20E030E0A9010E944EF018169D
:1094A00084F40E947F1E29E838E848E85CE30E94C3
:1094B000F6E76093350170933601809337019093FE
:1094C00038010E94BE8226969FAD2697911102C058
:1094D0000E9438C3A8A9A093F8030C947D53F70108
:1094E00080819181A281B381F60180839183A283DF
:1094F000B3839CCF80917E0190917F01A0918001E8
:10950000B091810180938F0490939004A093910473
:10951000B0939204B9CF80E50E945F1AC12CD12C80
:109520007601882321F00E94151E6B017C0183E5E2
:109530000E945F1A882361F00E947F1E20E030E0C5
:109540004AE754E40E94F6E70E9496EF6B017C0123
:109550000E94A07380911710811105C060E086ED14
:1095600098E00E942B9E0E94E0CCC60ED71EE81EFB
:10957000F91E0E94E0CC6C197D098E099F0997FFA6
:10958000A2CF80E00E945140F4CFA12E10E04C2DDC
:109590004170B42E4BCD60E070E080EA90E44ECD97
:1095A000A3019201C701B60194CD60E081EF98E07C
:1095B0000E942B9E0E94403E8FED98E00E949934BD
:1095C00073CE0E94145D7FCF0091291310912A134E
:1095D000F801208131814281538160917201709143
:1095E000730180917401909175010E94AFEEAB01FF
:1095F000BC0188E50E94A71E69837A838B839C83C4
:10960000D80114962D913D914D915C9117976091E1
:1096100076017091770180917801909179010E9493
:10962000AFEEAB01BC0189E50E94A71E6D837E836E
:109630008F839887BE016B5F7F4FCE0101960E949A
:10964000DBC3882309F43FCF80E00E94582A0E94A0
:10965000E68561E085E40E945F1E21E0482FBE019F
:109660006B5F7F4FCE0101960E9411C56B017C019B
:1096700049815A816B817C818CE099E00E94C434DD
:109680004D815E816F81788587E099E00E94C434C6
:10969000B701A60182E099E00E9403350E94CD85C2
:1096A0000E94018710CF10E0002331F0B6E0BF1513
:1096B00008F437CEE11032CE80E1E2E7F1E0A3E832
:1096C000B4E001900D928A95E1F7002319F16F2D16
:1096D000FF0C770B880B990B0E9497E72091A00451
:1096E0003091A1044091A2045091A3040E94F6E796
:1096F00020919304309194044091950450919604E4
:109700000E94AFEE60938304709384048093850479
:1097100090938604EE2019F1612F110F770B880BBF
:10972000990B0E9497E72091A4043091A5044091E1
:10973000A6045091A7040E94F6E720919704309167
:1097400098044091990450919A040E94AFEE60935E
:109750008704709388048093890490938A0460E05E
:1097600080E50E945F1E8823C1F10023D1F0E091C3
:109770002913F0912A132081318142815381609114
:1097800083047091840480918504909186040E94E2
:10979000AEEE609383047093840480938504909369
:1097A0008604EE20D1F0E0912913F0912A13248150
:1097B000358146815781609187047091880480913A
:1097C000890490918A040E94AEEE6093870470939E
:1097D00088048093890490938A0440E050E0BA01A1
:1097E00086E40E94A71E6B017C0120E030E0A90105
:1097F0000E944EF087FF03C0C12CD12C760129E8CE
:1098000038E848E85CE3C701B6010E94F6E76B015F
:109810007C018090350190903601A0903701B09086
:10982000380120E030E0A9010E9491E7882341F04F
:10983000C0923501D0923601E0923701F0923801A2
:109840000091390110913A0184E690E090933A0139
:1098500080933901C0906C01D0906D01E0906E0151
:10986000F0906F0180E090E0A0E8BFE380936C018E
:1098700090936D01A0936E01B0936F010E94BE8220
:109880008092350190923601A0923701B092380152
:1098900010933A0100933901C0926C01D0926D018E
:1098A000E0926E01F0926F010ECE1092F7030BCE94
:1098B0008FE08093F70307CEDD2009F486CD8EE795
:1098C00091E00E94B78081CD8091190490911A0493
:1098D0008237910511F40C949D5508F06FC18B34BB
:1098E000910509F4E2C608F0E9C08831910509F450
:1098F00005C508F0BAC08231910509F4EDC708F03A
:109900006EC08230910508F46FC4419709F006CB10
:109910000E94D719882309F4C3C40E94361A009103
:109920007505102F1095182309F4CDCDF12CE12CDD
:10993000D12CA12EB12CC5010E2C02C09595879576
:109940000A94E2F780FF08C08E2D0E944172F70151
:10995000E15EFD4F8081D82A5FEFE51AF50A83E0CA
:10996000E816F10441F713FF05C00E9403729D2D14
:109970009360D92E102B10951D2109F4A4CD88E2F7
:109980000E947834F12CE12CC12ED12CC6010E2C72
:1099900002C0959587950A94E2F780FF09C0F70108
:1099A000EE56FE4F80810E94783480E20E94783427
:1099B000AFEFEA1AFA0AB3E0EB16F10439F713FF36
:1099C00009C085E40E94783480E30E94783480E204
:1099D0000E94783480E499E00E94993474CD8531F6
:1099E000910509F475C458F5449709F097CA809118
:1099F000981484FF66C481E799E00E9499348091AD
:109A0000981484FF17C081ED92E10E94D56C8BE120
:109A1000E1EDF2E1DE01119601900D928A95E1F7F8
:109A200070E060E0CE0101960E9487DACE010196D7
:109A30000E94A56E82E699E00E94993444CD863159
:109A4000910509F448C4479709F068CA8091170442
:109A500090911804FC012191222309F44BC4203277
:109A6000D1F7DF0111971C92F6CF8D31910509F4E2
:109A7000D3C4A0F48A31910509F459C408F449C447
:109A80008B31910509F46EC44C9709F047CA809157
:109A90001704909118040E9414D915CD8F319105A7
:109AA00009F45DC508F4BEC48032910509F412C5FD
:109AB000C09709F033CA0E94003A05CD8836910557
:109AC00009F4FFC508F046C08235910509F4F4C6D3
:109AD000F0F48D34910509F4F0C508F4EAC5813538
:109AE000910509F01BCA0E94B17310927F070E9472
:109AF000EE6F0E945C8B68EE73E080E090E00E9465
:109B00000E2C60E08DE59AE00E942B9EDCCC843523
:109B1000910509F4E1C608F4D7C68535910509F425
:109B200075C78C35910509F0F9C90E94443E87FD3F
:109B3000CACC8091130484FD8EC78091150487FDE3
:109B40008AC780911604837009F085C781E00E945E
:109B50000BC3B9CC8D36910509F4B8C598F48A3693
:109B6000910509F4CFC508F4B6C58B36910509F403
:109B700002C68C36910509F0D1C910927804109272
:109B80006601A1CC8F36910509F413C608F4FEC511
:109B90008037910509F449C68137910509F0BEC99E
:109BA00083E50E945F1A882309F44FC60E94351E80
:109BB0008D3308F045C68093180185CC8D3221E0A5
:109BC000920711F40C94085908F0F1C18B399105F2
:109BD00009F44BC608F0F3C08737910509F4FEC7B6
:109BE00008F0BAC08537910509F4AFC708F0BDC7C2
:109BF0008337910509F092C989E29CE00E9499346B
:109C000060E089E19CE00E94AF3460E084E09CE089
:109C10000E94AF3461E08DEF9BE00E94AF3460E0C2
:109C200082EF9BE00E94AF3461E083EE9BE00E94F4
:109C3000AF3461E083ED9BE00E94AF3460E08AECDA
:109C40009BE00E94AF3461E080EC9BE00E94AF3467
:109C500061E086EB9BE00E94AF3460E08FEA9BE01E
:109C60000E94AF3461E087EA9BE00E94AF3461E07C
:109C700089E99BE00E94AF3460E08BE89BE00E94A2
:109C8000AF3460E08CE79BE00E94AF3460E08EE68A
:109C90009BE00E94AF3460E088E59BE00E94AF3417
:109CA00060E087E49BE00E94AF3460E082E39BE0E9
:109CB0000E94AF3460E083E29BE00E94AF3461E039
:109CC0008CE19BE00E94AF3460E085E19BE00E9464
:109CD000AF3461E08CE09BE00E94AF3460E087EF3E
:109CE0009AE00E94AF3460E089EE9AE00E94AF34BF
:109CF00060E08CED9AE00E94AF3461E089EC9AE07C
:109D00000E94AF3460E08CEB9AE00E94AF3460E0D8
:109D100087EB9AE00E94AF3461E08AEA9AE00E9401
:109D2000AF3460E086E99AE00E94AF3460E083E8F7
:109D30009AE00E94AF3460E087E792E10E94BE198A
:109D4000682F61708AE79AE00E94AF3460E08CE689
:109D50009AE00E94AF34B7CB8937910509F44BC71D
:109D600008F440C78139910509F44DC78A39910536
:109D700009F0D4C883E50E945F1A882309F4A3CBB5
:109D80000E94351E182F8C3308F08CE38093ED036E
:109D90000E94E0CC6B017C01212F30E0A8EEB3E003
:109DA0000E940DEEC60ED71EE81EF91EC092E903F2
:109DB000D092EA03E092EB03F092EC0384CB833D74
:109DC000910511F40C946757B0F58B3C910509F49B
:109DD00099C7B0F4893C910509F0A0C8809113049B
:109DE00084FD66C780911504887809F061C7809169
:109DF0001604837009F05CC781E00E945C3963CB74
:109E00008C3C910509F4B2C78D3C910509F086C8D8
:109E10008091130481FF01C0FEC78091140481FF6B
:109E200001C0F9C7809115048C7009F0F4C781E076
:109E30000E94E13848CB8D3D910511F40C94FB57FD
:109E400008F045C08C3D910509F068C882E40E9485
:109E5000E819882341F08091390190913A0190935B
:109E60001E0180931D0182E50E94E819882341F0BC
:109E700080911D0190911E0190933A0180933901C8
:109E800083E50E945F1A882331F00E94701E909330
:109E90003A01809339018091130490911404A091A8
:109EA0001504B0911604892B8A2B8B2B09F00BCB50
:109EB0006091390170913A0186E59DE00E94AE3EC5
:109EC00085E20E9478348AE00E947834FCCA8831A6
:109ED00041E0940711F40C9448588232914009F003
:109EE0001DC88AE50E945F1A882311F40C94E35878
:109EF0000E947F1E20E030E040E050EC0E944EF0D7
:109F0000C12CD12CE12C40ECF42E87FD13C00E9413
:109F10007F1E20E030E040E050E40E9491E7C12C39
:109F2000D12CE12C30E4F32E181624F00E947F1E71
:109F30006B017C0120915D0D30915E0D40915F0DB4
:109F40005091600DC701B6010E94F6E70E9491EFA3
:109F5000CB010E94BCC361E080E50E945F1E8823A4
:109F600011F40C94E958A7019601609125137091A2
:109F7000261380912713909128130E94AFEE6093CF
:109F800025137093261380932713909328130E9410
:109F9000403E4091251350912613609127137091F4
:109FA000281382E99DE00E9403350C94E958843F10
:109FB000A1E09A0711F40C946C5B08F0A3C08139FE
:109FC000E1E09E0711F40C949C5988F48F3221E053
:109FD000920711F40C94985910F40C94525980394A
:109FE000914011F00C948E470E94A0736CCA8A397C
:109FF00051E0950709F420C450F48239914011F0E2
:10A000000C948E470E9400280E9401875CCA843A03
:10A01000E1E09E0711F40C94A959853A914011F0A2
:10A020000C948E476FEF7FEF89E40E94731E8C01C2
:10A030006FEF7FEF8AE40E94731E7C018AE50E9425
:10A040005F1AD12C811108C081E50E945F1AD82EB9
:10A05000882311F40C94B05CC02E81E0800F88300E
:10A0600010F00C94645BBE2C81E08E0D883010F0F3
:10A070000C94645B102F0E947F1E2B013C01A02ECC
:10A0800007FDA12C17FF02C046E0C42E8E2DE7FC71
:10A09000E12C87FF02C036E0B32E27E0322ECA142F
:10A0A00008F411CAFE2C3A9C40011124BF1410F48C
:10A0B0000C94615B0F2D10E020E030E0A901DD2061
:10A0C00069F0F401E00FF11FEE0FFF1FEE0FFF1F0D
:10A0D000E055FB4F2081318142815381080D191DCC
:10A0E000000F111F000F111F00551B4FC301B201BC
:10A0F0000E94AFEED8016D937D938D939C9313973F
:10A10000F394D4CF8C3022E0920711F40C94825B4C
:10A1100028F5863F41E0940711F40C94745B10F429
:10A120000C94705B873FA1E09A0711F40C94785B64
:10A13000883F914011F00C948E4781E08093740524
:10A140000E94C3A410927405882309F4BCC90E941C
:10A15000403E87E59EE00E949934B5C9803AE3E02D
:10A160009E0709F4EEC1A8F48335934011F00C94D6
:10A170008E478091150487FF02C00C949A5B8091F2
:10A180001604837011F00C949A5B81E00E94D53420
:10A190009AC9873E33E0930711F40C946B5C893EB7
:10A1A000934011F00C948E470E94A07380919814F4
:10A1B000877F8B7F809398140E94C78A6D337105C7
:10A1C0008105910520F08EEC9EE00E94BC5C8AEC3B
:10A1D0009EE00E94BC5C86EB9EE00E94993482EB7C
:10A1E0009EE00E94BC5C6FC980E50E945F1AC12C92
:10A1F000D12C7601882321F00E94151E6B017C0171
:10A2000083E50E945F1A882361F00E947F1E20E090
:10A2100030E04AE754E40E94F6E70E9496EF6B01B3
:10A220007C010E94A07380911704909118040097FC
:10A2300011F10E9419C21091F80383E08093F80392
:10A2400081E080937804C114D104E104F10431F079
:10A250000E94E0CCC60ED71EE81EF91E809178043D
:10A260008823B9F0C114D104E104F10451F480E071
:10A270000E945140F3CF60E08DE299E00E942B9E56
:10A28000DACF0E94E0CC6C197D098E099F0997FDF9
:10A29000EECF109278041093F8030E9499C313C96B
:10A2A00060E08FE499E00E942B9E80E00E94417262
:10A2B00081E00E94417282E00E9441720E9403721A
:10A2C00002C90E94403E88E599E00E949934FBC88B
:10A2D0000E9453D3F8C88091981482FF02C087FF70
:10A2E000F2C80E9430D1809198148F7E8064809350
:10A2F0009814E9C860E00E945FD9E5C80E944B2C21
:10A30000882321F00E943ED10E94148B0E9499C3A1
:10A31000DAC88091981482FF05C087FD03C08B7F47
:10A32000809398140E94478B0E9499C3CCC8809157
:10A33000981484FFC8C883E50E945F1A882309F433
:10A34000C2C80E94251EAB01BC01409394145093D7
:10A35000951460939614709397148BE992E10E9480
:10A3600063D5B1C88091130490911404A091150491
:10A37000B091160432E0B695A795979587953A95D2
:10A38000D1F780FF1CC08FEA99E00E949934809138
:10A390009E12882379F0BE016F5F7F4F8BE992E1B7
:10A3A0000E94C96BCE0101960E947F348AE00E9410
:10A3B000783489C882E899E00E949934F7CF809177
:10A3C000981482FF24C0C0909414D0909514E0900B
:10A3D0009614F09097148DE999E00E949934C70182
:10A3E000B6010E9417B08FE20E94783460919014F9
:10A3F0007091911480919214909193140E9417B0CF
:10A400008DE00E9478348AE00E9478345CC88CE841
:10A4100099E00E94993457C8809198148E7F809358
:10A42000981451C88091981484FF4DC80E944DD54E
:10A430008091981484FF47C84091170450911804E4
:10A44000BE01645E7F4F80E00E9422D88C0100979D
:10A4500009F439C86C8D7D8D19821C8222E0AC0113
:10A46000CE0101960E94AA6E811115C0F12CCE0179
:10A4700001960E94A56EB801FF2011F189ED99E0C7
:10A480000E940FD910929414109295141092961461
:10A490001092971418C8CE0101960E94E8D588231F
:10A4A00029F361E0CE0101960E94AF6B0097F1F2B3
:10A4B00025EEFC0120831C820E947AD1F82ED7CF92
:10A4C00081EC99E00E94A6348EEB99E00E949934C9
:10A4D0000C94634A8091981482FF03C087FF0E9406
:10A4E000A0738091981484FD02C00C94634A60E0CC
:10A4F00080E50E945F1E182F682F809117049091AD
:10A5000018040E945FD983E50E945F1A882381F0B6
:10A510000E94251EAB01BC014093941450939514E6
:10A5200060939614709397148BE992E10E9463D51F
:10A530000E943ED111110C94634A0E94148B0C941A
:10A54000634A2091170430911804909198149260F6
:10A5500090939814C9010E9414D90C94634A0E94E4
:10A56000C78A6B017C0120E831E541E050E00E94A0
:10A57000BFEDC9016DE671E00E9435EE4B015C0153
:10A58000C701B60120E13EE040E050E00E94BFED8F
:10A59000CA01B90128E130E040E050E00E94BFED7F
:10A5A0002B013C011B01C701B6012CE330E040E068
:10A5B00050E00E94BFED6B017C01CA01B9012CE3A0
:10A5C00030E040E050E00E94BFED8E010F5F1F4F72
:10A5D0008114910419F1DF92CF927F936F935F9270
:10A5E0004F92BF92AF929F928F928FE09AE09F938B
:10A5F0008F931F930F930E942AE70FB6F894DEBF44
:10A600000FBECDBFC8010E9419C20E94403EB801D2
:10A6100083E29AE00E940FD90C94634AA114B1041A
:10A6200089F0DF92CF927F936F935F924F92BF92A8
:10A63000AF928FEF99E09F938F931F930F930E9498
:10A640002AE7DBCF4114510479F0DF92CF927F9358
:10A650006F935F924F9283EF99E09F938F931F9335
:10A660000F930E942AE7C9CF6115710569F0DF9247
:10A67000CF927F936F938BEE99E09F938F931F936D
:10A680000F930E942AE7B9CFDF92CF9287EE99E02D
:10A690009F938F931F930F930E942AE70F900F9021
:10A6A0000F900F900F900F90ADCF0E94148B0C94D1
:10A6B000634A0E94478B0C94634A0E945C8B0C9403
:10A6C000634A80E00E946F450C94634A81E00E94D7
:10A6D0006F450C94634A0E94443E182F87FD0AC0C0
:10A6E00080E39AE00E949934812F0E94636F8AE090
:10A6F0000E947834B8A9B093F803CB5BDF4FE2E156
:10A700000C9493EE60E080E50E94461E81110C944B
:10A71000634A8091130490911404A0911504B091A0
:10A72000160460917F07062F10E080FD02C00FEF36
:10A7300010E089E40E945F1A882311F40C94A45C51
:10A740000E94351E90E01816190614F481E090E07E
:10A75000880F991F880F991FFC01E855FB4F028154
:10A7600013810F3F110519F010F00FEF10E0009367
:10A770007F070C94634A60E080E50E94461E8111C9
:10A780000C94634A10927F070C94634A8EE40E94F3
:10A790005F1A882311F40C94634A0E94251E60936B
:10A7A0000D0E70930E0E80930F0E9093100E0C945E
:10A7B000634A83E50E945F1A882321F00E94351EB8
:10A7C0008093400D0E94403E81E49AE00E949934BB
:10A7D0008091400D882331F110E000E020E080916D
:10A7E000400D90E0002E02C0959587950A94E2F7FF
:10A7F00080FF12C0FF24F394F20E222319F08CE2A2
:10A800000E947834F801EE0FFF1FE95CF54F859147
:10A8100094910E9499342F2D0F5F1F4F0530110521
:10A82000F1F6C4CD83E39AE0C7CD41E070E060E08B
:10A8300088E49AE00E94603F0E94DD860C94634A9F
:10A840008CE3809318010C94634A0E94403E10915F
:10A85000180186E59AE00E949934812F0E947B2896
:10A860008AE00E9478340C94634A83E50E945F1A60
:10A87000882311F40C94634A0E94351E182F8C33E0
:10A8800008F08CE38093F2030E94E0CC6B017C0122
:10A89000212F30E0A8EEB3E00E940DEEC60ED71EC9
:10A8A000E81EF91EC092EE03D092EF03E092F0038F
:10A8B000F092F1030C94634A8091F7038F7D8061DD
:10A8C0008093F7030C94634A8091F7038F7E806234
:10A8D0008093F7030C94634A83E50E945F1A8823F0
:10A8E000F1F00E94E0CC60931C0470931D048093EF
:10A8F0001E0490931F040E947F1E20E030E04AE770
:10A9000054E40E94F6E70E9496EF60931901709359
:10A910001A0180931B0190931C010C94634A0E94BE
:10A92000D719882309F46EC00E94A0730E94361ABA
:10A93000082F10917505182311F40C94634AF12C1B
:10A94000E12CC82ED12CAA24A394B12CC6010E2C24
:10A9500002C0959587950A94E2F780FF12C08E2D6C
:10A960000E940A72882369F0F701E15EFD4F808141
:10A9700095010E2C01C0220F0A94EAF7822B8095D4
:10A980001823EFEFEE1AFE0AF3E0EF16F104F1F6EA
:10A9900003FF04C00E94F5718111147FF12CE12C9A
:10A9A000C12ED12CC6010E2C02C0959587950A9414
:10A9B000E2F780FF0FC0F701EE56FE4F80810E9444
:10A9C0007834F701E15EFD4F908180917505892310
:10A9D0000E9435DB2FEFE21AF20A33E0E316F104AE
:10A9E00009F713FD02C00C94634A85E40E94783491
:10A9F00080E30E9478348091750583700E9435DB76
:10AA00000C94634A0E94B1730C94634A83E50E94DC
:10AA1000E819882311F40C94634A0E94E0CC6093F7
:10AA20001C0470931D0480931E0490931F040E94C5
:10AA30007F1E20E030E04AE754E40E94F6E70E94DF
:10AA400096EF6093F3037093F4038093F503909370
:10AA5000F6030C94634AB2E9CB2EB1E0DB2E11E48D
:10AA6000E12E1DE0F12E10E0D6018D916D010E94C6
:10AA70005F1A882349F0133089F00E947F1EF70186
:10AA8000648B758B868B978B1F5FF4E0EF0EF11C48
:10AA9000143051F70E9478730C94634A0E947F1E11
:10AAA0004B015C0120E030E040EA51E40E9491E774
:10AAB00087FF3AC0A50194016091610D7091620D0C
:10AAC0008091630D9091640D0E9429EF2B013C0150
:10AAD000AC019B016091710D7091720D8091730DAD
:10AAE0009091740D0E94F6E76093710D7093720D52
:10AAF0008093730D9093740D609173077091740738
:10AB000080917507909176070E9495E7A3019201C5
:10AB10000E94F6E70E9496EF6093730770937407A4
:10AB200080937507909376078092610D9092620DE5
:10AB3000A092630DB092640DA7CF0E942BB380E367
:10AB400093E10E943C710C94634A809117049091A8
:10AB50001804009709F4DACBDC012C91222309F4C4
:10AB6000D5CB0E9419C20C94634A0091170410912E
:10AB7000180494E0F12C40E09150F9F0F801808144
:10AB8000282F2B7F213499F421812133B1F4813492
:10AB900011F1853409F441E098012E5F3F4F89019E
:10ABA0002F5F3F4FF80180818032C9F3E5CF8035B8
:10ABB00021F4818180538A3078F341110E94403E14
:10ABC000FF2021F080EF9CE00E949934C8010E9490
:10ABD0008A340C94634AFF24F394DECF0E94AC873E
:10ABE0000C94634A81E08093DB068093DA060E942E
:10ABF000F2870C94634A1092DB061092DA060E94E8
:10AC0000F2870C94634A70E060E083E50E94731E53
:10AC1000823040F00E943C3E83EF9CE00E949934D9
:10AC20000C94634A8C01112788E40E945F1A8823E0
:10AC3000A9F00E94701E8A3A910574F10E94701E5C
:10AC4000863F910564F50E94701EF801EE0FFF1F0C
:10AC5000EE0FFF1FE855FB4F9183808386E40E942F
:10AC60005F1A882311F40C94634A0E94701E97FDAA
:10AC700019C00E94701E8F3F910509F0B4F40E9424
:10AC8000701E000F111F000F111FF801E855FB4F38
:10AC9000938382830C94634A8AEA90E0D6CF85EF4F
:10ACA00090E0D3CF90E080E0ECCF8FEF90E0E9CF61
:10ACB0000E94443E87FF02C00C94634A02E911E0FF
:10ACC00051E4E52E5DE0F52E66E9C62E61E0D62E54
:10ACD000D8018D918D010E945F1A882359F00E943E
:10ACE0007F1E0E9496EFF7016083718382839383B6
:10ACF0000E943473F4E0EF0EF11CC016D10641F748
:10AD00000C94634A8091130484FD0DC08091150456
:10AD1000887849F480911604837029F481E00E94B8
:10AD200035390C94634A0E94443E87FF02C00C945C
:10AD3000634A42E9E42E41E0F42E10E000E0D7013E
:10AD40008D917D010E945F1A882349F00E947F1E29
:10AD5000F801EF5BF24F64A375A386A397A30C5F82
:10AD60001F4F0031110559F70C94634A8091140468
:10AD700087FD09C0809115048E7029F481E00E943E
:10AD800015390C94634A83E50E945F1A882391F079
:10AD90000E947F1E6093750D7093760D8093770DE2
:10ADA0009093780D60937D0D70937E0D80937F0D51
:10ADB0009093800D80E50E945F1A882351F00E94D5
:10ADC0007F1E6093750D7093760D8093770D909331
:10ADD000780D82E50E945F1A882351F00E947F1E41
:10ADE0006093790D70937A0D80937B0D90937C0D19
:10ADF00084E50E945F1A882311F40C94634A0E9430
:10AE00007F1E60937D0D70937E0D80937F0D9093D8
:10AE1000800D0C94634A82E40E945F1A882351F0EB
:10AE20000E94151E6093510D7093520D8093530D27
:10AE30009093540D83E50E945F1A882351F00E947D
:10AE40007F1E6093810D7093820D8093830D90938C
:10AE5000840D84E50E945F1A882351F00E947F1EB2
:10AE60006093850D7093860D8093870D9093880D68
:10AE70008AE40E945F1A882311F40C94634A0E94AA
:10AE80007F1E6B017C012AE037ED43E25CE30E9408
:10AE90004EF087FD14C02AE939E949E95EE3C701AC
:10AEA000B6010E9491E7181654F0C0926307D09241
:10AEB0006407E0926507F09266070C94634A0E946B
:10AEC0003C3E85E19DE00E9499340C94634A83E501
:10AED0000E94E819882331F00E94501E80933B01A4
:10AEE0000C94634A10913B01105D8DE49DE00E943B
:10AEF0009934812F0E94783489E49DE00E9499342E
:10AF000080913B010E94303E20913D0130913E01F5
:10AF100040913F01509140012CA33DA34EA35FA35C
:10AF20004090410150904201609043017090440173
:10AF30008090450190904601A0904701B090480153
:10AF4000C0904901D0904A01E0904B01F0904C0133
:10AF500080914D0190914E01A0914F01B09150010F
:10AF600088A799A7AAA7BBA72091510130915201A8
:10AF700040915301509154012CA73DA74EA75FA7C4
:10AF800081E49DE00E9499344CA15DA16EA17FA156
:10AF900084E39DE00E94C434B301A20184ED9FE2EA
:10AFA0000E94C434B501A40181ED9FE20E94C43423
:10AFB0008FE39DE00E94993487E39DE00E949934DD
:10AFC000B701A60184E39DE00E94C43448A559A5B9
:10AFD0006AA57BA584ED9FE20E94C4344CA55DA5C3
:10AFE0006EA57FA581ED9FE20E94C4348AE00E9495
:10AFF00078340C94634A0E94443E082F87FF02C0B5
:10B000000C94634A83E50E945F1A002E000C110B1A
:10B010007801EE0CFF1C882309F10E94701EF701D5
:10B02000EB5AFE4F91838083000F111F000F111FF9
:10B0300004591E4FBC01990F880B990B0E9497E78A
:10B040002AE037ED43E25CE30E94F6E7D8016D9316
:10B050007D938D939C9313970C94634A0E94403E7A
:10B0600085E40E94783480E3800F0E947834F701F1
:10B07000EB5AFE4F608171818AE59DE00E94AE3EF1
:10B0800085E20E9478348AE00E9478340C94634A06
:10B0900080E50E945F1A882311F40C94634A0E9491
:10B0A000701E8C01892B09F081C083E50E945F1A14
:10B0B000882389F00E94701E97FD07C0BC018AE1B9
:10B0C00093E10E947A320C94634A8AE193E10E94F0
:10B0D00059320C94634A0E94403E70E060E08BE776
:10B0E0009DE00E94AE3E80911C13E8E5CE2EE2E08A
:10B0F000DE2EC81AD10887FDD394CC0CDD1CCC0CF5
:10B10000DD1C0D2C000CEE08FF0880911B13A8E835
:10B110008A2E912C881A910887FD9394880C991C8B
:10B12000880C991C092C000CAA08BB0880911A13E2
:10B1300090E08F3FC9F1FC01EE0FFF1FE80FF91FF0
:10B14000EB50FD4E8181928163E0880F991F6A95D3
:10B15000E1F7B0E0A0E074E0B595A79597958795E5
:10B160007A95D1F702969C012F5F3F4F032E000C7A
:10B17000440B550B281939094A095B09A4EBB0E0C7
:10B180000E94FDEDA7019601281939094A095B09BA
:10B190000E94E1EDB90188E79DE00E94AE3E8AE0A1
:10B1A0000E9478340C94634A80E0DDCF0E943C3EDC
:10B1B000B80181E79DE00E94AE3E82E69DE00E94DC
:10B1C00099340C94634A83E50E945F1A81110C94B0
:10B1D000784F8091150487FD14C080911604837008
:10B1E00081F40E94403E40912513509126136091B6
:10B1F00027137091281383E89DE00E9403350C9477
:10B20000634A82E50E94E8198111EBCF0C94634AEE
:10B210008091130483FD09C080911404817829F47E
:10B2200081E00E946C3E0C94634A80E50E945F1AA4
:10B23000882351F00E947F1E60938D1270938E12AE
:10B2400080938F129093901289E40E945F1A882352
:10B2500081F00E947F1E2CEA35EC47E25EE30E94FB
:10B26000F6E76093911270939212809393129093E9
:10B27000941284E40E945F1A882311F40C94634AA8
:10B280000E947F1E20E030E543EC50E40E94F6E788
:10B2900060939512709396128093971290939812E0
:10B2A0000C94634A83E50E94E819182F882369F0FB
:10B2B0000E94701E9C01909371018093700191E037
:10B2C000232B09F090E09093741280E50E94E81916
:10B2D000882361F02091700130917101232B11F0CE
:10B2E0000E94501E809374120C94634A11110C94A6
:10B2F000634A0E94403E8DEB9DE00E94993480910C
:10B300007412882391F085EA9DE00E94993460913F
:10B310007001709171018CEA9DE00E94AE3E88EA56
:10B320009DE00E9499340C94634A81EA9DE0EDCF40
:10B330000E9406350C94634A83E50E94E819811146
:10B340000C94634A81E00E94F7880E9401870C9464
:10B35000634A83E50E94E819182F882309F426C15F
:10B360000E94501E8CA32091720130917301409174
:10B370007401509175012DAB3EAB4FAB58AF80912E
:10B38000760190917701A0917801B091790189AF10
:10B390009AAFABAFBCAF20917A0130917B01409165
:10B3A0007C0150917D0121962CAF3DAF4EAF5FAF38
:10B3B0002197112331F03CA1311103C080E00E949C
:10B3C000582A8091130490911404A0911504B0910F
:10B3D000160425E1B695A795979587952A95D1F7F7
:10B3E0009C01AD01217033274427552729AB3AAB87
:10B3F0004BAB5CAB20E030E0A9016091A004709100
:10B40000A1048091A2049091A3040E9491E7882353
:10B4100009F4D0C083E40E94E819882309F49AC093
:10B420000E947F1E25966CAF7DAF8EAF9FAF259794
:10B4300040EB54E059A748A78A0157E05CA7412C8C
:10B44000512CE8EC6E2EE2EC7E2E812C912CF8EC47
:10B45000AF2EF2E4BF2E312C212CF101EE0FFF1F95
:10B46000EE0FFF1FE00FF11FC080D180E280F3805C
:10B47000A7019601C501B4010E9491E7181614F4C2
:10B4800046015701A7019601C301B2010E944EF087
:10B4900087FF02C0260137018FEF281A380A97E08C
:10B4A00029163104D1F6ACA5A150ACA7045E1F4FFC
:10B4B000A111D1CFA3019201C501B4010E94AFEE49
:10B4C00020E030E040E05FE30E94F6E725962CADF7
:10B4D0003DAD4EAD5FAD25970E94AFEE4B015C01D7
:10B4E0002DEB37E346E855EB0E9491E787FD0AC054
:10B4F0002DEB37E346E855E3C501B4010E944EF059
:10B50000181644F580E00E94582A67E0F62E08A538
:10B5100019A557E0E52EF801619171918191919102
:10B520008F016F01F4E0CF1AD108A50194010E94A8
:10B53000AEEED6016D937D938D939C931397EA9411
:10B54000E110E9CFFA94E8A5F9A57C96F9A7E8A758
:10B55000F110DDCF89A99AA9ABA9BCA9892B8A2BA7
:10B560008B2B81F020E030E0A9016091A004709164
:10B57000A1048091A2049091A3040E9491E78111FB
:10B580000E94D13D8AE50E94E819882359F00E9463
:10B590007F1E69837A838B839C8360E0CE01019652
:10B5A0000E94E42A8CA10E94582A15C0B0919F04E1
:10B5B000BCA3D9CEFCA1F11108C029A93AA94BA975
:10B5C0005CA9232B242B252BE9F20E94403E8FE01F
:10B5D0009EE00E9499349CA1992351F080919F0490
:10B5E000811106C00E943C3E80EF9DE00E9499348C
:10B5F0000E94403E82EE9DE00E94993480919F041B
:10B600000E94303E0E94403E85ED9DE00E949934AC
:10B61000C0909B04D0909C04E0909D04F0909E0408
:10B6200020E030E0A901C701B6010E944EF01816D3
:10B630000CF042C042E0C701B6010E94BEB28DE0EC
:10B640000E9478348AE00E9478342091720130910F
:10B65000730140917401509175016DA97EA98FA964
:10B6600098AD0E9491E781110C94E54920917601F3
:10B6700030917701409178015091790169AD7AADAF
:10B680008BAD9CAD0E9491E781110C94E54920910E
:10B690007A0130917B0140917C0150917D0121968E
:10B6A0006CAD7DAD8EAD9FAD21970E9491E781116C
:10B6B0000C94E5490C94634A80ED9DE00E94993416
:10B6C000C4CFA3940C944F500E943C3E8EE39EE066
:10B6D0000E9499340C94634A0E94649E0C94634ABD
:10B6E0000E9434A80C94634A0E94FC870C94634A1D
:10B6F00061E083E50E945F1E91E089270E945672F7
:10B700000C94634A8091981482FF0CC087FD0AC094
:10B710000E944B2C9091981480FB97F99093981469
:10B720000C94634A84FD02C00C94634A0E944DD578
:10B730000C94634A40901D1350901E1360901F1389
:10B7400070902013209121133091221340912313E4
:10B75000509124132CA33DA34EA35FA3C0902513A7
:10B76000D0902613E0902713F090281388E50E94CC
:10B770005F1A182F882309F482C00E947F1E4B0194
:10B780005C0120E030E041E653EC0E944EF087FD82
:10B790000BC020E030E041E653E4C501B4010E9453
:10B7A00091E718160CF06DC061EE70E08FE99EE035
:10B7B0000E94AE3E61EE70E08AE99EE00E94AE3EDD
:10B7C00087E99EE00E94993410E089E50E945F1AA3
:10B7D000882341F10E947F1E4B015C0120E030E094
:10B7E00041E653EC0E944EF087FD0BC020E030E0B4
:10B7F00041E653E4C501B4010E9491E718160CF02C
:10B8000043C061EE70E084E89EE00E94AE3E61EECF
:10B8100070E08FE79EE00E94AE3E8CE79EE00E94C3
:10B82000993410E08AE50E945F1A882391F10E9402
:10B830007F1E6B017C0120E030E040EA51EC0E9469
:10B840004EF087FD0AC020E030E040EA51E4C70135
:10B85000B6010E9491E71816E4F46CEE7FEF8AE6D9
:10B860009EE00E94AE3E64E170E085E69EE00E94AC
:10B87000AE3E82E69EE00E9499340C94634A11E049
:10B88000A4CF24013501A1CF8CA29DA2AEA2BFA25C
:10B89000C9CF112311F40C94634A40921D135092A6
:10B8A0001E1360921F13709220138CA19DA1AEA154
:10B8B000BFA18093211390932213A0932313B093DD
:10B8C0002413C0922513D0922613E0922713F092EE
:10B8D00028130C94634A83E08093220710926C1023
:10B8E00060E083E50E945F1E81110C94634A0E9410
:10B8F00055C20C94634A0091190410911A040E94D5
:10B90000E0CC60931C0470931D0480931E049093FC
:10B910001F04002311F40C94634A0E94403E84E506
:10B920000E947834802F0E947B2880E20E94783425
:10B9300082ED9EE00E9499340C94634A11110C949C
:10B940000C4811E00C94FF4783E50E945F1A88239E
:10B9500011F40C94B1530E94251E8B010C94B15329
:10B960000E943C3E8EE19EE00E9499340C94634A12
:10B97000882339F30C941148B0E0A0E0E2ECFCE538
:10B980000C9479EE7C014DB65EB6609061077090C4
:10B9900062078DB69EB66AE070E0C7010E94CEE6EF
:10B9A0006C018C010E191F09892B21F4C7010E941B
:10B9B000E0E68C01C80101962DB73EB7281B390B74
:10B9C0000FB6F8943EBF0FBE2DBF8DB79EB7019640
:10B9D0005C01A801B7010E9401E7F501E00FF11F2A
:10B9E0001082C5010E949E2681E00E946247C11418
:10B9F000D10451F076019FEFE91AF90A0FB6F894D5
:10BA00009EBE0FBE8DBEC5CF0FB6F8949EBE0FBEB4
:10BA10008DBEC3010E949E260FB6F8945EBE0FBE77
:10BA20004DBEE0E10C9495EEA2E4B0E0EAE1FDE564
:10BA30000C9477EE0E94E0CC60931C0470931D047C
:10BA400080931E0490931F0480919F04811145C030
:10BA50008091130490911404A0911504B0911604E0
:10BA60003DE0B695A795979587953A95D1F780FFD4
:10BA700003C089E096E080DF87E00E947B8281112D
:10BA800033C080919F04888B80911304909114049B
:10BA9000A0911504B0911604AC01BD0126E1769584
:10BAA0006795579547952A95D1F740FFEDC020E05F
:10BAB00030E0A9016091A0047091A1048091A204DA
:10BAC0009091A3040E9491E7811113C00E943C3E13
:10BAD00087EF95E00E94993407C060E08FE40E94F0
:10BAE0005F1E882309F4B4CFCE5BDF4FE2E10C94F4
:10BAF00093EE8AE50E945F1A8823E9F00E947F1E78
:10BB00006B017C0120E030E040E251ECC701B6015E
:10BB10000E9491E787FD0AC020E030E040E251E456
:10BB2000C701B6010E944EF0181674F40E943C3E04
:10BB30008AEE95E0CFCFC0907A01D0907B01E09063
:10BB40007C01F0907D01DECF40E050E060EC7FE7CB
:10BB500088E50E94A71E2B013C0140E050E060EC0C
:10BB60007FE789E50E94A71E6BAB7CAB8DAB9EABDC
:10BB70006FEF89E40E94461E6FEF8AE40E94461E22
:10BB80008BA09CA0ADA0BEA020E030E040E05FE331
:10BB9000C501B4010E94F6E720919304309194040A
:10BBA00040919504509196040E94AEEEA30192013B
:10BBB0000E94AFEEA50194010E9429EF0E9491EF2F
:10BBC0002B013C01162F8FA098A4A9A4BAA420E0B1
:10BBD00030E040E05FE3C501B4010E94F6E7209148
:10BBE0009704309198044091990450919A040E94CE
:10BBF000AEEE2BA93CA94DA95EA90E94AFEEA5010E
:10BC000094010E9429EF0E9491EF062F042C000C52
:10BC1000550857FC31C027E0421651047CF5062E2A
:10BC2000000C770B77FD2CC0673071055CF5173081
:10BC300008F05ACF073008F057CF80E00E94582A0A
:10BC400037E01302F0011124E00FF11D07FDFA9512
:10BC5000EE0FFF1FEE0FFF1FE055FB4FC082D1829A
:10BC6000E282F38288890E94582A8889882309F40D
:10BC70003BCF0E94018738CF10E0D1CF16E0CFCF65
:10BC800000E0D5CF06E0D3CFE9E0B695A79597952C
:10BC90008795EA95D1F780FD0CC070E060E086E5FD
:10BCA0000E94731E9A838983059730F085EC95E096
:10BCB00011CF0E949A2A18CF60E084E40E945F1E90
:10BCC0008F8740E050E0BA018AE50E94A71E6BA76B
:10BCD0007CA78DA79EA740E050E669EF75E483E559
:10BCE0000E94A71E29E838E848E85CE30E94F6E7CE
:10BCF000609368017093690180936A0190936B016E
:10BD0000E0902913F0902A13D7014D905D906D902B
:10BD10007C9020E030E040EE50E4C301B2010E948C
:10BD2000AEEE4B015C0120E030E040E251E40E94C5
:10BD30004EF087FF06C0812C912C70E2A72E71E493
:10BD4000B72E20E030E041E653E4C301B2010E9487
:10BD5000AFEE6FAB78AF89AF9AAF20E030E047E548
:10BD600053E40E9491E7181644F480E090E0A7E5C0
:10BD7000B3E48FAB98AFA9AFBAAFD7011496CD900B
:10BD8000DD90ED90FC90179720E030E040E050E42B
:10BD9000C701B6010E94AEEE2B013C0120E030E06D
:10BDA00040E251E40E944EF087FF06C0412C512C26
:10BDB00060E2662E61E4762E20E030E041E653E456
:10BDC000C701B6010E94AFEE6BAB7CAB8DAB9EABF7
:10BDD00020E030E047E553E40E9491E7181644F470
:10BDE00080E090E0A7E5B3E48BAB9CABADABBEAB22
:10BDF00088E40E94E819882309F4F8C10E947F1E94
:10BE00000E9491EF23966CAF7DAF8EAF9FAF2397CB
:10BE100021966EAD7FAD219777FF02C06F5F7F4F98
:10BE20007595679571956195710960597F4F072EDA
:10BE3000000C880B990B0E9497E76B017C01CBAE3D
:10BE4000DCAEEDAEFEAEA30192010E944EF087FF84
:10BE500004C04BAE5CAE6DAE7EAEA5019401C701D1
:10BE6000B6010E944EF087FF02C075016401CB8AC3
:10BE7000DC8AED8AFE8A8BAD9CADADADBEAD8F8BFD
:10BE8000988FA98FBA8F2196AEADBFAD2197BD0116
:10BE9000BB0F880B990B0E9497E74B015C01A70130
:10BEA00096010E94AFEE6B017C012FA938AD49AD20
:10BEB0005AAD0E9491E7181624F4CFA8D8ACE9AC8B
:10BEC000FAACCB8EDC8EED8EFE8E2BAD3CAD4DAD47
:10BED0005EADC501B4010E94AFEE6B017C012BA9E0
:10BEE0003CA94DA95EA90E9491E7181624F4CBA89D
:10BEF000DCA8EDA8FEA8CF8ED8A2E9A2FAA2BE01C6
:10BF0000695E7F4FCE0143960E94DBC3882309F40C
:10BF100096C1BE01615E7F4FCE014B960E94DBC38E
:10BF2000E82E882309F48BC12F89388D498D5A8DCD
:10BF30006F8D78A189A19AA10E94AEEE2BEA3AEA10
:10BF40004AE25EE30E94F6E74B015C012B893C89E3
:10BF50004D895E896B8D7C8D8D8D9E8D0E94AEEEA0
:10BF60002BEA3AEA4AE25EE30E94F6E76BA37CA37F
:10BF70008DA39EA38FA298A6A9A6BAA689819A810D
:10BF80001816190674F483E995E00E9499348F8598
:10BF9000882321F089E895E00E9499348AE00E9484
:10BFA00078340E94A0730E94E68580E00E94582A9F
:10BFB00080E090E0A0E2B1E48FA798ABA9ABBAAB68
:10BFC000CE018F960E944BC32091A0043091A10412
:10BFD0004091A2045091A3046BA17CA18DA19EA1CC
:10BFE0000E9491E7811130C02091A4043091A504F2
:10BFF0004091A6045091A7046FA178A589A59AA5A0
:10C000000E9491E7811120C0209193043091940403
:10C0100040919504509196046B897C898D899E8905
:10C020000E9491E7811110C02091970430919804EB
:10C030004091990450919A046F89788D898D9A8DD9
:10C040000E9491E78823A9F00E949A2A88E0FE01C5
:10C05000B396A0EAB4E001900D928A95E1F788E0EA
:10C06000FE017396A3E9B4E001900D928A95E1F781
:10C07000188A60E085E40E945F1ECC24C39481117D
:10C0800002C043E0C42E1B861C861D861E861A8AAB
:10C09000DE2C97E0792E29E5A22E25E0B22E37E698
:10C0A000832E35E0932E8A8987300CF0D4C0DD20B2
:10C0B00009F4C8C066246394B7E0BBAB90E021E00C
:10C0C000D226879DF02C1124F394998B19896A89C3
:10C0D000FBA91F1709F4BCC0062E000C770B880BB8
:10C0E000990B0E9497E72FA138A549A55AA50E9450
:10C0F000F6E72F89388D498D5A8D0E94AFEE1B01CE
:10C100002C01612F110F770B880B990B0E9497E779
:10C110002BA13CA14DA15EA10E94F6E72B893C8991
:10C120004D895E890E94AFEE6B837C838D839E83F5
:10C130002F82388649865A8689819A81892B89F08F
:10C1400085E795E00E9499348F2D0E947B2861E35A
:10C1500070E083E795E00E94AE3E80E795E00E94A4
:10C1600099341F9221E32F931F92FF92BF92AF92B7
:10C170009F928F921F920E940E9E29814C2DBE018C
:10C18000695F7F4FCE0103960E9411C59B01AC01F0
:10C190002B873C874D875E8709898A89672D06032F
:10C1A00080011124080F111D87FD1A95000F111F22
:10C1B000000F111F00551B4F6BA57CA58DA59EA5DB
:10C1C0000E94AFEED8016D937D938D939C9313974E
:10C1D000188A81E00E945140F3948989860D898BE9
:10C1E0000FB6F894DEBF0FBECDBF70CFB301A20172
:10C1F00086E40E94A71E6B017C01B501A4018CE4BA
:10C200000E94A71E6B8B7C8B8D8B9E8BCF8AD88ECA
:10C21000E98EFA8E4BA95CA96DA97EA982E40E94E1
:10C22000A71E6B017C014FA958AD69AD7AAD82E5BF
:10C230000E94A71E6B8F7C8F8D8F9E8F5CCE89EAAC
:10C2400095E048CC66246A94EFEFEBAB96E037CFED
:10C250006F5F6A8B28CF0E9499C30E9400288823B1
:10C2600059F088890E94582A80E090E0A0ECBFE74E
:10C270008B879C87AD87BE870E94D13D0E94B12BE2
:10C280008F85811122C08AE791E00E9403284B012B
:10C290005C0182E791E00E948128A50194010E943F
:10C2A000F6E79B01AC0160917A0170917B0180916E
:10C2B0007C0190917D010E94AEEE60937A017093B3
:10C2C0007B0180937C0190937D018F858111E888AB
:10C2D000E0929F040E94CD8580919F04882309F4F9
:10C2E000C8CC0E94B386C5CCCF93DF93C091750EA6
:10C2F00081E6C89FE0011124C958D14F8091400DBB
:10C3000080FF05C00E94403ECE010E948A34CE01CB
:10C310000E949E2680E00E946247DF91CF9108959F
:10C32000A0E1B0E0E6E9F1E60C9485EE8C01DC01D9
:10C33000ED91FC910280F381E02DBE016F5F7F4F94
:10C340000995882309F45DC08981807C91F56F810E
:10C35000637070E0762F6627770F770F8885B4E0DB
:10C360008B9FC0011124682B792B89858295869536
:10C3700086958370682B6F5F7F4F90E080E02A8501
:10C380002370220F3B8537FB332730F9232B3E8167
:10C390003F70230F3327331F2750310904C0660F26
:10C3A000771F881F991F2A95D2F76096E4E00C94B6
:10C3B000A1EE803419F568856695669570E090E089
:10C3C00080E0CB01772766272A85622B098510E05C
:10C3D000102F0027012E000C220B330B602B712B2A
:10C3E000822B932B6F5F7F4F8F4F9F4F4AE0660FDB
:10C3F000771F881F991F4A95D1F7D7CF8BE0F80197
:10C40000848360E070E0CB01D0CF0895FC0182818D
:10C410000895FC0190E1A7E5B6E001900D929A9590
:10C42000E1F70895EF92FF920F931F93E092760544
:10C43000F09277050093780510937905B62F172FA2
:10C44000022FF32E242F582FB0937A0510937B05DB
:10C4500050937C056FEFFF27B01B1F09520B30F480
:10C4600050951095B195160B560B66276093A00258
:10C47000A6E0BA9F00929402712DEE271A9F700DCC
:10C48000E11D5A9FE00D70939502E0939602AFE094
:10C49000BA9F00929802712DEE271A9F700DE11D30
:10C4A0005A9FE00D70939902E0939A02AAE0BA9F16
:10C4B00000929C02712DEE271A9F700DE11D5A9F6C
:10C4C000E00D70939D02E0939E021F910F91FF90EB
:10C4D000EF900895A5E0B0E0E0E7F2E60C947EEE80
:10C4E0006F3671058105910578F4FB01EE0FFF1F92
:10C4F000EE0FFF1FED5AF14E659175918591949164
:10C500002596EBE00C949AEEF62EE72E282FE3E525
:10C51000FDE10027BB275F2D8E2D922F992341F43B
:10C52000982F852FB85F992319F4982F8827B85F23
:10C53000903138F482959295582F5F70807F952BBB
:10C54000BC5F903428F4880F991F880F991FBE5F35
:10C55000903818F4880F991FB395880F991FE90F29
:10C56000F01F549181E09927B85079F1C0F0B0FFE5
:10C5700002C0550F881FB1FF04C0550F881F550F0B
:10C58000881FB2FF06C082955295152F1F70507FED
:10C59000812BB3FF1AC0982F852F552716C0B19550
:10C5A000B0FF02C085955795B1FF04C0859557959A
:10C5B00085955795B2FF05C08295507F5295582BAF
:10C5C0008F70B3FF02C0582F8827BB247727AA2774
:10C5D000B2E0F59EB0187109A00BB00BE59E701982
:10C5E000A109B00B259FA019B109F89E7019A109E6
:10C5F000B00BE89EA019B109289FB019F99EA019A7
:10C60000B109E99EB0195B9DA12C992444276627A6
:10C6100033278B9DA00C911C401F601F301F9B9DDA
:10C62000900C411D601F301F579FA00C911C401F94
:10C63000601F301F879F900C411D601F301F979F08
:10C64000400D611D301F5A9F900C411D601F301F0F
:10C650008A9F400D611D301F9A9F600D311D5B9FA9
:10C66000400D611D301F8B9F600D311D9B9F300D54
:10C67000B1E0AA277727BB24F49EB0187109A00B5C
:10C68000B00BE49E7019A109B00B249FA019B10949
:10C69000F69E7019A109B00BE69EA019B109269F5C
:10C6A000B019F39EA019B109E39EB019BF187E0915
:10C6B000A20B20F0B1E04B0F601F301F1124762F2A
:10C6C000642F90E0832F1CCFFC017081472F50E036
:10C6D000062E02C0559547950A94E2F740FF14C014
:10C6E0004091EF0550E0062E02C0559547950A94FB
:10C6F000E2F740FF09C021E030E001C0220F6A9557
:10C70000EAF720952723208308958F929F92AF9276
:10C71000BF92CF92DF92EF92FF92FC01C080D18056
:10C72000E280F38020E030E048EC52E4C701B6013B
:10C730000E94F6E74B015C0120E030E0A901C7014F
:10C74000B6010E9491E720E030E040EA50E487FF24
:10C7500004C020E030E040EA50ECC501B4010E9482
:10C76000AFEE2DEC3CEC4CEC5DE30E94F6E70E9452
:10C7700091EF9B018BE237FF05C022273327261B51
:10C78000370B8DE280937C04C90168EE73E00E9450
:10C7900049EECB01EAE0F0E0BF010E9449EE805D86
:10C7A00080937D04C90164E670E00E9449EECB01EC
:10C7B000BF010E9449EE805D80937E04C901BF01E4
:10C7C0000E9449EE9C01CB01BF010E9449EE805DB1
:10C7D00080937F048EE280938004205D2093810407
:10C7E0008CE794E0FF90EF90DF90CF90BF90AF90F8
:10C7F0009F908F9008954F925F926F927F928F9249
:10C800009F92AF92BF92CF92DF92EF92FF92FC0184
:10C81000C080D180E280F38020E030E04AE754E439
:10C82000C701B6010E94F6E74B015C0120E030E051
:10C8300040E251ECC701B6010E9491E7181654F48A
:10C8400020E030E048EC52E4C701B6010E944EF00F
:10C8500087FD8AC020E030E0A901C701B6010E942F
:10C8600091E787FF72C060E070E080EA90ECA5017C
:10C8700094010E94AFEE2DEC3CEC4CEC5DE30E9489
:10C88000F6E70E9491EF6B017C01F7FC63C020E1A9
:10C8900037E240E050E00E94E1EDCA01B9012AE030
:10C8A00030E040E050E00E94E1ED605D60937C0488
:10C8B000C701B60128EE33E040E050E00E94E1ED10
:10C8C0009AE0892E912CA12CB12CCA01B901A501A5
:10C8D00094010E94E1ED605D60937D04C701B601A3
:10C8E00024E630E040E050E00E94E1EDCA01B901E9
:10C8F000A50194010E94E1ED605D60937E048EE2EB
:10C9000080937F04C701B601A50194010E94E1ED67
:10C910006B01CA01B901A50194010E94E1ED605DBE
:10C9200060938004F0E3CF0EC09281048CE794E022
:10C93000FF90EF90DF90CF90BF90AF909F908F903F
:10C940007F906F905F904F90089560E070E080EA74
:10C9500090E48DCFF094E094D094C094C11CD11C8D
:10C96000E11CF11C6DE2A2CF20E030E0A901C7017B
:10C97000B6010E9491E787FF6BC060E070E080EA3B
:10C9800090ECA50194010E94AFEE2DEC3CEC4CEC38
:10C990005DE30E94F6E70E9491EF4B015C0120E00D
:10C9A00030E0A901C701B6010E9491E787FD0BC0E5
:10C9B00020E030E040E251E4C701B6010E944EF0B1
:10C9C00060E287FD13C0B7FC48C0C501B40128EE82
:10C9D00033E040E050E00E94E1EDCA01B9012AE0F5
:10C9E00030E040E050E00E94E1ED605D60937D0446
:10C9F000C501B40124E630E040E050E00E94E1EDE2
:10CA00008AE0482E512C612C712CCA01B901A30176
:10CA100092010E94E1ED605D60937E048EE280935E
:10CA20007F04C501B401A30192010E94E1ED6B01F5
:10CA3000CA01B901A30192010E94E1ED605D60931A
:10CA4000800480E3C80EC09281048DE794E070CF2B
:10CA500060E070E080EA90E494CFB094A094909469
:10CA60008094811C911CA11CB11C6DE2BFCF282FAA
:10CA700081E3243609F080E280937E0490E22A303C
:10CA800040F03AE0822F632F0E941CEE0E941CEEC1
:10CA9000905D90937F04822F6AE00E941CEE905D6F
:10CAA0009093800485E2809381048EE794E008955A
:10CAB0006091550170915601072E000C880B990B5F
:10CAC0000E9497E72AE037ED43E25CE30E94F6E735
:10CAD00060936C0170936D0180936E0190936F0170
:10CAE0000895CF93DF93EC01CB01BA010E9497E741
:10CAF00023E333E343E250E40E94F6E720E030E032
:10CB000040E05FE30E94AFEE0E9496EF6883DF9102
:10CB1000CF9108950E9497E723E333E343E250E483
:10CB20000E94F6E720E030E040E05FE30E94AFEED5
:10CB30000E9496EF24E6629FC001112481589F4F06
:10CB40006FEF70E00E9449EE862F91CF80914C07E5
:10CB5000811104C08091230780937F0708958091FD
:10CB60008E148823C1F0815080938E14E1EDF2E1A0
:10CB7000882351F08150990B2BE1289FF001299FC8
:10CB8000F00D1124E058FC4E8BE1A6EBB2E10190D0
:10CB90000D928A95E1F720918E14211105C08091A4
:10CBA000981480648093981481E090E0A0E0B0E055
:10CBB000211103C080E090E0DC0180934207909354
:10CBC0004307A0934407B093450710923D0781E0C7
:10CBD00080933F0783E0809367010895CF93DF93AD
:10CBE000EC01CB01BA010E9497E7688379838A83BD
:10CBF0009B83DF91CF910895CF93DF93EC01CB011D
:10CC0000BA010E9497E72DEC3CEC4CEC5DE30E94EE
:10CC1000F6E7688379838A839B83DF91CF910895B8
:10CC2000CF93DF93EC01CB01BA010E9497E72AE092
:10CC300037ED43E25CE30E94F6E7688379838A83F9
:10CC40009B83DF91CF910895CF92DF92EF92FF9275
:10CC5000CF93DF9300D000D0CDB7DEB70E9497E727
:10CC60002AE037ED43E25CE30E94F6E76B017C01CA
:10CC700020E030E0A9010E9491E72DEB37E346E088
:10CC800055E387FF04C02DEB37E346E055EBC701C2
:10CC9000B6010E94AFEE69837A838B839C83CE01B9
:10CCA0000196A9DD0F900F900F900F90DF91CF911B
:10CCB000FF90EF90DF90CF900895CF93DF93EC013A
:10CCC000CB01BA010E9497E70E9491EF79836883B4
:10CCD000DF91CF9108958F929F92AF92BF92CF92A2
:10CCE000DF92EF92FF92FC01C080D180E280F3805E
:10CCF00020E030E0A901C701B6010E9491E787FD5D
:10CD000099C06DEB77E386E095E3A70196010E9459
:10CD1000AFEE9F7720E030E048EC52E40E94F6E767
:10CD200020E030E040EA50E40E94AFEE2DEC3CEC15
:10CD30004CEC5DE30E94F6E70E9491EF6B017C01F1
:10CD400080E280937B0460E2F0E1CF16F7E2DF0639
:10CD5000E104F1048CF0C701B60120E137E240E0C4
:10CD600050E00E94E1EDCA01B9012AE030E040E064
:10CD700050E00E94E1ED605D60937C0460E288EE2B
:10CD8000C81683E0D806E104F1048CF0C701B601AF
:10CD900028EE33E040E050E00E94E1EDCA01B90125
:10CDA0002AE030E040E050E00E94E1ED605D6093F9
:10CDB0007D0460E2E4E6CE16D104E104F1048CF0D7
:10CDC000C701B60124E630E040E050E00E94E1ED0A
:10CDD000CA01B9012AE030E040E050E00E94E1EDF4
:10CDE000605D60937E048AE0882E912CA12CB12C8A
:10CDF000C701B601A50194010E94E1ED6B01CA01D2
:10CE0000B901A50194010E94E1ED605D60937F048A
:10CE10008EE280938004F0E3CF0EC09281048BE712
:10CE200094E0FF90EF90DF90CF90BF90AF909F90F5
:10CE30008F9008956DEB77E386E095EB66CFA4E0E5
:10CE4000B0E0E5E2F7E60C9487EE0E9497E72DEC60
:10CE50003CEC4CEC5DE30E94F6E769837A838B83BC
:10CE60009C83CE01019637DF2496E2E00C94A3EE7A
:10CE7000CF93DF93EC018D810E94404060E08B8175
:10CE80000E94FBCBDF91CF910895CF92DF92EF927A
:10CE9000FF920F931F93CF938C01C62F69017A01E4
:10CEA000E7DF0E94CACD8C2F80640E9434408F2D12
:10CEB0000E9434408E2D0E9434408D2D0E943440BB
:10CEC0008C2D0E94344087E8C11101C085E90E9481
:10CED0003440CC3011F40E943940C0E00E94394007
:10CEE000F801868387FF04C0CF3F11F0CF5FF6CFF4
:10CEF000CF911F910F91FF90EF90DF90CF90089509
:10CF000061E0FC0183810E94FBCB8FEF0C943440E5
:10CF10000F931F93CF938C01ABDF0E94CACDC82F14
:10CF2000882369F08DEF0E9434400E94CACDC82F3B
:10CF3000C801E6DF8C2FCF911F910F91089582E1F8
:10CF4000F8018483F5CFB0E0A0E0E9EAF7E60C94BD
:10CF50007DEEEC016A017B014801590120E030E0DF
:10CF6000A90167E392DFA501980167E1CE018DDF9A
:10CF700081111DC08F81833039F089E0CC0CDD1C1C
:10CF8000EE1CFF1C8A95D1F7A701960169E1CE013D
:10CF90007CDF11E0882319F010E087E08C83CE015C
:10CFA000AFDF812FCDB7DEB7ECE00C9499EE89E0CE
:10CFB0008C8310E0F4CFCF93DF93EC016EBDFA01C8
:10CFC000CA019E5F0DB407FEFDCF20812EBD0DB4BA
:10CFD00007FEFDCF21812EBD3296E817F90791F7A4
:10CFE0000DB407FEFDCF8FEF0E9434408FEF0E94FB
:10CFF00034400E9439408E838F71853041F083E147
:10D000008C83CE017DDF80E0DF91CF91089581E0B8
:10D01000FBCF0F931F93CF93DF93EC018B0128DF9E
:10D020000E94CACD81110BC085E18C8310E0CE0136
:10D0300067DF812FDF91CF911F910F910895A80194
:10D040006CEFCE01B8DF182F882371F3F0CF0F9368
:10D050001F93CF93DF93EC0189018F81833039F0E7
:10D0600089E0440F551F661F771F8A95D1F79A01F3
:10D07000AB0168E1CE0109DF811127C0A8016EEF85
:10D08000CE0199DF182F8823A9F00E94CACD182F4E
:10D090008823C1F020E030E0A9016DE0CE01F5DE8B
:10D0A000882321F086E18C8310E004C00E9439407F
:10D0B0008111F8CFCE0124DF812FDF91CF911F9115
:10D0C0000F91089587E18C83F5CF86E0ECCF1F9315
:10D0D000CF93DF93EC01CCDE20E030E0A9016CE0DF
:10D0E000CE01D3DE11E0882319F010E083E08C83B9
:10D0F000CE0106DF812FDF91CF911F9108951F93FD
:10D10000CF93DF93EC018F81833039F089E0440FB6
:10D11000551F661F771F8A95D1F79A01AB0162E10F
:10D12000CE01B3DE11E0882319F010E085E08C8396
:10D13000CE01E6DE812FDF91CF911F9108958F926E
:10D140009F92AF92BF92EF92FF920F931F93CF9354
:10D15000DF938C01EB017A010E94E0CC4B015C0172
:10D160002CE2820E21E0921EA11CB11C0E943940CB
:10D17000F80186838F3F69F40E94E0CC6819790931
:10D180008A099B0997FDF2CF81E1F8018483C0E011
:10D1900021C08E3F69F5F1E0EF1AF1088FEF8EBDE7
:10D1A000FE012FEF0DB407FEFDCF8EB581932EBD8E
:10D1B000CF018C1B9D0B8E159F05A0F30DB407FEB0
:10D1C000FDCF8EB5CE0DDF1D88830E9439400E94B1
:10D1D0003940C1E0C80194DE8C2FDF91CF911F91BF
:10D1E0000F91FF90EF90BF90AF909F908F90089518
:10D1F0008FE0CBCF0F931F93CF93DF93EC018B0185
:10D2000037DE40E052E0B801CE0199DFDF91CF91E7
:10D210001F910F9108950F931F93CF93DF93EC010C
:10D2200089018F81833039F089E0440F551F661FD3
:10D23000771F8A95D1F79A01AB0161E1CE0125DE16
:10D24000882351F084E08C83CE015ADE80E0DF91A8
:10D25000CF911F910F91089540E052E0B801CE01A7
:10D260006EDFF5CFB0E0A0E0E8E3F9E60C947DEEE8
:10D27000EC01162F1F821C824B830E94E0CC6B01B5
:10D280007C0120EDC20E27E0D21EE11CF11CA89506
:10D2900061E08B810E94FBCB8B810E949FB2249A1C
:10D2A0002C9A279A2698259A81E00E94404085E092
:10D2B0008D830E9440400AE08FEF0E94344001506D
:10D2C000D9F7A89520E030E0A90160E0CE01DDDDCE
:10D2D0008E83813079F00E94E0CC6C197D098E0933
:10D2E0009F0997FDEFCF81E08C83CE0109DE1A8282
:10D2F00080E065C0A8952AEA31E040E050E068E0AF
:10D30000CE01C3DD853031F581E08F83A8958F8113
:10D31000812C912C5401823029F4812C912CA12C48
:10D3200080E4B82E20E030E0A90167E3CE01ADDD56
:10D33000A501940169E2CE01A8DD8E838823F1F076
:10D340000E94E0CC6C197D098E099F0997FDEACFF8
:10D350008AE0CACF04E00E9439408E830150D9F799
:10D360008A3A11F482E0D1CF0E94E0CC6C197D0999
:10D370008E099F0997FDBFCF82E0B6CF8F818230A3
:10D38000B9F420E030E0A9016AE3CE017EDD882314
:10D3900011F088E0A9CF0E943940807C803C11F4D4
:10D3A00083E08F830E9439400E9439400E943940B7
:10D3B000CE01A6DD81E08A83173030F41D83CDB71E
:10D3C000DEB7ECE00C9499EE88E18C8391CF0F935B
:10D3D0001F93CF93DF93EC018B0120E030E0A90194
:10D3E00069E053DD882351F080E18C83CE0188DD34
:10D3F00080E0DF91CF911F910F91089540E150E0BF
:10D40000B801CE019CDEF5CFCF93C82FCB010E948F
:10D41000993487E89CE10E94993488E79CE1CC2309
:10D4200011F08DE79CE10E9499348AE00E947834E3
:10D43000CF9108950C94ECCC4091740521E04227E3
:10D440006CE070E00C9473B24091740521E04227C7
:10D4500064E070E00C9473B24091740521E04227BF
:10D4600061E070E00C9473B24091740521E04227B2
:10D4700061E070E00C9473B24091740521E04227A2
:10D4800068E070E00C9473B24091740521E042278B
:10D490006CE070E00C9473B241E061E070E00C94D9
:10D4A00073B24091740521E042270C9473B26CE092
:10D4B00070E00C948ACC61E070E00C948ACC61E05E
:10D4C00070E00C948ACC6CE070E00C948ACC64E040
:10D4D00070E00C948ACC90919F0481E089270C9491
:10D4E000582A61E083E297E00C94E42A20E030E0DF
:10D4F000A901BC0182E791E00C94ADC280E090E00C
:10D50000A0E8B0E480937A0190937B01A0937C0122
:10D51000B0937D0183E492E0E9DF80E090E0A0EF4A
:10D52000B1E48093720190937301A0937401B0935E
:10D5300075018093760190937701A0937801B09361
:10D540007901E091CC05EE0FFF0BED5DFD4F808181
:10D5500091818330910539F184309105C9F10297A9
:10D5600061F480E090E0A3E4B3E4809372019093CF
:10D570007301A0937401B09375018BE292E0B6DF62
:10D5800010927A0110927B0110927C0110927D0121
:10D5900083E492E0ABDF8091CC058F5F8430ECF4C4
:10D5A0008093CC05089580E090E0A3E4B3E48093F9
:10D5B000720190937301A0937401B09375018093ED
:10D5C000760190937701A0937801B0937901D5CF3C
:10D5D00080E090E0A3E4B3E4F2CF1092CC0508958C
:10D5E000A4E0B0E0E6EFFAE60C9487EE84EF91E079
:10D5F000A0E0B0E089839A83AB83BC83BE016F5FF8
:10D600007F4F88E70E943F332496E2E00C94A3EE1C
:10D61000B0E0A0E0EEE0FBE60C9487EE20E24F8164
:10D6200058856E818D810E94AEC7E2E00C94A3EE16
:10D6300080912307909124070C9421CD6AEF74E91F
:10D6400082E00C94BCC96EEF74E981E00C94BCC913
:10D6500062E075E980E00C94BCC966E075E983E09E
:10D660000C94BCC910923D070C9453D34FE350E087
:10D670006CEB7AE181EE96E00C9463F180912E13CD
:10D6800090912F13891B8F7011F40C94382C81E02A
:10D69000089580916701882341F06091C4057091DD
:10D6A000C50541E081E00C944EC708950F931F9388
:10D6B000CF93DF93FC012381222331F080E0DF91BF
:10D6C000CF911F910F9108958B01EC01FB01878988
:10D6D000803139F582E08B831D8A1E8A1F8A188E5D
:10D6E000808D918DB0E0A0E025E0880F991FAA1FE2
:10D6F000BB1F2A95D1F7898B9A8BAB8BBC8B1A8F6A
:10D70000098F81E08983188619861A861B861C82F8
:10D710001D821E821F82188A1C861D861E861F86F9
:10D72000CECF803259F683E08B83428D538D648D4A
:10D73000758D4D8B5E8B6F8B788F9E012F5E3F4F6B
:10D74000C8010E94B1D48111DACFB8CFCF93DF9353
:10D75000EC010E941AD51B82DF91CF910895CF93DF
:10D76000DF93EC01462F41706C857D858E859F850A
:10D770000E94C3D1882351F0888920E2829FC00192
:10D78000112483599F4EDF91CF91089590E080E05E
:10D79000FACFCF93DF93EB01FC012381211104C069
:10D7A00080E0DF91CF9108952250223028F48FE25B
:10D7B0008883198281E0F5CF60E0D1DF009781F3A3
:10D7C000DC0160E080E09EE22D91203299F088300B
:10D7D00031F49E01260F311DF90190836F5F9E0188
:10D7E000260F311DAD0141505109FA014081F90167
:10D7F00040836F5F8F5F8B3039F7FE01E60FF11DBD
:10D800001082D8CFACE0B0E0E8E0FCE60C9478EE13
:10D810005C01DC0159968D909C90F4018185928584
:10D82000A385B4859C01AD012F5F3F4F4F4F5F4FE4
:10D8300029873A874B875C87D50114964D905D9078
:10D840006D907C901797411451046104710409F4A0
:10D8500059C0BFEF4B1A5B0A6B0A7B0A312C73016C
:10D8600062011D821E821F821886F40181859285C5
:10D87000A385B4852D813E814F81588528173907AE
:10D880004A075B0708F056C089859A85AB85BC8539
:10D890008C159D05AE05BF0550F482E0C82ED12C35
:10D8A000E12CF12C92E0492E512C612C712C9E011F
:10D8B0002F5F3F4FB701A601C4010E9435D48823D2
:10D8C000C9F189819A81AB81BC81892B8A2B8B2BF1
:10D8D00001F1260137019FEF491A590A690A790AAD
:10D8E0002D813E814F8158852F5F3F4F4F4F5F4FB6
:10D8F0002D833E834F8358873FEFC31AD30AE30A31
:10D90000F30AB3CF40805180628073803324339414
:10D91000A6CFC414D504E604F70411F70FEF1FEFE8
:10D920002FEF3FE0B701A601C4010E94BBD3782EC0
:10D93000811106C0712C872D2C96E1E10C9494EE98
:10D94000F501448155816681778141155105610555
:10D95000710539F097018601C4010E94BBD3882369
:10D9600049F3D5011496CD92DD92ED92FC92179772
:10D97000332051F0D701C6010196A11DB11DF4015C
:10D9800080839183A283B383F50185899689A789D2
:10D99000B08D892B8A2B8B2B71F6C58AD68AE78AA4
:10D9A000F08E818180688183C6CF40E050E0BA016B
:10D9B0000C9463D54F925F926F927F92AF92BF9219
:10D9C000CF92DF92EF92FF920F931F93CF93DF934B
:10D9D0001F92CDB7DEB78C017B015A01C22EDB014D
:10D9E00059968D919C91F801928F818FCB01DDDF4B
:10D9F000712CF70180859185A285B3854189528973
:10DA00006389748984179507A607B70708F052C081
:10DA100055E0B695A795979587955A95D1F7F82F24
:10DA2000FF70DF2ED70113968C91823010F480E0C6
:10DA3000DAC041E050E0BE016F5F7F4FC7010E9436
:10DA40005ED60197A1F7F70180859185A285B38500
:10DA50004F96A11DB11D80879187A287B387F0E201
:10DA6000DF9EB001112463597F4E61157105F9F2F3
:10DA7000DB018C91882341F0853E09F04BC0772073
:10DA800029F077247394B5CF71100EC080916D1278
:10DA900090916E12A0916F12B0917012F80184876C
:10DAA0009587A687B787D08ADB018C918111E9CF52
:10DAB000772473948C2D8274823409F0B8CF772048
:10DAC00009F4A1C0F801D08861E0C80148DE0097E0
:10DAD00009F4ADCF20E2DC011D922A95E9F72BE095
:10DAE000F501DC0101900D922A95E1F721E238E27F
:10DAF000FC01318B208B40E058E057874687338B01
:10DB0000228B318F208F578B468B0E947AD18111C7
:10DB100009C08DCF4BE050E0C5010E9413F1892B65
:10DB200009F067CFF0E2DF9ED00111249D01235957
:10DB30003F4EF9018385817121F08C2D827109F0AE
:10DB400000C1F801818D928D40916D1250916E123D
:10DB500060916F127091701244875587668777873E
:10DB6000D08AFD01E359FF4E44885588712C612C01
:10DB7000320155244424D80155964D925D926D9200
:10DB80007C925897428D538D70E060E0442955296E
:10DB90006629772955964D935D936D937C9358979D
:10DBA000D9011B962C91287109F0BDC0848D958DEB
:10DBB000A68DB78DF801818B928BA38BB48B81E0FE
:10DBC00083838C2D8F70F8018183148215821682D5
:10DBD0001782108611861286138681E0C4FE03C068
:10DBE000C8010E94E8D50F90DF91CF911F910F914E
:10DBF000FF90EF90DF90CF90BF90AF907F906F90AD
:10DC00005F904F900895D70113968C9113978230AF
:10DC100009F40DCF51968D919D910D90BC91A02D41
:10DC2000803E9F4FAF41B10508F001CFC701EADD4B
:10DC3000882309F4FCCE0E947AD1882309F4F7CE18
:10DC4000D7015996ED91FC915A9714964D905D909D
:10DC50006D907C901797B2E04B1A510861087108DB
:10DC6000858504C0440C551C661C771C8A95D2F728
:10DC700086859785A089B189480E591E6A1E7B1E2C
:10DC800081E08093711240926D1250926E126092F8
:10DC90006F1270927012EDE6F0E180E092E0DF0129
:10DCA0009C011D9221503040E1F7DD24D394D7012F
:10DCB0005996ED91FC918481D816C0F4809172122E
:10DCC00090917312DC01ED91FC910288F389E02DB3
:10DCD0002DE630E1B301A2014D0D511D611D711DF5
:10DCE0000995882309F4A3CED394E1CF258580E05C
:10DCF00092E0A0E0B0E004C0880F991FAA1FBB1FEC
:10DD00002A95D2F7F7014189528963897489840F72
:10DD1000951FA61FB71F818B928BA38BB48B8DE6AB
:10DD200090E1D12CD7CE203161F498012F5E3F4F86
:10DD30000E94B1D4882329F084E0D80113968C93F3
:10DD400040CFD80113961C9272CEFC012381211181
:10DD5000FDCC0895A1E4B0E0E0EBFEE60C9477EE94
:10DD60004C015B017A01222E19821C821C8E1F8EAF
:10DD70006115710569F410E0CE014C96E6DFCE0125
:10DD80000196E3DF812FCF5BDF4FE2E10C9493EE4E
:10DD9000FC0183818111EFCFFA0180818F3251F133
:10DDA0008B01CE0101966C012C0180E2382E3601E8
:10DDB00022963FAE229721963FAE21973FAE3EAED0
:10DDC0003DAE3CAE3BAE3AAE39AE38AE3FAA97015F
:10DDD00090E047E0D9018D91882309F446C08F3245
:10DDE00009F443C08E3201F54A3029F298E04AE046
:10DDF0009D01F0CFFB0183818250823098F0618DCC
:10DE0000728DCE014C9652DC882309F4B4CF8E017A
:10DE1000045E1F4FC7017C010196F70120812F325C
:10DE2000D1F3BFCF8B01F6CFEEEBFAE224912223A0
:10DE300021F031968213FACF9ECF491708F49BCF79
:10DE4000813208F498CF8F3709F495CF3FE9380F26
:10DE50003A3108F420EEE7E3F0E0EC0FFD1FE90FA4
:10DE6000F11D820F80839F5FC3CF8FA9803209F499
:10DE700082CF7901F90180812F5F3F4F8F32C9F343
:10DE80008823C1F021E0AE01495C5F4FB801C601B3
:10DE900091DD882309F46FCF0A151B0511F0C80125
:10DEA00055DCCE014C964C145D0409F0C30186018B
:10DEB0006C017ECF222DAE01495C5F4FB801C401D9
:10DEC00079DD182F59CF8F929F92AF92BF92CF9248
:10DED000DF92EF92FF920F931F93CF93C82F02E828
:10DEE00012E1F80160857185072E000C880B990BF3
:10DEF0000E9497E76B017C01F80184809580A680E1
:10DF0000B78080E20E94783484E50E9478348AE306
:10DF10000E94783442E0C501B4010E94BEB287EB92
:10DF20009AE20E94993442E0C701B6010E94BEB253
:10DF300062E070E080E090E00E9457CC87E1C80288
:10DF4000F0011124EE57FD4E628570E08AEB9AE2F3
:10DF50000E94AE3ECF911F910F91FF90EF90DF9006
:10DF6000CF90BF90AF909F908F9008950F930FB771
:10DF70000F9300916E000B7F00936E0078940F93C7
:10DF80000BB70F930CB70F921F922F933F934F93A2
:10DF90005F936F937F938F939F93AF93BF93EF9311
:10DFA000FF9311240E94F2A3FF91EF91BF91AF91D3
:10DFB0009F918F917F916F915F914F913F912F91A1
:10DFC0001F900F900CBF0F910BBF0F910460F8943E
:10DFD00000936E000F910FBF0F911895CF93DF93B1
:10DFE00010927E05C2E8D2E1198618860E94ECCC18
:10DFF0001A865D98DF91CF910895EF92FF920F936B
:10E000001F93CF93C82F7B018A0180912207833011
:10E01000E0F00E943C3EC7010E9499348DE39AE2F1
:10E020000E949934C7FD0EC08BE39AE20E94993496
:10E030006C2FCC0F770B880B990B0E9474B08AE081
:10E040000E9478348AE00E947834C8DFA8958091D5
:10E05000670681110DC081E08093670682E080939E
:10E060002207BCDF40E068E37AE2C8010E94603F1B
:10E07000CF911F910F91FF90EF900895CF93DF9371
:10E08000A89580918412909185120E94ECB16093C2
:10E090008612709387128093881290938912C09190
:10E0A0008412D09185128091600190916101C8170E
:10E0B000D90734F449E75AE266E87AE280E09DDF66
:10E0C00080918A1290918B12181619066CF4809127
:10E0D0005E0190915F018C179D0734F448E95AE284
:10E0E00065EA7AE280E089DFDF91CF9108958F922F
:10E0F0009F92AF92BF92CF92DF92EF92FF92CF9317
:10E10000DF9300D000D0CDB7DEB780912207811118
:10E1100010C0A8950F900F900F900F90DF91CF91A6
:10E12000FF90EF90DF90CF90BF90AF909F908F9037
:10E130000895809168068111EDCF81E08093680693
:10E1400080917F05811103C010926806E3CF96DFAE
:10E1500010927F050E94E0CC6B017C010E948FB081
:10E160004B015C016091640170916501072E000C08
:10E17000880B990B0E9497E79B01AC01C501B40184
:10E180000E944EF018160CF469C060918A127091CA
:10E190008B12072E000C880B990B0E9497E769835E
:10E1A0007A838B839C83CE0101960E942BCD809035
:10E1B000861290908712A0908812B0908912609178
:10E1C000620170916301072E000C880B990B0E946D
:10E1D00097E79B01AC01C501B4010E944EF01816EF
:10E1E000CCF46091640170916501072E000C880BDE
:10E1F000990B0E9497E79B01AC01C501B4010E94F5
:10E2000091E787FF07C00E9498B00E9491EF759533
:10E21000679501C060E060938C1280917E129091AE
:10E220007F12A0918012B09181120097A105B105D3
:10E2300009F48ACFC81AD90AEA0AFB0AF7FC84CF84
:10E240000E948FB00E9491EF20917C1230917D123C
:10E250006217730754F00E94ECCC76CF49E75AE27C
:10E2600066E87AE280E0C9DE90CF4BE55AE26AE6E2
:10E270007AE280E0C2DE68CFCF92DF92EF92FF9227
:10E28000CF93DF93EC01C880D980EA80FB808EE2D7
:10E290009AE20E949934C701B6010E949C26CC8064
:10E2A000DD80EE80FF8080EC90E30E949934C7010E
:10E2B000B6010E949C26C884D984EA84FB848CEB36
:10E2C00090E30E949934C701B6010E949C268AE01F
:10E2D0000E947834DF91CF91FF90EF90DF90CF9044
:10E2E0000895BC01209148063091490640914806A6
:10E2F000509149062417350731F481E02617370776
:10E3000009F080E008959A01F1CF0F930FB70F93B2
:10E3100000916E000F930B7F00936E0000916F00D1
:10E320000D7F00936F000F930BB70F930CB70F92F5
:10E330001F922F933F934F935F936F937F938F938E
:10E340009F93AF93BF93EF93FF931124D7D5FF9182
:10E35000EF91BF91AF919F918F917F916F915F915D
:10E360004F913F912F911F900F900CBF0F910BBFBA
:10E370000F910260F89400936F000F9100936E006C
:10E380000F910FBF0F91189500C000C08091DC065F
:10E3900080FF1FC0459A8FEF809301068091DC06B5
:10E3A00081FF1AC0479A8FEF809302068091DC06A6
:10E3B00082FF15C02A988FEF809303068091DC06B8
:10E3C00083FF10C028988FEF8093040600C000C020
:10E3D0000895459881E0E0CF479881E0E5CF2A9AFB
:10E3E00081E0EACF289A81E0EFCF80917505982FE0
:10E3F000977F90937505982F937081E011F080E0DE
:10E4000008955E9A08955E9880917505886080935E
:10E4100075050895E82FF0E021E030E0082E02C0F5
:10E42000220F331F0A94E2F72095309590917505DD
:10E43000922390937505E15EFD4F2081922321E0A8
:10E4400019F020E0822F0895813079F038F0823081
:10E45000C9F7159A90914F079B7F04C05E9A9091DF
:10E460004F079E7F90934F07EDCF5E9A90914F0795
:10E470009D7FF8CF80E0CEDF81E0CCDF82E0CADF95
:10E48000B4CF813079F070F0823071F021E030E06B
:10E4900001C0220F8A95EAF780917505822B80933F
:10E4A000750508955E98F2CF1598F0CFB0E0A0E022
:10E4B000ECE5F2E70C9481EEC82F61E072E20E9475
:10E4C000EBC2C11102C00E94403E89EF91E20E945E
:10E4D000993485E691E20E9499348AE00E9478346A
:10E4E00067EE71E28C2F0E94EBC2C11102C00E9444
:10E4F000403E8AEC91E20E9499348C2F0E940BC31B
:10E500008C2F0E9435398C2F0E945C398C2F0E94F1
:10E5100015398C2F0E94E13861E871E28C2F0E943E
:10E5200002C3D0919F0488E791E20E9499346D2F35
:10E5300070E090E080E00E9474B040919B045091A4
:10E540009C0460919D0470919E0481ED9FE20E9465
:10E55000C4348BE691E20E94993480919F040E941A
:10E56000303E20E030E0A9016091A0047091A10448
:10E570008091A2049091A3040E9491E78823A1F1C5
:10E5800080EBE82E84E0F82E10E0670100E0C11176
:10E5900002C00E94403E80EC91E20E949934802F9C
:10E5A0000E947B288DEB91E20E949934812F0E947A
:10E5B0007B2881ED9FE20E949934F6016081718190
:10E5C0008281938145E00E94BEB28AE00E94783445
:10E5D0000F5FFCE1CF0ED11C0730C9F61F5F84E04E
:10E5E000E80EF11C173089F662EA71E28C2F0E9466
:10E5F000EBC208EA14E0D0E0C11102C00E94403E24
:10E6000089E991E20E9499348D2F0E947B28F801BC
:10E6100060817181072E000C880B990B0E9497E78F
:10E62000AB01BC0186E991E20E94C434F801E280AA
:10E63000F38083E991E20E949934C7010E94332C50
:10E640008AE00E9478340C5F1F4FD13059F48C2F30
:10E650000E946C3E8C2F0E94D534CDB7DEB7E8E027
:10E660000C949DEED1E0C8CFB0E0A0E0EAE3F3E780
:10E670000C947FEEC1E4DDE007E617E081E5A82E0B
:10E680008DE0B82EC12CD12C7601C394699179917B
:10E69000899199910E9495E7288939894A895B89EE
:10E6A0000E94F6E70E9496EFF801619371938193BF
:10E6B00091938F01C616D706E806F90610F46B0190
:10E6C0007C01AC16BD0611F76FEF7FEFCB01A70100
:10E6D00096010E94BFED209377073093780740930F
:10E6E000790750937A07CDB7DEB7EAE00C949BEE3A
:10E6F0000F931F93CF93DF9305E51DE0C0E8D7E0AC
:10E70000F80121913191419151918F0160E070E0C8
:10E7100080E89FE30E9429EF699379938993999305
:10E72000F7E0C039DF0761F70E94D0C29DDFDF91BB
:10E73000CF911F910F910895DBCFDACFD9CFD8CFEA
:10E7400090912E1380912F13981306C08091890DFC
:10E7500090918A0D892B21F080E00E945140F0CFEA
:10E76000089590912E1380912F13981307C08091D4
:10E77000890D90918A0D892B09F47CCE80E00E944E
:10E780005140EFCFCF92DF92EF92FF92CF93DF9382
:10E7900020919F04222319F1EC0108960E9403287E
:10E7A0006B017C0120E030E0A9010E9491E720E0AC
:10E7B00030E0A901882349F0CE010E948128A701F9
:10E7C00096010E94F6E79B01AC01688579858A85F0
:10E7D0009B850E94AEEE688779878A879B87DF9149
:10E7E000CF91FF90EF90DF90CF900895CF92DF927E
:10E7F000EF92FF92CF93DF9320919F04222319F190
:10E80000EC0108960E9403286B017C0120E030E0B7
:10E81000A9010E9491E720E030E0A901882349F096
:10E82000CE010E948128A70196010E94F6E79B0174
:10E83000AC01688579858A859B850E94AFEE6887E3
:10E8400079878A879B87DF91CF91FF90EF90DF9048
:10E85000CF900895AEE1B0E0E0E3F4E70C9479EEF8
:10E860009E8F8D8F5B018A01FC01EA5BFF4F208147
:10E87000318142815381298B3A8B4B8B5C8BCA014E
:10E88000B9010E9495E76B017C01D5012D913D9165
:10E890004D915C910E94F6E70E9413EF2B013C0121
:10E8A000F8012081318142815381C701B6010E9464
:10E8B000F6E70E9413EF4B015C01C301B2010E9415
:10E8C00096EF6D8B7E8B8F8B988F683771058105E6
:10E8D000910540F428E730E040E050E02D8B3E8B7E
:10E8E0004F8B588FC501B4010E9496EF698F7A8FC4
:10E8F0008B8F9C8F683771058105910540F488E7FF
:10E9000090E0A0E0B0E0898F9A8FAB8FBC8FED8D47
:10E91000FE8DEE5AFF4F208131814281538129873C
:10E920003A874B875C87CA01B9010E9497E72B01A0
:10E930003C016D897E898F89988D0E9495E76D8352
:10E940007E838F83988720E030E0A901C301B20164
:10E950000E9491E7882309F4BBC1A7019601C70172
:10E96000B6010E94F6E74B015C012D813E814F818B
:10E970005885CA01B9010E94F6E79B01AC01C501A7
:10E98000B4010E94AEEE4B015C01A3019201C301F0
:10E99000B2010E94AFEE9B01AC01C501B4010E941F
:10E9A00029EF0E9413EF0E9496EF69837A838B838D
:10E9B0009C8369857A858B859C85909580957095DB
:10E9C00061957F4F8F4F9F4F0E9497E74B015C01EE
:10E9D000698D7A8D8B8D9C8D0E9495E769877A87EA
:10E9E0008B879C8720E030E0A901C501B4010E941B
:10E9F00091E7882309F470C129853A854B855C85A8
:10EA0000CA01B9010E94F6E76D877E878F87988BD0
:10EA1000A7019601C701B6010E94F6E79B01AC0170
:10EA20006D857E858F8598890E94AEEE6B017C0195
:10EA3000A5019401C501B4010E94AFEE9B01AC0198
:10EA4000C701B6010E9429EF0E94C2EFAD8DBE8DB5
:10EA500095962D913D914D915C9198972D873E878C
:10EA60004F87588B69017A0129813A814B815C81FA
:10EA7000C21AD30AE40AF50A0E9496EFC61AD70A08
:10EA8000E80AF90AF7FE8CC02D813E814F81588536
:10EA9000CA01B9010E94F6E76B017C0120E030E079
:10EAA000A901C301B2010E9491E7882309F418C1AA
:10EAB0006D857E858F8598890E9495E79B01AC01C5
:10EAC0000E94AFEEA30192010E94F6E74B015C01A8
:10EAD00029853A854B855C85CA01B9010E94F6E714
:10EAE0009B01AC01C501B4010E94AFEEA7019601E4
:10EAF0000E94AEEE4B015C0120E030E040E850E4C3
:10EB0000C301B2010E94F6E79B01AC01C501B4014B
:10EB10000E9429EF0E9413EF4B015C0120E030E0DE
:10EB2000A9010E944EF087FF03C0812C912C540153
:10EB3000C501B4010E9496EF69837A838B839C831D
:10EB40002D853E854F855889261737074807590771
:10EB500020F429833A834B835C8369817A818B819A
:10EB60009C810E9495E74B015C01A3019201C301C6
:10EB7000B2010E94AFEE9B01AC01C501B4010E943D
:10EB8000F6E7A70196010E94AFEE0E948DF00E9469
:10EB900096EF698B7A8B8B8B9C8BC12CD12C760159
:10EBA00069897A898B899C892D893E894F89588DFD
:10EBB000621B730B840B950B0E9495E7A3019201D6
:10EBC0000E9429EF20E034E244EF59E40E94F6E786
:10EBD0000E9496EF4B015C0169897A898B899C8937
:10EBE000298D3A8D4B8D5C8D621B730B840B950BBD
:10EBF0000E9495E7A30192010E9429EF20E034E2F0
:10EC000044EF59E40E94F6E70E9496EF6D837E83FD
:10EC10008F839887C501B4010E946A622B013C0171
:10EC20006D817E818F8198850E946A6229813A81F7
:10EC30004B815C81AD8DBE8D99962D933D934D9307
:10EC40005C939C9789019A010C0D1D1D2E1D3F1D83
:10EC5000FD0105A716A727A730ABE65BFF4F2D895F
:10EC60003E894F89588D2083318342835383D596C3
:10EC70008D929D92AD92BC92D8972D813E814F810D
:10EC80005885D9962D933D934D935C93DC973D9792
:10EC90004082518262827382349660837183828360
:10ECA000938329893A894B895C89D1962D933D9329
:10ECB0004D935C93D4973D96298D3A8D4B8D5C8D09
:10ECC00020833183428353836E96E0E10C9495EE6A
:10ECD00060E070E0CB0165CE60E070E0CB01B4CEC7
:10ECE00060E070E0CB0116CF90916F0081E091FD64
:10ECF00002C080E0089590916F009D7F90936F0017
:10ED00000895EFE6F0E08081826080830895CF93DC
:10ED1000C82FEADF94E0C99F90011124F901E55B57
:10ED2000F94F295A394FD9014D915D916D917C91DF
:10ED3000408351836283738391E090934A068111EB
:10ED4000E0DFCF910895CF93DF938091DB068111AF
:10ED500005C08091DD06882309F464C08091DC053C
:10ED6000329B63C081608093DC058091DC05339B1E
:10ED70005EC082608093DC058091DC05349B59C0C5
:10ED800084608093DC058091DC05029B54C0886020
:10ED90008093DC05C0913B06C0FF0FC08091DC066C
:10EDA00080FF0BC08091DC0580FF07C080912107A8
:10EDB00081608093210780E0AADFC1FF0FC08091AE
:10EDC000DC0681FF0BC08091DC0581FF07C08091CC
:10EDD000210782608093210781E099DFC2FF22C072
:10EDE0008091DC0682FF1EC08091DD0681110BC080
:10EDF0008091DC0582FF07C08091210784608093A9
:10EE0000210782E084DF8091DD06882359F080911C
:10EE1000DC0583FF07C0809121078860809321076C
:10EE200082E075DFDF91CF9108958E7F9CCF8D7F3B
:10EE3000A1CF8B7FA6CF877FABCF56DF10927B070A
:10EE400010927C0710927D0710927E07811159CF96
:10EE500008950F931F9380912E1390912F13891B68
:10EE60008F7009F449C090912B13992361F083307E
:10EE700040F48FEF890F29F080932B1390E080E00E
:10EE800038C010922B1380912F132BE5829FC00165
:10EE900011248057984FFC01208120FDEFCF409135
:10EEA0007B0750917C0760917D0770917E07E95A3E
:10EEB000FF4F0081118122813381401B510B620B76
:10EEC000730B40937B0750937C0760937D0770938F
:10EED0007E0720912F132F5F2F7020932C133091DA
:10EEE0002F1320912D13321304C020912C13209343
:10EEF0002D131F910F910895A0DFC0CFA3E1B0E0C3
:10EF0000E4E8F7E70C9477EE8FEF9FEF909389009A
:10EF1000809388002AE02983312C212C78948091D9
:10EF2000440690914506A0914606B0914706892B6C
:10EF30008A2B8B2B09F0C2C180914A068823D1F01D
:10EF4000809148069091490610924A06892B91F0CB
:10EF5000109249061092480610923B0690912E138B
:10EF600080912F13981731F080912F138F5F8F703E
:10EF700080932F138091480690914906892B09F4BC
:10EF80009DC14091400650914106609142067091AA
:10EF9000430680913C0690913D06A0913E06B091BB
:10EFA0003F060091320610E030E020E0841B950B14
:10EFB000A60BB70B081719072A073B0710F4D9014E
:10EFC000C8018A8B840F951FA61FB71F8093400628
:10EFD00090934106A0934206B0934306E1E0C090AF
:10EFE0000906D0900A06E0900B06F0900C0680917E
:10EFF000190690911A06A0911B06B0911C06C80E26
:10F00000D91EEA1EFB1EC0921906D0921A06E09283
:10F010001B06F0921C06F7FC33C040910106042E3B
:10F02000000C550B660B770B809157069091580694
:10F03000A0915906B0915A06840F951FA61FB71FBD
:10F040008093570690935806A0935906B0935A069A
:10F050008091050690910606A0910706B0910806DA
:10F06000B701A601481B590B6A0B7B0BDB01CA01D8
:10F070008093190690931A06A0931B06B0931C0662
:10F0800000910D0610910E0620910F06309110068A
:10F0900080911D0690911E06A0911F06B09120063A
:10F0A000080F191F2A1F3B1F00931D0610931E06F1
:10F0B00020931F063093200637FD33C0409102068F
:10F0C000042E000C550B660B770B80915B0690911C
:10F0D0005C06A0915D06B0915E06840F951FA61F89
:10F0E000B71F80935B0690935C06A0935D06B09378
:10F0F0005E068091050690910606A0910706B091E4
:10F10000080628013901481A590A6A0A7B0AD301FC
:10F11000C20180931D0690931E06A0931F06B09314
:10F1200020064091110650911206609113067091CD
:10F1300014068091210690912206A0912306B09199
:10F140002406480F591F6A1F7B1F409321065093C6
:10F150002206609323067093240677FD33C08090C7
:10F160000306082C000C9908AA08BB0880915F06CA
:10F1700090916006A0916106B0916206880D991D7C
:10F18000AA1DBB1D80935F0690936006A093610645
:10F19000B09362068091050690910606A09107063D
:10F1A000B09108063A014B01681A790A8A0A9B0A4B
:10F1B000D401C3018093210690932206A0932306D5
:10F1C000B09324068090150690901606A09017061E
:10F1D000B09018068091250690912606A0912706EA
:10F1E000B0912806880D991DAA1DBB1D8093250688
:10F1F00090932606A0932706B0932806B7FD33C048
:10F2000040900406042C000C55086608770880908E
:10F21000630690906406A0906506B0906606840C24
:10F22000951CA61CB71C8092630690926406A0925F
:10F230006506B09266068090050690900606A0903E
:10F240000706B09008062C013D01481859086A08C5
:10F250007B08530142018092250690922606A092D7
:10F260002706B0922806E11104C0E0918400F091D5
:10F270008500F7FE5F9A37FF469A77FF2B9AB7FF14
:10F28000299AE0918400F0918500E0918400F0914A
:10F290008500F7FE5F9837FF469877FF2B98B7FFFA
:10F2A00029985A88552021F08091840090918500FA
:10F2B0002A8921502A8BE0E0211191CE80914406C9
:10F2C00090914506A0914606B0914706892B8A2B5E
:10F2D0008B2B09F0B0C640904806509049065B8AD7
:10F2E0004A8A4114510409F402C780914006909162
:10F2F0004106A0914206B091430640913C065091D0
:10F300003D0660913E0670913F0684179507A6075B
:10F31000B70708F449C010924906109248061092A7
:10F320003B0690912E1380912F13981709F4DFC696
:10F3300080912F138F5F8F7080932F13A0EDCA2EB3
:10F34000A7E0DA2EE12CF12C809148069091490635
:10F35000892B09F068C67DDD9093490680934806A5
:10F36000892B09F460C640904806509049065B8A94
:10F370004A8AD2018C9183FF08C5C20145960E943A
:10F380000962109249061092480610923B0690912D
:10F390002E1380912F139817F1F280912F138F5F06
:10F3A0008F7080932F13D7CF409137065091380636
:10F3B0006091390670913A06481759076A077B072A
:10F3C00008F40FC24091330650913406609135061F
:10F3D00070913606EA89FB8985A996A9A7A9B0ADDF
:10F3E000481759076A077B0708F0D0C14115510536
:10F3F0006105710509F066C080907A0590907B05E3
:10F40000A0907C05B0907D058EE09AE2A1E0FC0121
:10F410000591159125913491081519052A053B058B
:10F4200058F4B694A79497948794AA0F0496EAE2A6
:10F43000FAE2E817F90759F7A0933206F0E28F16BF
:10F440009104A104B10428F4E0E28E2E912CA12CA9
:10F45000B12C20E2821A9108A108B108811438E089
:10F460009306A104B10408F49AC1A4E09A9EC001D5
:10F470001124825F994DFC01329625913491B82D6B
:10F48000EE27B39F8001B29F010D1E1F06940E1F31
:10F490001E1F112430E020E0FC01C590D490F12C17
:10F4A000E12CC01AD10AE20AF30A4C0D5D1D6E1D53
:10F4B0007F1D409333065093340660933506709356
:10F4C000360642CF10E00A81942F852E862FBC810C
:10F4D000AD81FE81EF81388529854B80E0917605ED
:10F4E000E99FA12DFF2730917705399FA00DF11DD0
:10F4F00010907805199EF00DE89DA00DF11D389D26
:10F50000F00DE89FF00D4A2EBF2F4A9EE12D3327C4
:10F5100022274F9EE00D311D211FBA9FE00D311DA6
:10F52000211FBF9F300D211D432EB22F4A9E012D5A
:10F53000332722274F9E000D311D211FBA9F000D3A
:10F54000311D211FBF9F300D211D432EB22FEE27ED
:10F5500090917A0580907B0580917C050090A002B7
:10F56000012A09F483C030919C02349DE119910B6A
:10F57000810A810B20919D02249DE0199109810A45
:10F58000810B00919E02049D90198108810B3B9F85
:10F59000E0199109810A810B2B9F90198108810B39
:10F5A0000B9F801881094A9E012D332722274F9EE9
:10F5B000000D311D211FBA9F000D311D211FBF9F5E
:10F5C000300D211D432EB22F30919802349DE10D54
:10F5D000911F811E811F20919902249DE00D911D94
:10F5E000811E811F00919A02049D900D811C811F34
:10F5F0003B9FE00D911D811E811F2B9F900D811C53
:10F60000811F0B9F800C811D4A9E012D33272227CD
:10F610004F9E000D311D211FBA9F000D311D211F6E
:10F62000BF9F300D211D432EB22F30919402349D87
:10F63000E119910B810A810B20919502249DE0191B
:10F640009109810A810B00919602049D901981080D
:10F65000810B3B9FE0199109810A810B2B9F901927
:10F660008108810B0B9F8018810982C030919C0218
:10F67000349DE10D911F811E811F20919D02249DCB
:10F68000E00D911D811E811F00919E02049D900D31
:10F69000811C811F3B9FE00D911D811E811F2B9FAF
:10F6A000900D811C811F0B9F800C811D4A9E012D96
:10F6B000332722274F9E000D311D211FBA9F000DB9
:10F6C000311D211FBF9F300D211D432EB22F3091C0
:10F6D0009802349DE119910B810A810B20919902C6
:10F6E000249DE0199109810A810B00919A02049DE1
:10F6F00090198108810B3B9FE0199109810A810BC8
:10F700002B9F90198108810B0B9F801881094A9EBD
:10F71000012D332722274F9E000D311D211FBA9F37
:10F72000000D311D211FBF9F300D211D432EB22F13
:10F7300030919402349DE10D911F811E811F209113
:10F740009502249DE00D911D811E811F009196025E
:10F75000049D900D811C811F3B9FE00D911D811E1A
:10F76000811F2B9F900D811C811F0B9F800C811D81
:10F7700011244B820A83BC83AD83FE83EF833887D9
:10F780002987982C892EB12CA82E3ECEAA89BB8918
:10F79000D1968D909D90AD90BC90D49735CED501EB
:10F7A000C401B695A795979587958C7F825F9D4DEF
:10F7B000FC01C590D490FC01329625913491E82D3E
:10F7C000E7708E2EE29FC001E39F900D112433E07D
:10F7D000969587953A95E1F7C81AD90AF12CE12C4C
:10F7E00064CE40912E0650912F06609130067091A4
:10F7F0003106481759076A077B0708F030C2809026
:10F80000290690902A06A0902B06B0902C06809195
:10F810002D06EA89FB8981117CC0EF5BFF4FE080F8
:10F82000F18002811381EA89FB89E25BFF4F20812D
:10F83000318142815381AA89BB89D1966D917D9195
:10F840008D919C91D4970E941262B1E0B0932D06E5
:10F85000EA89FB8941A952A963A974A98EE09AE2B9
:10F86000A1E0FC010591159125913491041715072C
:10F870002607370758F47695679557954795AA0F49
:10F880000496EAE2FAE2E817F90759F7A09332067C
:10F89000403251056105710520F440E250E060E01E
:10F8A00070E040525109610971094115F8E05F07A4
:10F8B0006105710508F4B3C124E0529FC001112411
:10F8C000825F994DFC01329625913491AA27439F7E
:10F8D000F001429FE10DFA1F0694EA1FFA1F11245E
:10F8E000AF0170E060E0FC01C590D490F12CE12CF8
:10F8F000C41AD50AE60AF70A8C0C9D1CAE1CBF1C64
:10F900008092290690922A06A0922B06B0922C068D
:10F910001BCD81AD92ADA3ADB4AD88169906AA06F4
:10F92000BB0608F072C181149104A104B10449F42A
:10F9300040917A0550917B0560917C0570917D0521
:10F940008DCFA0E0BA85982D492D8A2DFB85EC85B9
:10F950007D856E855F853889298950917605599F07
:10F96000712D662730917705399F700D611D1090BC
:10F970007805199E600D549F700D611D349F600DB8
:10F98000589F600DF72FE62FF79F512D3327222721
:10F99000F69F500D311D2A1FE79F500D311D2A1F64
:10F9A000E69F300D211DF32FE22FF79FB12D332756
:10F9B0002227F69FB00D311D2A1FE79FB00D311D84
:10F9C0002A1FE69F300D211DF32FE22F552790911E
:10F9D0007A0540917B0580917C050090A0020A2A5F
:10F9E00009F483C030919C023F9F51199A0B4A0B36
:10F9F0008A0B20919D022F9F501991094A0B8A0B67
:10FA0000B0919E02BF9F901941098A0B3E9F5019E9
:10FA100091094A0B8A0B2E9F901941098A0BBE9FB0
:10FA200040198109F79FB12D33272227F69FB00D8A
:10FA3000311D2A1FE79FB00D311D2A1FE69F300D93
:10FA4000211DF32FE22F309198023F9F510D9A1FF5
:10FA50004A1F8A1F209199022F9F500D911D4A1F06
:10FA60008A1FB0919A02BF9F900D411D8A1F3E9F31
:10FA7000500D911D4A1F8A1F2E9F900D411D8A1FF8
:10FA8000BE9F400D811DF79FB12D33272227F69F82
:10FA9000B00D311D2A1FE79FB00D311D2A1FE69FB3
:10FAA000300D211DF32FE22F309194023F9F511909
:10FAB0009A0B4A0B8A0B209195022F9F501991099E
:10FAC0004A0B8A0BB0919602BF9F901941098A0B8D
:10FAD0003E9F501991094A0B8A0B2E9F901941099C
:10FAE0008A0BBE9F4019810982C030919C023F9FC2
:10FAF000510D9A1F4A1F8A1F20919D022F9F500D62
:10FB0000911D4A1F8A1FB0919E02BF9F900D411DFB
:10FB10008A1F3E9F500D911D4A1F8A1F2E9F900DD8
:10FB2000411D8A1FBE9F400D811DF79FB12D3327B8
:10FB30002227F69FB00D311D2A1FE79FB00D311D02
:10FB40002A1FE69F300D211DF32FE22F30919802DE
:10FB50003F9F51199A0B4A0B8A0B209199022F9FB4
:10FB6000501991094A0B8A0BB0919A02BF9F9019C4
:10FB700041098A0B3E9F501991094A0B8A0B2E9F0F
:10FB8000901941098A0BBE9F40198109F79FB12D39
:10FB900033272227F69FB00D311D2A1FE79FB00D96
:10FBA000311D2A1FE69F300D211DF32FE22F3091CA
:10FBB00094023F9F510D9A1F4A1F8A1F2091950260
:10FBC0002F9F500D911D4A1F8A1FB0919602BF9F13
:10FBD000900D411D8A1F3E9F500D911D4A1F8A1F87
:10FBE0002E9F900D411D8A1FBE9F400D811D112427
:10FBF000BA87FB87EC877D876E875F87388B298B79
:10FC0000542F492F70E0682F29CE2A893B89225B27
:10FC10003F4FD9014D915D916D917C911FCEDB01DC
:10FC2000CA01B695A795979587958C7F825F9D4D64
:10FC3000FC01C590D490FC01329625913491477017
:10FC4000429FC001439F900D1124A3E09695879594
:10FC5000AA95E1F7C81AD90AF12CE12C4DCE809172
:10FC6000570190915801A0915901B0915A01B7FFE5
:10FC700061C0EA89FB89EA5BFF4FC080D180E280E6
:10FC8000F3808EE09AE221E0FC0145915591659167
:10FC900074914C155D056E057F0558F4F694E79454
:10FCA000D794C794220F04964AE25AE2481759079C
:10FCB00059F72093320650E2C516D104E104F1044D
:10FCC00028F470E2C72ED12CE12CF12C60E2C61A88
:10FCD000D108E108F108C11478E0D706E104F10485
:10FCE00008F431C0A4E0DA9EC0011124825F994D6E
:10FCF000FC01329625913491BC2D6627B39FA0015B
:10FD0000B29F410D561F0694461F561F112470E0E6
:10FD100060E0FC0185919491B0E0A0E0841B950B1C
:10FD2000A60BB70B8093570190935801A0935901EC
:10FD3000B0935A01C0905701D0905801E0905901FA
:10FD4000F0905A0101CBD701C601B695A7959795BA
:10FD500087958C7F825F9D4DFC0125913491FC013C
:10FD6000329645915491EC2DE770E49FC001E59FD8
:10FD7000900D112463E0969587956A95E1F7281B0D
:10FD8000390BC901B0E0A0E0CDCFEA89FB898588B5
:10FD90009688A788B08C81E081149104A104B104F5
:10FDA00009F480E0AA89BB895996CD90DD90ED9049
:10FDB000FC905C97C114D104E104F10409F0826065
:10FDC000EA89FB89458D568D678D70A141155105D6
:10FDD0006105710509F0846080933B061092290645
:10FDE00010922A0610922B0610922C0610923306BF
:10FDF000109234061092350610923606EA89FB8975
:10FE000085A196A1A7A1B0A580933C0690933D063D
:10FE1000A0933E06B0933F06442455243201481A6D
:10FE2000590A6A0A7B0A4092190650921A06609291
:10FE30001B0670921C0640921D0650921E06609290
:10FE40001F06709220064092210650922206609270
:10FE500023067092240641A052A063A074A0440C13
:10FE6000551C661C771C880C991CAA1CBB1C809214
:10FE7000090690920A06A0920B06B0920C06CC0CD2
:10FE8000DD1CEE1CFF1CC0920D06D0920E06E09207
:10FE90000F06F0921006440F551F661F771F409300
:10FEA0001106509312066093130670931406409245
:10FEB0001506509216066092170670921806880F63
:10FEC000991FAA1FBB1F8093050690930606A09357
:10FED0000706B09308061092400610924106109251
:10FEE00042061092430681A592A5A3A5B4A58093CE
:10FEF000370690933806A0933906B0933A0685A545
:10FF000096A5A7A5B0A980932E0690932F06A0933F
:10FF10003006B0933106EB5BFF4F80819091DC0699
:10FF2000891721F08093DC060E94C4710E94A37699
:10FF300044244A94542C3201409257015092580163
:10FF40006092590170925A01EA89FB89FD96E0801E
:10FF5000F18002811381AA89BB89D1962D913D91AF
:10FF60004D915C91D4976D01BAE4CB0ED11CF60192
:10FF700060817181828193810E94126210922D06AC
:10FF8000D6014D915D916D917C918EE09AE2A1E058
:10FF9000FC01059115912591349104171507260749
:10FFA000370758F47695679557954795AA0F0496A5
:10FFB000EAE2FAE2E817F90759F7A093320640326D
:10FFC00051056105710520F440E250E060E070E009
:10FFD00040525109610971094115F8E05F07610557
:10FFE000710508F462C024E0529FC0011124825FB1
:10FFF000994DFC01329625913491AA27439FF00137
:020000021000EC
:10000000429FE10DFA1F0694EA1FFA1F1124AF0167
:1000100070E060E0FC01C590D490F12CE12CC41A92
:10002000D50AE60AF70AC0924406D0924506E09245
:100030004606F09247068091440690914506A091AD
:100040004606B0914706AC01BD01009731E0A30719
:10005000B10520F04FEF5FEF60E070E0841B950B7F
:10006000A60BB70B8093440690934506A0934606D3
:10007000B0934706F8948091840090918500409653
:10008000A981A150A983AA2381F1240E351E281627
:10009000390610F40C948E773092890020928800F3
:1000A00078946396E2E10C9493EEDB01CA01B69575
:1000B000A795979587958C7F825F9D4DFC01C59094
:1000C000D490FC013296259134914770429FC00133
:1000D000439F900D112433E0969587953A95E1F76B
:1000E000C81AD90AF12CE12C9ECF1C01D5CF80ED86
:1000F000C82E87E0D82EE12CF12C2DC9CF93DF93A9
:1001000080912E1390912F13891B80958F7019F475
:100110000E945140F5CF80912E138F5F8F70A09178
:100120002E139BE5A99FD0011124FD01E057F84F44
:10013000EF0119929A95E9F798E09083AB55B84F83
:1001400090E1E0E3F3E101900D929A95E1F72091BF
:100150002E1390912F13291303C094E690932B1321
:1001600080932E130E948176DF91CF910895FC0138
:1001700020813181428153816091610D7091620DC6
:100180008091630D9091640D0E94F6E70E9453F0F8
:1001900060933C1370933D1380933E1390933F13F1
:1001A00090912E1380912F13981709F0A7CF0E94DA
:1001B000A0730E94747640913C1350913D1360915E
:1001C0003E1370913F13409363065093640660930F
:1001D00065067093660681110C94817608954F929E
:1001E0005F926F927F928F929F92AF92BF92CF92C7
:1001F000DF92EF92FF92CF93DF93EC012091610D9C
:100200003091620D4091630D5091640D6C857D8538
:100210008E859F850E94F6E70E9453F06B017C015A
:1002200020915D0D30915E0D40915F0D5091600DFC
:10023000688579858A859B850E94F6E70E9453F040
:100240004B015C012091590D30915A0D40915B0D8D
:1002500050915C0D6C817D818E819F810E94F6E7BB
:100260000E9453F02B013C012091550D3091560D09
:100270004091570D5091580D688179818A819B81F9
:100280000E94F6E70E9453F060933013709331138D
:10029000809332139093331340923413509235135A
:1002A00060923613709237138092381390923913FC
:1002B000A0923A13B0923B13C0923C13D0923D13DC
:1002C000E0923E13F0923F1390912E1380912F13E2
:1002D000981781F013DFDF91CF91FF90EF90DF90BF
:1002E000CF90BF90AF909F908F907F906F905F90D6
:1002F0004F9008950E94A0730E947476C82F80E3E7
:1003000093E10E940962CC2331F30E948176E3CF0E
:10031000CF92DF92EF92FF92CF93DF93C82F0E948C
:10032000747694E0C99FE0011124FE01E95AF94F67
:10033000C080D180E280F38081110E948176C05814
:10034000D84FC701B6010E9497E7288139814A81B9
:100350005B810E94F6E7DF91CF91FF90EF90DF90F5
:10036000CF9008958F929F92AF92BF92CF92DF92DB
:10037000EF92FF921F93CF93DF93CDB7DEB76097D5
:100380000FB6F894DEBF0FBECDBF182F80E0C0DFE0
:100390004B015C018092DD059092DE05A092DF05A5
:1003A000B092E00581E0B4DF6B017C01C092E10511
:1003B000D092E205E092E305F092E40582E0A8DF46
:1003C0006093E5057093E6058093E7059093E80553
:1003D0001D861E861F86188A89829A82AB82BC82FD
:1003E000CD82DE82EF82F88669877A878B879C8749
:1003F00083E08EDF6D877E878F87988BCE01019695
:100400000E94C2731E3FD9F480E1FE013196A2E73B
:10041000B1E001900D928A95E1F760960FB6F894DD
:10042000DEBF0FBECDBFDF91CF911F91FF90EF9048
:10043000DF90CF90BF90AF909F908F90089584E011
:10044000189FF0011124DF01AE58BE4F81E090E00B
:100450008C0F9D1FE80FF91F4081518162817381CC
:100460004D935D936D937C931397D7CFCF92DF928B
:10047000EF92FF92CF93DF93C82F0E94747694E09F
:10048000C99FE0011124FE01E55BF94FC080D180D6
:10049000E280F38081110E948176C058D84FC70155
:1004A000B6010E9497E7288139814A815B810E94C9
:1004B000F6E7DF91CF91FF90EF90DF90CF90089516
:1004C000A1E0B0E0E6E6F2E80C9487EE898360E014
:1004D000CE0101960E94646361E0CE0101960E9404
:1004E000646362E0CE0101960E9464638981219673
:1004F000E2E00C94A3EEA2E1B0E0E1E8F2E80C94B3
:1005000083EEDEDF8823C1F1EDB6FEB642E952E0AC
:1005100082FF02C049E852E022E932E081FF02C0D6
:100520002BE832E080FD25C082E992E05F934F9393
:100530003F932F939F938F9388EF9CE19F938F938B
:100540008E010F5F1F4F1F930F930E942AE70E9497
:10055000403EC8010E948A34C8010E9419C20FB6E9
:10056000F894DEBF0FBECDBF81E06296E6E00C944A
:100570009FEE8DE892E0DACF80E0F7CFA0E2B0E026
:10058000E4ECF2E80C9477EE80913B01882309F4C7
:10059000BEC08091EF05082F10E080FF3CC0C090E6
:1005A0003D01D0903E01E0903F01F090400120914C
:1005B0008304309184044091850450918604C701DE
:1005C000B6010E944EF0181644F4C0928304D092F3
:1005D0008404E0928504F0928604C0904901D09092
:1005E0004A01E0904B01F0904C012091830430913E
:1005F00084044091850450918604C701B6010E948D
:1006000091E787FF08C0C0928304D0928404E092EF
:100610008504F092860401FF3CC0C0904101D09057
:100620004201E0904301F090440120918704309111
:1006300088044091890450918A04C701B6010E9440
:100640004EF0181644F4C0928704D0928804E092C9
:100650008904F0928A04C0904D01D0904E01E09040
:100660004F01F0905001209187043091880440910F
:10067000890450918A04C701B6010E9491E787FF5F
:1006800008C0C0928704D0928804E0928904F09256
:100690008A0402FF3CC0C0904501D0904601E09022
:1006A0004701F090480120918B0430918C044091D7
:1006B0008D0450918E04C701B6010E944EF01816A9
:1006C00044F4C0928B04D0928C04E0928D04F0929A
:1006D0008E04C0905101D0905201E0905301F090EF
:1006E000540120918B0430918C0440918D045091E1
:1006F0008E04C701B6010E9491E787FF08C0C0922F
:100700008B04D0928C04E0928D04F0928E04809140
:10071000400D83FD61C020917E0130917F014091A9
:1007200080015091810160918F04709190048091BB
:100730009104909192040E9491E7882309F44CC09F
:100740000E946CB3182F882331F00E94403E8DED3B
:100750009CE10E94993420917E0130917F0140916B
:1007600080015091810160918F047091900480917B
:100770009104909192040E94AEEE9F7720916C01BB
:1007800030916D0140916E0150916F010E94F6E72A
:1007900020E030E046E154E40E944EF01816D4F414
:1007A0000E94403E8EEB9CE10E94993480918F0420
:1007B00090919004A0919104B091920480937E0155
:1007C00090937F01A0938001B09381018FE894E022
:1007D000CEDC02C01111EACF2AE037ED43E25CE340
:1007E0006091350170913601809137019091380107
:1007F0000E94F6E76B017C016091390170913A012A
:10080000072E000C880B990B0E9497E79B01AC0107
:10081000C701B6010E94F6E7698B7A8B8B8B9C8BA4
:1008200080919F04882309F180909B0490909C0400
:10083000A0909D04B0909E04C0908B04D0908C0436
:10084000E0908D04F0908E0420E030E0A901C50115
:10085000B4010E9491E78823F9F0A7019601C50130
:10086000B4010E944EF01816BCF020E030E0A9015F
:10087000BE016F5E7F4F83E894E00E94ADC280E1CD
:10088000E3E8F4E0A2E7B1E001900D928A95E1F788
:10089000A096E2E10C9493EE2091720130917301E5
:1008A00040917401509175016091830470918404AA
:1008B00080918504909186040E94AEEE4B015C010C
:1008C0002091760130917701409178015091790122
:1008D00060918704709188048091890490918A04C2
:1008E0000E94AEEE6D8B7E8B8F8B988F20917A015C
:1008F00030917B0140917C0150917D01C701B6018F
:100900000E94AEEE6D8F7E8F8F8F98A320917E0117
:1009100030917F01409180015091810160918F045D
:100920007091900480919104909192040E94AEEE97
:10093000698F7A8F8B8F9C8F20E030E0A901C501F1
:10094000B4010E9491E781110CC020E030E0A901C0
:100950006D897E898F89988D0E9491E7882309F49B
:1009600084CFA5019401C501B4010E94F6E76B0193
:100970007C012D893E894F89588DCA01B9010E9499
:10098000F6E79B01AC01C701B6010E94AFEE6B0117
:100990007C012D8D3E8D4F8D58A1CA01B9010E9459
:1009A000F6E79B01AC01C701B6010E94AFEE6B01F7
:1009B0007C01298D3A8D4B8D5C8DCA01B9010E9455
:1009C000F6E79B01AC01C701B6010E94AFEE6B01D7
:1009D0007C010E948DF02B013C012CEC3CEB4CE89F
:1009E0005BE2C701B6010E9491E787FF06C0498C10
:1009F0005A8C6B8C7C8CE89477F82DEB37E346E8C7
:100A000055E3C301B2010E9491E787FD38CF2DEC79
:100A10003CEC4CE45EE3C301B2010E94F6E70E94A5
:100A200096EF1B01672B19F422242394312CB1017A
:100A300090E080E00E9495E79B01AC0160E070E0EF
:100A400080E89FE30E9429EF6B017C01AC019B01D0
:100A5000C301B2010E94F6E72B013C01A7019601F8
:100A6000C501B4010E94F6E74B015C01A7019601A4
:100A70006D897E898F89988D0E94F6E76D8B7E8BBC
:100A80008F8B988FA70196016D8D7E8D8F8D98A18C
:100A90000E94F6E76D8F7E8F8F8F98A3A701960136
:100AA000698D7A8D8B8D9C8D0E94F6E7698F7A8F88
:100AB0008B8F9C8F80E1E2E7F1E08E010F5F1F4F8B
:100AC000D80101900D928A95E1F70E94E0CC6B016C
:100AD0007C0128ECC20ED11CE11CF11C81E0281A1B
:100AE000310809F454C00E94E0CC9B01AC012C19E0
:100AF0003D094E095F0957FD4DC06B017C0128EC93
:100B0000C20ED11CE11CF11C80E00E945140A501E5
:100B1000940169817A818B819C810E94AFEE698307
:100B20007A838B839C832D893E894F89588D6D8173
:100B30007E818F8198850E94AFEE6D837E838F8347
:100B400098872D8D3E8D4F8D58A169857A858B852F
:100B50009C850E94AFEE69877A878B879C87298D59
:100B60003A8D4B8D5C8D6D857E858F8598890E9431
:100B7000AFEE6D877E878F87988BA3019201BE01B0
:100B80006F5E7F4FC8010E94ADC28111A7CFA30144
:100B900092016ECE0E947770BACF8091EB05909152
:100BA000EC05A091ED05B091EE0580933501909391
:100BB0003601A0933701B09338018091E9059091F7
:100BC000EA0590933A0180933901089580913501A7
:100BD00090913601A0913701B09138018093EB05D7
:100BE0009093EC05A093ED05B093EE05809139014B
:100BF00090913A019093EA058093E90584E690E0AC
:100C000090933A01809339010895ACE0B0E0EBE0B5
:100C1000F6E80C9479EE2B013C0129873A874B8743
:100C20005C8747015801D601CD90DD90ED90FC9096
:100C300020E030E0A901C701B6010E9491E78111CF
:100C400071C08091680190916901A0916A01B09191
:100C50006B0189839A83AB83BC8320E030E0A901D8
:100C6000C701B6010E9491E7811106C0C12CD12CA9
:100C700080E8E82E80E4F82ECD82DE82EF82F886CE
:100C8000A501940160917A0170917B0180917C01B2
:100C900090917D010E9491E787FF0CC080927A01BC
:100CA00090927B01A0927C01B0927D01CE010596CD
:100CB0000E94766A409272015092730160927401B0
:100CC0007092750189859A85AB85BC858093760184
:100CD00090937701A0937801B0937901CE010196AA
:100CE0000E94766AA501940160917A0170917B015E
:100CF00080917C0190917D010E944EF0181664F461
:100D000080927A0190927B01A0927C01B0927D0149
:100D1000CE0105960E94766A0E94A0732C96E0E1AF
:100D20000C9495EED701C60194CFCF92DF92EF924B
:100D3000FF920F931F936B01FC01E080F180028111
:100D40001381E2E7F1E0248135814681578160819A
:100D500071818281938159DF1F910F91FF90EF90F4
:100D6000DF90CF9008950C94D0C20F931F93CF9330
:100D7000DF93EC018B010E94193F882331F081E061
:100D8000DF91CF911F910F910895B801CE01CDDF72
:100D900080912107C82FC87083FD0AC010922107D7
:100DA00082E0E0DAE0DF81E0CC2351F380E0E8CFBD
:100DB0000E94D83E882391F3E2CFCF930E947476AD
:100DC000C82F80912F1380932E1380932D1380931F
:100DD0002C1384E680932B130E941D7780ED93E003
:100DE00090938A0D8093890DC1110E94817681E0D4
:100DF00080934A060E94A0738EEFB4DAB4DFCF91DD
:100E00000895ACE0B0E0E7E0F7E80C9487EE0E94CC
:100E10002BB30E9474769CE0E7E5F6E0DE011196C4
:100E200001900D929A95E1F781110E948176CE0191
:100E300001960E943C712C96E2E00C94A3EEB0E087
:100E4000A0E0E5E2F7E80C9479EE40907201509052
:100E5000730160907401709075018090760190909C
:100E60007701A0907801B0907901C0907A01D0907C
:100E70007B01E0907C01F0907D010E9434736091D1
:100E8000550170915601072E000C880B990B0E949A
:100E900097E72AE037ED43E25CE30E94F6E76093D0
:100EA0006C0170936D0180936E0190936F010DE35F
:100EB00011E0D0E0C0E0CE01855E9F4D0E94FA2790
:100EC000F80161937193819391938F01CE01815FBA
:100ED0009F4D0E94FA27F801608771878287938768
:100EE0002496CC30D10539F760E08DEF95E00E9473
:100EF000E42A0E94B12B0E947873A30192016091B1
:100F000072017091730180917401909175010E943A
:100F100091E781111BC0A501940160917601709148
:100F2000770180917801909179010E9491E7811178
:100F30000DC020917A0130917B0140917C0150914C
:100F40007D01C701B6010E9491E781115ADFCDB73B
:100F5000DEB7E0E10C9495EEA4E0B0E0E2EBF7E858
:100F60000C9487EE84EF91E0A0E0B0E089839A834F
:100F7000AB83BC83BE016F5F7F4F8CE30E943F3326
:100F800084EA9CE10E94993486B16EE97CE182FB9F
:100F9000882780F90E94046A86B168E97CE183FBB6
:100FA000882780F90E94046A86B162E97CE1829513
:100FB00081700E94046A80B16AE87CE182FB882724
:100FC00080F90E94046A029907C00E947433249633
:100FD000E2E00C94A3EE06C00E945D332496E2E0AA
:100FE0000C94A3EE8091DB06811103C08091DD0695
:100FF00081110C94A3760895ACE0B0E0E2E0F8E84B
:101000000C9487EEA1E4BDE090E080E0FC01EB5A97
:10101000FE4D45915591659174914D935D936D93FE
:101020007D93FC01EB5BFE4D45915591659174916B
:1010300050964D935D936D937C935397FC01EB5CBD
:10104000FE4D459155916591749190964D935D93A8
:101050006D937C939397049680319105B9F680E265
:101060009EE4A0E0B0E08093510D9093520DA093C8
:10107000530DB093540D80E090E0AAEFB3E4809359
:10108000750D9093760DA093770DB093780D8093A6
:10109000790D90937A0DA0937B0DB0937C0D809386
:1010A0007D0D90937E0DA0937F0DB093800D1092D7
:1010B000810D1092820D1092830D1092840D10926A
:1010C000850D1092860D1092870D1092880D8AE082
:1010D00097EDA3EABDE38093630790936407A09321
:1010E0006507B093660780E090E0A0E2B1E48093EA
:1010F000FD059093FE05A093FF05B09300060E94A6
:101100009A2A8CE0EEEAF1E0DE01119601900D9250
:101110008A95E1F789819A81AB81BC8180931D1307
:1011200090931E13A0931F13B09320138D819E8163
:10113000AF81B8858093211390932213A09323133A
:10114000B093241389859A85AB85BC85809325133C
:1011500090932613A0932713B09328138EEB90E05F
:101160009093A9048093A8041092AB041092AA044F
:1011700086EE90E09093AD048093AC041092AF049F
:101180001092AE048FE892ECADE8B1E480938D123A
:1011900090938E12A0938F12B09390128CE998EFD7
:1011A000A5E4BEE38093911290939212A0939312C0
:1011B000B093941281E49CEBABECB3E48093951272
:1011C00090939612A0939712B09398121092DB0608
:1011D0001092DA0607DF33DE0E94403E82E191E2A0
:1011E0000E9499342C96E2E00C94A3EE05CFA4E083
:1011F000B0E0EDEFF8E80C9478EE9091DD069817EA
:1012000009F455C0382E80E090E0A0E2B1E4898373
:101210009A83AB83BC83C0902513D0902613E090B3
:101220002713F090281320E030E0A901C701B60190
:101230000E9491E787FF0CC0A701960160E070E073
:1012400080E291E40E94AEEE69837A838B839C8373
:10125000CE0101960E944BC34090720150907301E1
:101260006090740170907501809076019090770184
:10127000A0907801B09079013320F1F00E94193FDD
:1012800019821A821B821C82E0907A01F0907B0105
:1012900000917C0110917D01CE0101966C01A501A8
:1012A0009401C301B201B1DC3092DD069BDE80E027
:1012B0002496E1E10C9494EE0E94D83EE1CFB0E098
:1012C000A0E0E5E6F9E80C9479EEC82FE82EF12CC1
:1012D000F701EA58F04DD491823071F481E087DF54
:1012E000811105C00E94193F882309F4E2C0CDB7DF
:1012F000DEB7E0E10C9495EE6D2FDD0F770B880BD8
:10130000990B0E9497E72B013C01C701880F991F99
:10131000880F991F895B924E0E94FA274B015C014E
:10132000A3019201C501B4010E94F6E74B015C01E3
:101330006701CC0CDD1CCC0CDD1CC601855C924E1B
:101340000E94FA27A30192010E94F6E720E030E014
:1013500040EC5FE30E94F6E7AB01BC0100E010E067
:1013600098018C2F0E94A1C6C23009F0CCC00E9407
:10137000D83E20E030E0A901C501B4010E9491E708
:10138000882329F100E010E020E830E4B501A40151
:1013900070588C2F0E94A1C6C23009F467C0A50105
:1013A0009401C501B4010E94AFEE4B015C01C23053
:1013B00009F062C000E010E020E030E4B501A401D3
:1013C0008C2F0E94A1C6C23011F40E94D83E81E049
:1013D00090E00C2E01C0880F0A94EAF790914F0715
:1013E000982B90934F079091EF05892B8093EF05F1
:1013F000C601815D924E0E94FA27F601EE58FE4F1B
:101400006083718382839383C230D1F4209125134A
:1014100030912613409127135091281360917A013F
:1014200070917B0180917C0190917D010E94AEEED4
:1014300060937A0170937B0180937C0190937D018E
:1014400092DCF601ED57FB4FD601AE58BE4F8D91A1
:101450009D910D90BC91A02D80839183A283B38335
:10146000C23009F044CF0E94002841CF0E94193FAA
:10147000882309F494CF3BCFF701E45DF24E6491E9
:10148000611107C00E94403E8AE09DE10E949934AC
:101490006AE070E090E080E00E9495E79B01AC017B
:1014A00061E070E088E492E40E9429EF8B019C01E6
:1014B00085CF8FE49DE10E94FA2720E030E0A9016A
:1014C0000E9491E7882309F417CF6D2FDD0F770B6A
:1014D000880B990B0E9497E72B013C018FE49DE15B
:1014E0000E94FA274B015C0120E030E040EA50E422
:1014F0000E944EF087FF14CF812C912C90EAA92EE8
:1015000090E4B92E0DCF20E030E0A901C501B4016F
:101510000E9491E7882309F45ACF00E010E0980177
:1015200035CF80912107882319F010922107089563
:1015300040E070E060E08AE69CE10E94603F1F921C
:101540000F920FB60F9211240BB60F922F933F9369
:101550004F935F936F937F938F939F93AF93BF93BB
:10156000EF93FF930E94A376FF91EF91BF91AF910C
:101570009F918F917F916F915F914F913F912F91AB
:101580000F900BBE0F900FBE0F901F9018950F93EA
:101590001F9380915F07813019F50E94E0CC009184
:1015A000D4051091D5052091D6053091D705601B43
:1015B000710B820B930B28EE33E040E050E00E9469
:1015C000BFED6091D0057091D1058091D2059091C9
:1015D000D305620F731F841F951F1F910F910895EC
:1015E0006091D8057091D9058091DA059091DB055D
:1015F000D6CF10925F071092D4051092D5051092A5
:10160000D6051092D7051092D8051092D9051092E0
:10161000DA051092DB051092D0051092D1051092D8
:10162000D2051092D305089580915F078130E1F0D3
:101630008230C1F4ACDF6093D0057093D105809304
:10164000D2059093D30581E080935F070E94E0CCA0
:101650006093D4057093D5058093D6059093D705F4
:1016600081E00895C6DFEFCF80E008950E9499C31E
:101670000E944B2C882351F08091981482FD06C063
:101680008FED97E19093E0068093DF06CDCF8091B8
:101690005F07813079F482E080935F070E94E0CC9D
:1016A0006093D8057093D9058093DA059093DB0594
:1016B00081E0089580E0089580915F078150823035
:1016C00070F410925F070E94E0CC6093D80570938D
:1016D000D9058093DA059093DB0581E0089580E0D9
:1016E00008959C0197FF26C0EE27FF27E81BF90B02
:1016F0002D398FEF38070CF05DC08DE280937E04AA
:10170000CF0164E670E00E9449EECB012AE030E0B0
:10171000B9010E9449EE805D80937F04CF01B90139
:101720000E9449EECB01B9010E9449EE805D809391
:1017300080042AC0283E83E03807B4F1C90168EE6E
:1017400073E00E9449EECB01EAE0F0E0BF010E94A5
:1017500049EE805D80937E04C90164E670E00E94DA
:1017600049EECB01BF010E9449EE805D80937F046A
:10177000C901BF010E9449EECB01BF010E9449EEA1
:10178000805D80938004F901CF016AE070E00E94DF
:1017900049EE805D809381048EE794E008958DE2A8
:1017A00037FDC5CF80E2C3CFF90180E22436310591
:1017B0000CF0A4CF80E280937E0480937F04EA3013
:1017C000F1056CF38DE237FF80E280937F04CF0157
:1017D0006AE070E00E9449EE605D60938004D4CFBF
:1017E0009C0197FD2DC080E2243631055CF0C901D3
:1017F00064E670E00E9449EECB016AE070E00E946E
:1018000049EE805D80937F0480E22A3031055CF0F0
:10181000EAE0F0E0C901BF010E9449EECB01BF013F
:101820000E9449EE805D80938004C9016AE070E007
:101830000E9449EE805D809381048FE794E00895D3
:101840003195219531098DE2DDCFCF92DF92EF9274
:10185000FF92FC01C080D180E280F38020E030E084
:10186000A901C701B6010E9491E787FD26C06DEB73
:1018700077E386E095E3A70196010E94AFEE6B0146
:101880007C0120E030E0A9010E9491E720E030E0F7
:1018900040E05FE387FF04C020E030E040E05FEB22
:1018A000C701B6010E94AFEE0E9491EFCB0198DF15
:1018B000FF90EF90DF90CF9008956DEB77E386E097
:1018C00095EBD9CFA4E0B0E0E8E6FCE80C9487EE15
:1018D0000E9497E769837A838B839C83CE0101966C
:1018E000B4DF2496E2E00C94A3EEFC0160817181E8
:1018F000828193810E9491EFCB0172CFA4E0B0E08E
:10190000E4E8FCE80C9487EE0E9497E769837A8309
:101910008B839C83CE010196E8DF2496E2E00C9451
:10192000A3EE8F929F92AF92BF92EF92FF920F938E
:101930001F93CF93DF93EC018B01E42EF22E809165
:101940004013909141138C179D07C9F121EAC334CC
:10195000D20709F03FC089559C4271F40E94E0CC47
:101960006E517B4F8F4F9F4F6093C0057093C105A1
:101970008093C2059093C305D0934113C093401345
:1019800030E020E000934207109343072093440780
:1019900030934507E0923D07F0923E07C955DC427F
:1019A00021F410927A041092BF0582E080936701BF
:1019B00081E080933F07109279041092CB05DF916C
:1019C000CF911F910F91FF90EF90BF90AF909F909C
:1019D0008F9008952CE2C935D20771F68354914A4D
:1019E000D9F40E94E0CC8090C0059090C105A090F1
:1019F000C205B090C305681979098A099B0997FF48
:101A00000BC080914F078770873031F40E943E6B86
:101A1000CEEED9E98111B0CFC9E5DCE2ADCF20E04F
:101A200040E070E060E08DE29BE67BCF0E946CB30B
:101A3000882339F020E040E070E060E080E199E93F
:101A400070CFEDCF21E020937A04FC018081918159
:101A5000A281B3818093310190933201A09333012D
:101A6000B093340120E040E070E060E080912C070A
:101A700090912D0756CFA4E0B0E0E1E4FDE80C948E
:101A800087EE8DEC9CECACECBCE389839A83AB8352
:101A9000BC83CE010196D6DF2496E2E00C94A3EE3F
:101AA000A4E0B0E0E6E5FDE80C9487EE8DEC9CEC5C
:101AB000ACECBDE389839A83AB83BC83CE010196F2
:101AC000C1DF2496E2E00C94A3EEA4E0B0E0EBE6E4
:101AD000FDE80C9487EE80E090E0A0E8BFE3898306
:101AE0009A83AB83BC83CE010196ACDF2496E2E0FF
:101AF0000C94A3EEA4E0B0E0E0E8FDE80C9487EEDF
:101B000080E090E0A0E2B1E489839A83AB83BC8358
:101B1000CE01019697DF2496E2E00C94A3EE81E0DB
:101B200080937A0480914F078770873051F010922C
:101B30004F071092EF0584E09CE19093E0068093BC
:101B4000DF0680919F048093CD0580E00E94582A93
:101B500020E040E070E060E08FEA9DE8E2CE809116
:101B60006701882331F041E06AE979E182E00E946F
:101B70004EC78091EF058770873071F41092CC05C5
:101B800020E040E070E060E080E999E9CADE81E0B1
:101B90008093CB050C947E6A089520E040E070E0CD
:101BA00060E089E59CE2BDCE10927F070E94EE6F57
:101BB000F4CFCF93DF93C0912307C7FD1FC084E00C
:101BC000C802E0011124FE01E855FB4F808191819C
:101BD000181619063CF4863F910514F085EF90E045
:101BE0000E9421CDC855DB4F8A819B818F3F910593
:101BF00019F010F08FEF90E080937F07CEDFDF9138
:101C0000CF910895B0E0A0E0E8E0FEE80C9481EE0A
